:100000000C94C8480C943C490C943C490C943C49D1
:100010000C943C490C943C490C943C490C943C494C
:100020000C943C490C943C490C943C490C943C493C
:100030000C943C490C9499490C94D9490C943C4932
:100040000C943C490C943C490C943C490C943C491C
:100050000C943C490C943C490C943C490C943C490C
:100060000C943C490C943C490C943C490C943C49FC
:100070005A5501200101003808000000000000006E
:100080000000000000000000000000000000000070
:100090008100450027FF24FF2A902B1C210C22FB06
:1000A000850084008903888D81096F0244424700DE
:1000B0004501B083B300B10125118A4F8B03AD4DCB
:1000C000B04D7F4ECC51C451B14DB64DBB4DB25128
:1000D000BE4DC14DC44D084E00020800085504082D
:1000E0005A0000F8000990000A1E32050000FF00C7
:1000F0000000D80000000000000000000000000028
:1001000000000000000000000000000000000000EF
:1001100000000000000000000000000000000000DF
:1001200000000000000000000000000000000000CF
:1001300000000000000000000000000000000000BF
:10014000000000000000000000000049000000491D
:100150005252000052525C2D0000000000000000CE
:1001600000000000000000000040000000494A526A
:10017000004952525B1C52531C25241B2425251B6D
:100180000A0A2D1C12120A0A0000000000000000DA
:10019000404949494949525B5B5B525B1C1C131245
:1001A000241C1209090912090909090A0A0A0A0A7A
:1001B0000A13120A0A12130A0000000000009252E9
:1001C0005252525213121309001C0A1212401B659C
:1001D000090A0009241B120000251C1C010025240B
:1001E0001C1C002425242424000000000000524987
:1001F000494000001B1352494900641C1C5B4A48DB
:100200001C651C2552491C1C652464491C1C652561
:1002100064491C1C6D2E5C490000000000000000B9
:100220000000004900000000535200000053522516
:1002300000004A52252500005B251300005B530097
:100240000A1C095B1C657F374052522E2E1C525CE3
:100250002E251B1324251C1C12002525120000121C
:100260001B0000132E37001B37372E2E37372E2E4C
:100270002E2E2E2E6E6E6E1C1313120009131200FA
:10028000001213130012251C13132E371C13131303
:10029000361C131B1B1B25131C1C1B1B1B1C1C1C93
:1002A0001C1C1C1C1C1C1C131312121313001313F4
:1002B000131C000913131C010037131C13002E2EEE
:1002C0001C1C001C772E2500137F251C010A3724D7
:1002D0001C1C0A2E25250900132E242525252E2534
:1002E0002525252525252D2E251B2E2E251C1325C0
:1002F000251C1C1C1C011C1C1300011C0A00016590
:10030000775C016E7F6E521B25256D1C5249252599
:100310001C1353001C1C1C524A001B135B5B000087
:1003200009525C0000005B5C000000001B00000044
:100330000000000000000000135B7F776E6E136505
:1003400077766E6E1B65777676761B5BBF76B676B4
:1003500009136DBFB7B6001B125C76BF0000121BFD
:10036000125B00000000090A6E6E6E77241C6E6E30
:1003700077251C1C6E776E1C1C1C76761C1C242595
:10038000B765646D6D1B766D6D5B09125B5C5B120E
:100390005B641213131B12121C1C1C1C1C241C1C3F
:1003A000242525242425251B00002513000064BFD7
:1003B00000096EBFBF6D6EBF6D5B12135B1213122F
:1003C00009000901000000002E1C0900096E01004F
:1003D00009767F7F12777F7F6412BF775B121B09DC
:1003E0005B121B0900001B09000000000000000058
:1003F00000000000000000007F7F53131300641210
:100400001B0100001B1200000000000000000000A3
:1004100000000000000000000000000000000000DC
:1004200000000000000000000000000000002600A6
:10043000000026002F0000002F00370000003700CA
:10044000FF000000FF00BF000000BF0037000037C2
:100450000000002626000000000000000000262604
:1004600026262600000000002F00000000370000B4
:100470000000FF00000000BF000000003700000087
:100480000000262626262600000000000000262662
:10049000262626002F000000000037000000000084
:1004A000FFFFFFFF0000BF0000000000370000005A
:1004B0000000262626262600000000000000262632
:1004C000262600002F0000002F0037000000370014
:1004D000FFFFFFFF0000BF000000BF00370000006B
:1004E000370026262626000000000000000000003D
:1004F00026262600002F00002F00370000003700BE
:10050000FF000000FF00BF000000BF003700003701
:100510000000262626000000000000000000260043
:10052000000026002F0000002F00003700370000D9
:100530000000FF00000000BF00BF00003700000007
:100540003700260000002600000000000000000028
:10055000000000000000000000000000000000009B
:1005600000000000000000000000009B000000529E
:100570009BA400005B9B6D77000000000000000062
:100580000000000000000000005B000000E4F6FF37
:10059000099BEDF6FFBFA4ADBFBFBFBF767F7FB79E
:1005A000B7BF7F766EB7B7BF000000000000000045
:1005B0005BB6F6F6F6FFFFFFFFBFFFFFFFBFBFAE64
:1005C000FFFFFFB7AD65FFFFB7B6AD65FFFFBFB774
:1005D000AE6EFFFFBFB7B765000000000000F6F683
:1005E000EDEDADA4B66D6D5C526E656565526576D8
:1005F0005C5C52536E246552526E25255B52772DFA
:100600002525526E6E2D2525000000000000A49BBC
:100610009B4900006564A49B92006D252564934965
:10062000656E652E9B5224256D25655225246D2D02
:10063000655225256E2E6452000000000000000067
:100640000000004A000000005B9B0000005B5B2D87
:100650000000525B2E2E00015B2D1C01005C5B0133
:100660004A654A5B1C6E7F77495B9B77776D5B655C
:10067000776E65656D2D25255C522E25130949641D
:100680001C09095C7F7F091C7F7F777F777F7777E5
:100690007F7F7776777F7F6E656E6EA4B6FF655B32
:1006A000A4B7BFFF526DBFBFBFFF7FBFBFBFBFFFBC
:1006B000BFBFB7BFFFFF7FB7BFBFFFFF6EB7BFBFF3
:1006C000FFFF77BFBFBFFFFFFFFFBFBFB75BFFFFEE
:1006D000BFBFA464FFFFBFADA47FFFFFBFA4BF7F68
:1006E000FFBFADBFBFBFFFB6BFBFBF77F7BFBFBFC5
:1006F0007777FFBFBFBF64526D7F6E2E2D2D7F7643
:100700006E6E6E2E777777762E1C7F776E251C2582
:10071000776525251C096E6E1C0949255B494A6EC3
:100720007F645377BF775B5C256E6E255B4A2565DA
:100730001C1B5B002524245B53001C1B5B5C00001E
:100740000A5B640000006464000000005C000000BC
:1007500000000000000000005B5C7FBF77765C6DEE
:100760007FB777775C6D7FBF77775C64BFBFBFBFB4
:100770000A5C6EBFBFBF0065646DBFBF00005B6DEC
:10078000646D00000000125B7777777F6E6E77777D
:100790007F766D7677BF776D6E76BF7F6D6E767F75
:1007A000BF7676BFBF76BFBFBFB664ADADB6B6ADE0
:1007B000BFFF646DADB6AD6477BFBFBFFFFF77BF4E
:1007C000BFBFFFFF7FBFBFBFFFF6BFB7ADF6FFFFE5
:1007D000A4ADFFFFFFFFFFFFFFFFFFFFFFFFFFF6DF
:1007E000A4005B5200000000BFBFAD5B64BFB6ADAC
:1007F000ADBFFFBFFFFFFFFFBF64FFFFBFB6765B6C
:10080000FFBFBF5B0000FF5C0000000000000000B5
:100810000000000000000000BFBF645C5C006E5C74
:10082000654900006D5B0000000000000000000052
:1008300000000000000000000000000000000000B8
:10084000000000000000000006000400000001009D
:10085000020003000400050006000700080009006C
:100860000A000B000C000D000E000F00100000002D
:1008700011001200130014001500160006000300FA
:1008800000001700180019001A001B001C001D00B2
:100890001E001F002000210022002300240025004C
:1008A0002600000000408891D2E4ADB5B6BEBFFF7F
:1008B0003230313320444F4D494E494B20274B496C
:1008C0004C4F27204B52495354454E005448452025
:1008D000555A45424F58205355424D4152494E4575
:1008E0002053494D554C4154494F4E0042454152C9
:1008F000494E473A00535441525400544152472EF6
:10090000444953542E3A0053455420444953542EDD
:100910003A004C4556454C004252494546494E47DF
:10092000004845414C54480053434F52450047410D
:100930004D45204F564552212100505245535320DA
:10094000535441525400524144415200534849507B
:10095000533A00444946464943554C543A20454190
:10096000535920202000444946464943554C543AA7
:100970002041564552414745004449464649435562
:100980004C543A20484152442020200047414D45D4
:100990002053504545443A20534C4F5720200047A0
:1009A000414D452053504545443A204E4F524D410C
:1009B0004C0047414D452053504545443A2046415F
:1009C000535420200000B0075A00B1076500C20050
:1009D00000B2076500C30100B3075001C2180092BE
:1009E00030760CC3190293247610C1180291377621
:1009F00020370004387622C01802903F7681269274
:100A0000300007913800079324000092307612904E
:100A10003F0000932476129136761F360005377614
:100A200024903E7681229230001293240000913768
:100A3000000092307612903E000093247612913698
:100A4000761F360005377624903D7681229230005D
:100A500012932400009137000092307612903D00EE
:100A600000932476129135761F3500053776249051
:100A70003C7681223C0009923000099324000090CA
:100A80003F7B0092307B1293247B1F903F00053EFA
:100A90007B0E3E00043C7B0E3C00043E7B0E3E0081
:100AA000043F7B0E3F0004437B0F932400039043DD
:100AB00000009230000090467B00923E7B09932B11
:100AC0007B2D90460000457B0F450003437B11437F
:100AD0000001457B0E450004467B0D9137000290D6
:100AE000460002923E0000904A7B05913E76003E11
:100AF000760C932B0001904A00004D5C00923A7BEB
:100B000009932E766A913E00093E0009904D000936
:100B1000932E0005923A000090417B0091397600B7
:100B200092327B0993267B2890410005407B0F4041
:100B300000033E7B0D3E0005407B0D400005417BE0
:100B40000F410003457B0C93260001923200029076
:100B5000450003487B0092407B09932D7B2B9048F6
:100B60000002477B0E470004457B0F450003477B8F
:100B70000E470004487B0E48000491390000904C59
:100B80007B0992400009904C0000932D0000904397
:100B90006A00913C760092307B1293247B6C9043E8
:100BA000000492300005913C00099324000092302B
:100BB0007912932479129137791F370005387924F7
:100BC000903F7981259230000F93240000913800E6
:100BD0000092307912903F00009324791291367977
:100BE0001F360004377924903E7981279230000D1A
:100BF000913700009230790193240011903E00005B
:100C00009324791291367920360004377924903D67
:100C10007981269230000C932400029137000092D3
:100C2000307912903D000093247912913579203566
:100C30000004377924903C79813093240004923069
:100C4000000091370000903C0000FF2F00000000E2
:100C50000000000000000000000000000000000094
:100C60000000000000000000000000000000000084
:100C7000000000000000000000000000000000FF75
:100C800000000000FFFFFF000000FFFFFF0000006A
:100C900000FF0000000000FF000000000000000056
:100CA000000000FF000000000000000000FFFF0047
:100CB000FFFF00FFFF00FFFF00FF0000FF0000003C
:100CC0000000000000000000000000000000000024
:100CD0000000000000000000000000000000000014
:100CE00000000000FF00FF0000FFFFFFFFFF00000B
:100CF000FF00FF000000FF00FF0000FFFFFFFFFFFD
:100D00000000FF00FF000000000000000000FF00E6
:100D100000000000FFFFFF0000FF000000000000D7
:100D2000FFFF000000000000FF0000FFFFFF0000C9
:100D3000000000FF000000000000000000FFFF00B6
:100D400000FF00FFFF0000FF00000000FF000000A8
:100D500000FF00000000FF00000000FF0000FFFF98
:100D600000FF0000FFFF0000000000000000FF0087
:100D7000000000FF00FF000000FF00FF0000000077
:100D8000FF00000000FF00FF00FF00FF0000FF0069
:100D90000000FFFF00FF0000000000000000FFFF58
:100DA00000000000FFFF00000000FF000000000046
:100DB0000000000000000000000000000000000033
:100DC000000000000000000000000000000000FF24
:100DD00000000000FF0000000000FF000000000015
:100DE000FF0000000000FF0000000000FF00000006
:100DF000000000FF00000000000000000000FF00F5
:100E00000000000000FF0000000000FF00000000E4
:100E100000FF0000000000FF0000000000FF0000D5
:100E20000000FF00000000000000000000000000C3
:100E300000000000FF00FF000000FFFFFF0000FFB8
:100E4000FFFFFFFF0000FFFFFF000000FF00FF00AB
:100E50000000000000000000000000000000000092
:100E60000000000000FF0000000000FF000000FF85
:100E7000FFFFFFFF000000FF0000000000FF000078
:100E80000000000000000000000000000000000062
:100E90000000000000000000000000000000000052
:100EA000000000000000000000000000FFFF000044
:100EB0000000FFFF00000000FF0000000000000035
:100EC000000000000000000000000000000000FF23
:100ED000FFFFFFFF00000000000000000000000016
:100EE0000000000000000000000000000000000002
:100EF00000000000000000000000000000000000F2
:100F0000000000000000000000000000FFFF0000E3
:100F10000000FFFF000000000000000000000000D3
:100F200000000000000000FF00000000FF000000C3
:100F300000FF00000000FF00000000FF00000000B4
:100F400000000000000000000000000000002F2F43
:100F50002F00002F0000002F002F00002F2F002F48
:100F6000002F002F002F2F00002F002F0000002F38
:100F700000002F2F2F000000000000000000002FB5
:100F8000000000002F2F00000000002F00000000D4
:100F9000002F00000000002F00000000002F0000C4
:100FA00000002F2F2F0000000000000000002F2F56
:100FB0002F00002F0000002F00000000002F000075
:100FC000002F2F0000002F000000002F0000000065
:100FD000002F2F2F2F2F00000000000000002F2FC8
:100FE0002F00002F0000002F00000000002F000045
:100FF0002F2F2F0000000000002F002F0000002FD7
:1010000000002F2F2F000000000000000000000053
:101010002F000000002F2F0000002F002F00002FB6
:1010200000002F00002F2F2F2F2F000000002F0077
:10103000000000002F00000000000000002F2F2FF4
:101040002F2F002F00000000002F00000000002FB5
:101050002F2F2F0000000000002F002F0000002F76
:1010600000002F2F2F000000000000000000002FC4
:101070002F0000002F000000002F00000000002FB4
:101080002F2F2F00002F0000002F002F0000002F17
:1010900000002F2F2F00000000000000002F2F2F36
:1010A0002F2F00000000002F000000002F00000084
:1010B000002F000000002F00000000002F000000A3
:1010C00000002F00000000000000000000002F2F93
:1010D0002F00002F0000002F002F0000002F000025
:1010E0002F2F2F00002F0000002F002F0000002FB7
:1010F00000002F2F2F0000000000000000002F2F05
:101100002F00002F0000002F002F0000002F0000F4
:101110002F2F2F2F00000000002F000000002F00B5
:1011200000002F2F00000000000000000000000061
:1011300000000000000000000000FFFF00000000B1
:10114000FFFF00000000000000000000FFFF0000A3
:101150000000FFFF00000000000000000000000091
:1011600000000000000000000000FFFF0000000081
:10117000FFFF00000000000000000000FFFF000073
:101180000000FFFF00000000FF0000000000000062
:1011900000FF00000000FF00000000FF0000000052
:1011A000FF000000000000FF000000000000FF0042
:1011B0000000000000FF0000000000000000000030
:1011C000000000000000000000FFFFFFFFFF000024
:1011D0000000000000000000000000FFFFFFFFFF14
:1011E0000000000000000000000000000000FF0000
:1011F0000000000000FF000000000000FF000000F1
:10120000000000FF00000000FF00000000FF0000E1
:101210000000FF0000000000000000000000FFFFD1
:10122000FF0000FF000000FF0000000000FF0000C2
:1012300000FFFF00000000FF0000000000000000B1
:10124000000000FF00000000000000000000FFFFA1
:10125000FF0000FF000000FF00FF00FFFFFF00FF96
:1012600000FF00FF00FF00FFFFFF00FF0000000085
:101270000000FFFFFF000000000000000000FFFF73
:10128000FF0000FF000000FF00FF000000FF00FF64
:10129000000000FF00FFFFFFFFFF00FF000000FF56
:1012A00000FF000000FF00000000000000FFFFFF43
:1012B000FF0000FF000000FF00FF000000FF00FF34
:1012C000FFFFFF0000FF000000FF00FF000000FF25
:1012D00000FFFFFFFF000000000000000000FFFF14
:1012E000FF0000FF000000FF00FF0000000000FF03
:1012F0000000000000FF0000000000FF000000FFF1
:101300000000FFFFFF0000000000000000FFFFFFE3
:10131000FF0000FF000000FF00FF000000FF00FFD3
:10132000000000FF00FF000000FF00FF000000FFC2
:1013300000FFFFFFFF0000000000000000FFFFFFB4
:10134000FFFF00FF0000000000FF0000000000FFA2
:10135000FFFFFF0000FF0000000000FF0000000092
:1013600000FFFFFFFFFF00000000000000FFFFFF85
:10137000FFFF00FF0000000000FF0000000000FF72
:10138000FFFFFF0000FF0000000000FF0000000062
:1013900000FF000000000000000000000000FFFF50
:1013A000FF0000FF000000FF00FF0000000000FF42
:1013B00000FFFFFF00FF000000FF00FF000000FF34
:1013C0000000FFFFFFFF00000000000000FF000022
:1013D00000FF00FF000000FF00FF000000FF00FF13
:1013E000FFFFFFFF00FF000000FF00FF000000FF05
:1013F00000FF000000FF0000000000000000FFFFF1
:10140000FF00000000FF0000000000FF00000000DF
:1014100000FF0000000000FF0000000000FF0000CF
:101420000000FFFFFF0000000000000000000000BF
:1014300000FF0000000000FF0000000000FF0000AF
:10144000000000FF00FF000000FF00FF000000FFA1
:101450000000FFFFFF0000000000000000FF000090
:1014600000FF00FF0000FF0000FF00FF000000FF82
:10147000FF00000000FF00FF000000FF0000FF0071
:1014800000FF000000FF00000000000000FF00005F
:10149000000000FF0000000000FF0000000000FF4F
:1014A0000000000000FF0000000000FF000000003E
:1014B00000FFFFFFFFFF00000000000000FF000032
:1014C00000FF00FFFF00FFFF00FF00FF00FF00FF25
:1014D000000000FF00FF000000FF00FF000000FF11
:1014E00000FF000000FF00000000000000FF0000FF
:1014F00000FF00FFFF0000FF00FF00FF00FF00FFF4
:101500000000FFFF00FF000000FF00FF000000FFE1
:1015100000FF000000FF0000000000000000FFFFCF
:10152000FF0000FF000000FF00FF000000FF00FFC1
:10153000000000FF00FF000000FF00FF000000FFB0
:101540000000FFFFFF0000000000000000FFFFFFA1
:10155000FF0000FF000000FF00FF000000FF00FF91
:10156000FFFFFF0000FF0000000000FF0000000080
:1015700000FF000000000000000000000000FFFF6E
:10158000FF0000FF000000FF00FF000000FF00FF61
:10159000000000FF00FF00FF00FF00FF0000FF0051
:1015A0000000FFFF00FF00000000000000FFFFFF41
:1015B000FF0000FF000000FF00FF000000FF00FF31
:1015C000FFFFFF0000FF0000FF0000FF000000FF22
:1015D00000FF000000FF0000000000000000FFFF0F
:1015E000FF0000FF000000FF00FF000000000000FF
:1015F000FFFFFF000000000000FF00FF000000FFF1
:101600000000FFFFFF0000000000000000FFFFFFE0
:10161000FFFF000000FF0000000000FF00000000CE
:1016200000FF0000000000FF0000000000FF0000BD
:10163000000000FF000000000000000000FF0000AC
:1016400000FF00FF000000FF00FF000000FF00FFA0
:10165000000000FF00FF000000FF00FF000000FF8F
:101660000000FFFFFF0000000000000000FF00007E
:1016700000FF00FF000000FF00FF000000FF00FF70
:10168000000000FF00FF000000FF0000FF00FF005F
:10169000000000FF000000000000000000FF00004C
:1016A00000FF00FF000000FF00FF00FF00FF00FF41
:1016B00000FF00FF00FF00FF00FF00FF00FF00FF32
:1016C0000000FF00FF0000000000000000FF00001D
:1016D00000FF00FF000000FF0000FF00FF0000000F
:1016E00000FF00000000FF00FF0000FF000000FFFF
:1016F00000FF000000FF00000000000000FF0000ED
:1017000000FF00FF000000FF00FF000000FF0000DE
:10171000FF00FF00000000FF0000000000FF0000CD
:10172000000000FF000000000000000000FFFFFFBD
:10173000FF0000000000FF00000000FF00000000AC
:10174000FF00000000FF0000000000FF000000009C
:1017500000FFFFFFFF00000000000000000000FF8E
:10176000FF000000FF0000000000FF00000000FF7D
:10177000FF0000000000FF0000000000FF0000006C
:10178000000000FFFF00000000000000000000FF5C
:10179000FF000000FF0000FF00FF00FFFF00FFFF51
:1017A00000FF0000FFFF00FFFF00FF00FF0000FF41
:1017B000000000FFFF000000000000000000FFFF2D
:1017C000000000000000FF0000000000FF0000001B
:1017D0000000FFFF00000000FF0000000000FF000D
:1017E0000000FFFF00000000000000000028001CB7
:1017F00000190019001900190019001900430044CC
:10180000004500460047004800490049004A004B97
:10181000004B004C004D004D004D004E004B004B66
:101820000049004900490049004F0047005000515D
:10183000005200530019001900190019001900196D
:10184000001900190054005500560057004D004D76
:10185000004D004D004D004D004D004D004D004D20
:1018600000580059005A005B005C005B005D004DB1
:10187000004D004D004D004D004D004D004D004D00
:10188000004D004D005E005F005300190019001963
:10189000001900600061004D004D004D004D004DED
:1018A000004D004D004D004D004D004D00620063A5
:1018B0000064006500650065006500650066006302
:1018C0000067004D004D004D004D004D004D004D96
:1018D000004D004D004D004D006800190019001921
:1018E00000190069004D004D006A006B006C006D2E
:1018F000006E006F0070007100720073007300735F
:101900000073007300740075007600730073007339
:1019100000730077007200780079007A007B007C09
:10192000007D007E007F004D008000190019001925
:101930000019006900810082008300840084008413
:101940000084008400850086008700880089008A62
:10195000008B008C008D008E0086008F009000911F
:101960000087008700870092009300840084008431
:1019700000840094001900950096001900190019C0
:10198000001900970098005300190099009A009BD5
:1019900000840084009C0087008700870087008700
:1019A00000870087009D009E0087008700870087D2
:1019B000008700870087008700930084009F00A0B5
:1019C00000A100A2001900A300A400190019001929
:1019D00000190019001900A500A600A700A800A979
:1019E00000AA00AB00AC00AD00AE00AE00AE00AE91
:1019F00000AE00AE00AF00B000AD00AE00AE00AE75
:101A000000AE00AE00AE00B100B2001900B300B4E9
:101A100000B500B600B700B8001900190019001988
:101A200000B900BA00BA00BA00BA00BA00BA00BBE6
:101A300000BC00BD00BE00BF008700870087008794
:101A4000008700870087008700870087008700875E
:101A500000870087008700C000C100C200C300C427
:101A600000C400C400C400C400C400C500C60019FE
:101A70000024001900190019001900190019001993
:101A8000001900C700C800C90087008700870087C9
:101A900000CA00CB00CC00CD00CE00CF008700876D
:101AA00000870087008700D000D100D200190019FC
:101AB0000019001900190019001900D300D40019E9
:101AC0000024001900190019001900190019001943
:101AD000001900C700D500D600D700D700D700D71F
:101AE00000D700D700D700D700D700D700D700D73E
:101AF00000D700D700D700D800D900D200190019AC
:101B00000019001900190019001900D300D4001998
:101B100000240019001900190019001900190019F2
:101B2000001900C700DA00DB00DC00DD00DE00DFAA
:101B300000E000E100E200E300E000E100E400E595
:101B400000E500E500E500E600E700D20019001915
:101B50000019001900190019001900D300D4001948
:101B600000240019001900190019001900190019A2
:101B7000001900C700DA00E80001000100010001BF
:101B8000000100010001000100010001000100014D
:101B900000010001000100E900E700D2001900196E
:101BA0000019001900190019001900D300D40019F8
:101BB0000024001900190019001900190019001952
:101BC000001900C700DA00EA00010001000100016D
:101BD00000010001000100010001000100010001FD
:101BE00000010001000100E900E700D2001900191E
:101BF0000019001900190019001900D300D40019A8
:101C000000EB00EC00EC00EC00EC00EC00EC00EC75
:101C100000EC00ED00DA00EE00010001000100011F
:101C200000010001000100010001000100010001AC
:101C300000010001000100E900E700EF00EC00EC0A
:101C400000EC00EC00EC00EC00EC00F000F10019FE
:101C500000190019001900190019001900190019BC
:101C600000F200F200F300F40001000100010001A5
:101C7000000100010001000100010001000100015C
:101C800000010001000100E900F500F600F600F790
:101C9000001900190019001900190019001900197C
:101CA0000019001900190019001900F800F900FACC
:101CB0000087008700FB00EE00000000000000002D
:101CC0000000000000000000000000000000000014
:101CD00000000000000000E900FC0087008700878A
:101CE00000FD00FE00190019001900190019001963
:101CF0000019001900190019001900D30087008786
:101D00000087008700FB00EE0000000000000000DC
:101D100000000000000000000000000000000000C3
:101D200000000000000000E900FC00870087008739
:101D3000008700FF00190019001900190019001987
:101D40000019000001010101010101020187008762
:101D50000087008700FB00E8000000000000000092
:101D60000000000000000000000000000000000073
:101D700000000000000000E900FC008700870087E9
:101D8000008700030101010101010104011900198B
:101D900000190005010501050105010601870087FD
:101DA0000087008700FB00E8000000000000000042
:101DB0000000000000000000000000000000000023
:101DC00000000000000000E900FC00870087008799
:101DD000008700070105010501050105011900192A
:101DE00000190008010901090109010A010B018715
:101DF0000087000C010D010E010F010F010F010FF3
:101E0000010F010F010F010F010F010F010F010F52
:101E1000010F010F010F011001110112018700874D
:101E20000013011401090109010901150119001923
:101E300000190019001900190019001900160117DE
:101E400001170117011701180121002100210021AC
:101E5000002100210021002100210021002100217A
:101E60000021002100210019011701170117011796
:101E7000011A011900190019001900190019001997
:101E800000B900BA00BA00BA00BA00BA00BA00BA83
:101E900000BA00BA00BA00BA00BA00BA00BA00BA72
:101EA00000BA00BA00BA00BA00BA00BA00BA00BA62
:101EB00000BA00BA00BA00BA00BA00BA00BA00BA52
:101EC00000BA00BA00BA00BA00BA00BA001B011981
:101ED000002400190019001900190019001900192F
:101EE000001900190019001900190019001900192A
:101EF000001900190019001900190019001900191A
:101F00000019001900190019001900190019001909
:101F1000001900190019001900190019001C0119F5
:101F200000240019001900190019001900190019DE
:101F300000190019001900190019001900190019D9
:101F400000190019001900190019001900190019C9
:101F500000190019001900190019001900190019B9
:101F6000001900190019001900190019001C0119A5
:101F7000002400190019001900190019001900198E
:101F80000019001900190019001900190019001989
:101F90000019001900190019001900190019001979
:101FA0000019001900190019001900190019001969
:101FB000001900190019001900190019001C011955
:101FC000001D011E011E011E011E011E011E011E1B
:101FD000011E011E011E011E011E011E011E011E09
:101FE000011E011E011E011E011E011E011E011EF9
:101FF000011E011E011E011E011E011E011E011EE9
:10200000011E011E011E011E011E011E011F0119DC
:1020100000190019001900190019001900190019F8
:1020200000190019001900190019001900190019E8
:1020300000190019001900190019001900190019D8
:1020400000190019001900190019001900190019C8
:1020500000190019001900190019001900190019B8
:1020600000190019001900190019001900190019A8
:102070000019001900190019001900190019001998
:102080000019001900190019001900190019001988
:102090000019001900190019001900190019001978
:1020A0000019001900190019001900190019001968
:1020B000002100090019002001210122012301242F
:1020C00001250126012701280129012A012B012CC4
:1020D000012D012E012F0130013101320133013474
:1020E000013501360137013801390139013A013B27
:1020F000013C013D013E0119003F01400141014207
:102100000143014401450146014701480149014A93
:10211000014B0100004C01000000004D01000000D7
:10212000004E014F0150015101520153015401551C
:102130000156015701580159015B015C015D010025
:10214000005E015F0160016101620163016401657C
:102150000166016701680169016A01000000000071
:102160000000006B016C016D01190019006E016F18
:10217000017001710172017301740119007501761A
:102180000100007701780179017A017B017C017DF2
:10219000017E017F01800181018201830100000035
:1021A0000000000000840185018601190019001952
:1021B0000019001900190087018801890119008B95
:1021C000018C0100008D018E018F0190019101921F
:1021D0000193019401950196019701980100000077
:1021E000000000000084019901190019001900196C
:1021F0000019001900190019009A019B019C01198E
:10220000009E019F01A001A101A201A301A401A5BB
:1022100001A601A701A801A901AA01AB01AC01AD6A
:1022200001AE01AF01B001B101B201B3011900B4B7
:1022300001B501B60119001900190019001900199A
:10224000001900B701B801B901BA01BB01BC01BD59
:1022500001BE01BF01C001BF01C101C201BF01C375
:1022600001C401C501C601C701C801C901CA01CB2A
:1022700001CC01CD01CE01CF01D001D101D201D3DA
:1022800001D401D601D701D801D901DA01DB01DC83
:1022900001DD01DE01DF01E001E101E201E301E432
:1022A00001E501E601E701E801E901EA01EB01ECE2
:1022B00001ED01EE01EF01F001F101F201F301F492
:1022C00001F501F601F801F901FA01FB01FC01FD3C
:1022D00001FE01FF010002010202020302040205E5
:1022E0000206020702080209020A0200000B020CA1
:1022F000020D020E020F021002110212021302144A
:102300000215021602170203000200190019001933
:102310000019001900190003000200190019001922
:102320000019001900190003000200190019001912
:102330000019001900190003000200190019001902
:1023400000190019001900484848484848484848BA
:1023500048484848484848484848484848484848FD
:1023600048484848484848484848484848484848ED
:1023700048484848484848F4F4F4F4F4F4F4F4F4D1
:10238000F4F4F4F4F4F4F4F4F4F4F4F4F4F4F4F40D
:10239000F4F4F4F4F4F4F4F4F4F4F4F4F4F4F4F4FD
:1023A000F4F4F4F4F4F4F4ADAD09090000AD09045B
:1023B0000E0607AD01060606070901070F0F0FAD50
:1023C0000106070F0FAD00030E0E0FADAD01020B9E
:1023D0000BADAD0900090909ADADADADAD0301AD62
:1023E000ADADAD0D0101ADADAD4E0100ADADAD4E2C
:1023F0000100ADADAD0A09ADADADAD0000ADADAD07
:10240000AD09ADADADADADADAD09090000AD090192
:102410000B0B0CAD010B0B0B0C09010C0C0C0CADD8
:10242000010B0C0C0CAD00010B0B0CADAD0101014F
:1024300001ADAD0900090909ADADADADAD0101AD0D
:10244000ADADAD0B0101ADADAD4B0100ADADAD4BD3
:102450000100ADADAD0109ADADADAD0000ADADADAF
:10246000AD09ADADADADADF4F4F4F4F4F4F4F4F4C1
:10247000F4120AF4F4125B5B5BF4F4F45B5B5B1242
:102480001212121212F4125B5B5B5BF4F4125B5BD0
:102490005BF4F4F412125BF4F4F4F4F4F4F4F4F4F2
:1024A000F4F4125BF4F4F4F4125BF4F4F4125B123F
:1024B00012121212125B5B5B5B5B5B5B5B5B5B5BD9
:1024C0005B5B5B5B5B5B5B125B5B5BF4F45B5B5B73
:1024D0005B5B5B00005B5B00005B5B125B5B5B124A
:1024E00012121212125B5B5B5B5B5B5B5B5B5B5BA9
:1024F0005B5B5B5B5B5B5BF4F4F4F4F4F4F4F4F4CB
:10250000F4F4F45B5B5BF4F4F45B12125BF4F4122E
:1025100012121212F45B5B5B5B12F45B5B5B12F4F6
:10252000F45B5B12F4F4F4F4125B5B5BF4F4F4120E
:102530005BF4F4F41200005BF4F4125B5B5BF412E6
:102540001212121212125B5B5B5B5B125B5B5B5BDA
:102550005BF4125B5B5BF4F45B5BF45BF4F4F45BE5
:10256000F40F0F5BF4F40F0F1F5BF4F4121F2F1224
:1025700012125B1F3F5B5B5B5B0F1F5B5B5B0F5B69
:102580005B5B5B5B5B5B5B125B5B5BF4F45B0F5BFE
:102590005BF45B1F1F0F00005B3F3F1F0F5B5B3F48
:1025A0002F1F1212122F1F0F5B5B5B5B0F5B5B5BBE
:1025B0005B5B5B5B5B5B5B5BF4F4F40FF4F40FF46D
:1025C000F40F0F5BF40F0F0F1FF4F4F40F1F2F1213
:1025D000120F0F1F3F5B5B0F1F2F3F5B0F0F1F2F54
:1025E0001F5B5B5B5B0F0F125B5B0FF4F41F1F0F36
:1025F0000F0F5B2F3F1F0F00003F3F2F1F0F5B3F51
:102600003F1F1F0F123F2F1F0F0F0F2F1F0F0F5BAB
:102610005B0F5B5B0F5B5BF4125B5B5BF4F4F412D0
:102620005B0F0FF40F0F1F0FF4F4121F3F1FF41274
:10263000123F3F0F12120F5B1F0F5B125B5B5B5B66
:102640005BF4125B5B5BF4F4120F5B5BF4F40F0F53
:102650000F0F0F0F0F1F1F0FF4F41F3F3F1FF41238
:102660001F1F3F1F0F0F0F1F1F0F0F120F0F0F0FF7
:102670005BF4120F5B5BF448484848889848484828
:102680008898A848484888984848488898A848485A
:102690008898A848484888984848488898A848484A
:1026A0004898A848484848988848484848489888DA
:1026B00048484848988848484848A898884848481A
:1026C00048A8988848484848988848484848A8985A
:1026D0008848484848A898ADAD09090000AD0931BF
:1026E00034343DAD013434343D09013D3D3D3DAD13
:1026F00001343D3D3DAD003134343DADAD013131AE
:1027000031ADAD0900090909ADADADADAD3101ADDA
:10271000ADADAD343101ADADAD343100ADADAD34A5
:102720003100ADADAD3109ADADADAD0000ADADAD7C
:10273000AD09ADADADADADADAD09090000AD091050
:10274000222828AD0122222228090128282828AD84
:102750000122282828AD0010222228ADAD0110103A
:1027600010ADAD0900090909ADADADADAD0101ADCB
:10277000ADADAD281001ADADAD101000ADADAD10DB
:102780001000ADADAD1009ADADADAD0000ADADAD5E
:10279000AD09ADADADADAD000000000000280028D2
:1027A00028282822282222222222222222222222F1
:1027B00021222222222100212121210000000000CB
:1027C0000000000000000000000000000028282891
:1027D0000000002222222800002222222228002299
:1027E0002222210000212121000000000000000021
:1027F00000000000000000000000000000000000D9
:1028000000000000000000000000000000000000C8
:1028100000000000000000000000000000000000B8
:1028200000000000000000484828224848482822AC
:1028300022224848482822484848484848484848AA
:102840004848484848484848484848484848484808
:10285000484848484848484848282248484848285E
:102860002248484828222222484828222222482852
:102870002222222222482822222248484848484828
:102880004848484848484848482822484848282254
:102890002222484828222222482822222222222894
:1028A00022222222222822222222222822222222FC
:1028B00022482822222248005B5B5B5B5B5BADAD5C
:1028C000ADADAD5BAD00ADAD005BADADAD00005BE2
:1028D000ADAD0000005BAD000000005BAD0000008E
:1028E000005BAD000000005B5B5B5B5B00ADADAD12
:1028F000ADAD5B00ADAD00AD5B0000ADADAD5B005F
:102900000000ADAD5B00000000AD5B00000000AD5D
:102910005B00000000AD5B5BAD000000005BAD0044
:102920000000005BAD000000005BADAD0000005B8F
:10293000ADADAD00005BAD00ADAD005BADADADAD1F
:10294000AD005B5B5B5B5B00000000AD5B0000000B
:1029500000AD5B00000000AD5B000000ADAD5B00B2
:1029600000ADADAD5B00ADAD00AD5BADADADADAD42
:102970005B5B5B5B5B5B005B5B5B5B5B5BADADAD0C
:10298000ADADAD0000000000000000000000000040
:102990000000000000000000000000000000000037
:1029A0000000000000000000000000000000000027
:1029B0000000000000000000000000000000000017
:1029C0000000000000000000000000ADADADADADA6
:1029D000AD5B5B5B5B5B5B5BAD000000005BAD0018
:1029E0000000005BAD000000005BAD000000005B7C
:1029F000AD000000005BAD000000005BAD0000001A
:102A0000005BAD0000000000000000AD5B000000B6
:102A100000AD5B00000000AD5B00000000AD5B009E
:102A2000000000AD5B00000000AD5B00000000ADE9
:102A30005B00000000AD5BF4F4F4F4F4F4F4F4F49F
:102A4000FFFFFFF4FFFFFFF6F6FFFFF6FFFFFFFFBC
:102A5000FFFFF6FFFFF4FFFFFFFFFFF4F4FFF4F4C6
:102A6000FFF4F4F4F4F4F4F4F4F4F4F4F4FFFFF405
:102A7000F4FFFFFFFFFFFFF6FFFFF6FFF6FFFFF695
:102A8000FFFFF6FFFFFFFFFFFFFFF6FFF4F4F4FF89
:102A9000FFF4F4F4F4F4F4F4F4F4F4F4F4FFF4FFD5
:102AA000F4F4F4FFFFFFFFF4F4F6FFF6FFFFF4FF8A
:102AB000FFFFFFFFF4FFFFF6FFF4F4FFF4F4F4F47C
:102AC000F4F4F4F4F4F4F4F4F4F4F4F4F4F4F4F4C6
:102AD000F4F4F4F4F4F4F4F4F4F4F4F4F4F4F4F4B6
:102AE000F4F4F4F4F4F4F4125A5A5AF4125B5B5B03
:102AF0005BF4125B5B5B5BF4F4F4F4F4F4F4F4F475
:102B0000F4F412F4F4F4F4125BF4F4F4F4125BF45D
:102B1000F4F4F4125B5A5A5A5A5B5A5B5A5B5B5B89
:102B20005B5B5B5B5B5B5BF4F4F4F4F4F412F4F476
:102B3000F4F4F45B5BF4F4F4F45B5BF4F4F4F45B52
:102B40005BF4F4F4F45A5A5A5A5A5A5B5B5B5A5B78
:102B50005B5B5B5A5B5B5BF4F4F4F4F4F4F4F4F465
:102B6000F4F4F4F4F4F4F4F4F4F4F4F4F4F4F4F425
:102B7000F4F4F4F4F45A5A5AF4F4F45B5A5B5BF448
:102B8000F45A5A5B5BF4F4F4F4F4F4F4F4F4F45B04
:102B90005BF4F4F4F4125BF4F4F4F4125BF4F4F484
:102BA000F4125BF4F4F45A5B5B12F45A5B5B5B5B0C
:102BB000125A5B5B5B5B12F4F4F4F4F4F4F4F45B30
:102BC000F40F0FF45BF40F0F1FF4F4F4F41F2FF461
:102BD000F45BF41F3F5A5A5A5A0F1F5B5B5B0F5B43
:102BE0005B5B5B5B5B5B5BF4F4F4F4F4F45B0FF452
:102BF000F45BF41F1F0FF4F4F43F3F1F0FF45B3F2F
:102C00002F1F5B5BF42F1F0F5B5B5A5B0F5B5B5BE4
:102C10005B5B5B5A5B5B5BF4F4F4F40FF4F45BF422
:102C2000F40F0F5BF40F0F0F1F5BF4F40F1F2FF463
:102C3000F40F0F1F3F5A5A0F1F2F3F5B0F0F1F2F0D
:102C40001F5B5B5B5B0F0FF4F4F40FF4F41F1F0FBB
:102C50000F0FF42F3F1F0FF4F43F3F2F1F0FF43FD0
:102C60003F1F1F0FF43F2F1F0F0F0F2F1F0F0F5B63
:102C70005B0F5B5A0F5B5BF4F4F4F4F4F4F4125B57
:102C80005B12F4F4F4125B0F0FF40F0F1F0FF4F448
:102C9000F41F3F1FF4F45A3F3F0FF45A0F5B1F0F0E
:102CA000125A5B5B5B5B12F4F40FF4F4F4F40F0F55
:102CB0000F0F0F0F0F1F1F0FF4F41F3F3F1FF4F4F0
:102CC0001F1F3F1F0F0F0F1F1F0F0F5B0F0F0F0F48
:102CD000125B5B0F5B5B12484848484848484848CD
:102CE0004848E2484898E298984848484848484840
:102CF0004848484848484848484848484848484854
:102D000048484848484848484848484848E2E2480F
:102D10004848484848484848484848484848484833
:102D20004848E2E2484848989898484848484848FF
:102D300048F4F4F4F4F4F44848E2E24848484848D7
:102D400048489848484848484848484848484848B3
:102D500048484848484848484848484848F4F4489B
:102D600048F4F4484848484848484848489848483B
:102D700048484848484848484848484848484848D3
:102D800048484848484848484848484848484848C3
:102D9000484848484848F448484848484848484807
:102DA0004848484848484848489898E29848484819
:102DB0004848484848484848484848484848484893
:102DC00048F4F448484848484848484848484898DB
:102DD00098984848484848484848484848484848D3
:102DE0004848484848484848484848484848F4F40B
:102DF000F4484848484848484848484848484848A7
:102E0000484848484848E2E248484848484848480E
:102E10009898984848484848484848F4F4F448483E
:102E200048484848484848484848E2E248484848EE
:102E30004898984848484848484848484848484872
:102E400048484848984848484848484848484848B2
:102E500048484848484848484848484848984848A2
:102E6000484848484848484848484848484848E248
:102E70009848484848484848484848484848484882
:102E800048484848484848484848484848484848C2
:102E9000484848484848E2E298484848484848482E
:102EA000484848484848484848484848F4F4F4F4F2
:102EB0004848484848484848484848484848484892
:102EC0004848489848484848484848484848484832
:102ED0004848484848484848484848484848484872
:102EE0004848484848F4F4484848484848484898BA
:102EF000E2984848484848484848E2E24848484834
:102F00004848484848484848484848484848484841
:102F100048F4484848484848484848484848484885
:102F200048484848484848484848484848484898D1
:102F300098484848484848484848484848484848C1
:102F40004848484848484848484848484848989861
:102F5000E2484848484848484848484848989848B7
:102F6000484848484848484848F4F4484848484889
:102F70004848484848484848484848484848E24837
:102F800048484848484848484848484848484848C1
:102F90004848484848F4F4F4F4F448484848484855
:102FA0004848484848484800000000002800000001
:102FB0000000280000000028280000000028002849
:102FC0000000282800002800280000002800280011
:102FD00000000028000000000000000000000000C9
:102FE00000000000000000000000000000000000E1
:102FF00000000000000000000000000000000000D1
:10300000000000090909090000000000000000009C
:1030100000000000000000000000000000000000B0
:10302000000000000000000000000909090909096A
:103030000909090909090900000000000000000051
:103040000000000000000000000000000000000080
:1030500000000909090909090909090909090909F2
:103060000909090909090900000000000000000021
:10307000000000000000000000000000000009093E
:1030800009090909090909090909090909090909B0
:1030900009090909090909000000000000000000F1
:1030A00000000000000000000009090909090909E1
:1030B0000909090909090909090909090909090980
:1030C00009090909090909000000000000000000C1
:1030D0000000000000000909090909090909090996
:1030E0000909090909090909090909090909090950
:1030F0000909090909090900000000000000000091
:10310000000000090909090909090909090909094A
:10311000090909090909090909090909090909091F
:103120000909090909090900000000000000000060
:103130000000090909090909090909090909090911
:1031400009090909090909090909090909090909EF
:103150000909090909090900000000000009090915
:1031600009090909090909090909090909090909CF
:1031700009090909090909090909090909090909BF
:1031800009090909090909000909090909090909B8
:10319000090909090909090909090909090909099F
:1031A000090909090909090909090909090909098F
:1031B000090909090909090909090909090909097F
:1031C000090909090909090909090909090909096F
:1031D000090909090909090909090909090909095F
:1031E0000909090909090909090909090009090958
:1031F000090909090909090909090909090909093F
:10320000090909090909090909090909090909092E
:10321000090909090909090000000000000000006F
:103220000000000900000000000909090909090956
:1032300009090909090909090909090909090909FE
:10324000090909090909090000000000000000003F
:10325000000000000000000000090000000000095C
:1032600009090909000909090909090909090909D7
:10327000090909090909090000000000000000000F
:10328000000000000000000000000000000000003E
:1032900000000000000909090900000909090909DD
:1032A00009090909090909000000000000000000DF
:1032B000000000000000000000000000000000000E
:1032C00000000000000000000000000909000000EC
:1032D00000090909090909000000000000000000B8
:1032E00000000000000000000000000000000000DE
:1032F00000000000000000000000000000000000CE
:1033000000090900000000000000000000000000AB
:1033100000000000000000000000000000000000AD
:10332000000000000000000000000000000000009D
:103330000900000000090900000000000000000072
:103340000000000000000000000000000000090074
:1033500000000909090009090909090909090909F8
:10336000090909090909090000000000000000001E
:1033700009090900090909090909090909090909C6
:1033800009090909090909090909090909090909AD
:1033900009090909090909000009090909090909AF
:1033A000090909090909090909090909090909098D
:1033B000090909090909090909090909090909097D
:1033C000090909090909090909090101090909097D
:1033D000010109090909010109090909010109098D
:1033E000090901010909090901010909090901017D
:1033F0000909090901010109090909090909090955
:10340000090909090909090909090909090909092C
:10341000090909090909090909090909090909091C
:10342000090101010101010101090901010101096C
:103430000901010101090901010101090901010154
:10344000010909010101010909090901010909012C
:103450000101010909010101010101010109090934
:103460000909090909090909090101010101010104
:1034700001010101010909090909090909090909E4
:10348000090101010101010101090901010101090C
:1034900009010101010909010101010909010101F4
:1034A00001090901010101090901010101090901DC
:1034B00001010109090101010909090909010109BC
:1034C000090909090909090909010909090909017C
:1034D0000109090909010109090909010109090984
:1034E0000901090909090909000000000009090981
:1034F0000000000909090909000909090909090960
:10350000090909090909090909090909090909092B
:10351000090909090909090000000000000000006C
:103520000000000000000000000900000000000989
:10353000090900000009090909090009090909091F
:10354000090909090909090000000000000000003C
:10355000000000000000000000000000000000006B
:103560000000000000000000000009000000000052
:10357000090000000000090000090909090000090C
:1035800009090900090909090900090909090909BD
:10359000090909090909090909090909090909099B
:1035A000090909090909090909090909090909098B
:1035B000090909090909090909090909090909097B
:1035C000090909090909090909090909090909096B
:1035D00009090909ADADAD0909090909090909096F
:1035E000090909090909090909090909090909094B
:1035F000090909090909090909090909090909093B
:1036000009ADADADADADAD09090909090909090952
:10361000090909090909090909090909090909091A
:10362000090909090909090909090909095B5B5B14
:103630005BADADADADADAD090909090909090909D0
:1036400009090909090909090909090909090909EA
:1036500009090909090909090909095B5B5B5B5B40
:103660005BADADADADADAD090909090909090909A0
:1036700009090909090909090909090909090909BA
:1036800009090909090909090909095B5B5B0909B4
:1036900009ADADADADADAD090909090909090909C2
:1036A000090909090909090909090909090909098A
:1036B000090909090909090909090909090909097A
:1036C00009ADADAD090909090900000000090909A2
:1036D00000000009090900000009090909000009A2
:1036E000090909090009090909090009090909095C
:1036F0000009090909090000000000000900000094
:10370000000009000000000009000000000009009E
:103710000000000009000000000009000000000097
:103720000900000000000909090909090909090936
:1037300009090909090909090909090909090909F9
:1037400009090909090909090909090909090909E9
:103750000909090900095B09090909090909090990
:1037600009090909090909090909090909090909C9
:10377000090909090909095B5B5B5B5B5B5B5B5BD7
:103780005B5B5B5B5B5B5B0909090909090909096B
:103790000909090909090909090909090909090999
:1037A00009090909095B5B5B5B5B5B5B5B5B5B5B03
:1037B0005B5B5B5B5B5B5B0909090909090909093B
:1037C00009090909090909090909090909095B0917
:1037D0005B5B5B5B5B5B5B5B5B5B5B5B5B5B5B5B39
:1037E0005B5B5B5B5B5B5B0909090909090909090B
:1037F000090909095B5B5B5B5B5B5B5B5B5B5B5B61
:103800005B5B5B5B5B5B5B5B5B5B5B5B5B5B5B5B08
:103810005B5B5B5B5B5B5B09090909090909095B88
:103820005B5B5B5B5B5B5B5B5B5B5B5B5B5B5B5BE8
:103830005B5B5B5B5B5B5B5B5B5B5B5B5B5B5B5BD8
:103840005B5B5B5B5B5B5B09090909095B5B5B5B62
:103850005B5B5B5B5B5B5B5B5B5B5B5B5B5B5B5BB8
:103860005B5B5BADAD5B5B5BADAD5B5B5BADAD5BBC
:10387000AD5B5BAD5BADAD5B5B5B5B5B5B5B5B5B50
:103880005B5BAD5B5B5BADADADADADADADADADAD02
:10389000ADADADADAD5B5B5B5B5B5BADADADADAD44
:1038A000AD09ADADADADAD5B5B5B5B5B5BADADADD8
:1038B000ADADADADADADADADADADADADADADADAD38
:1038C000ADADADADAD5B5B5B5B5B5BADADADADAD14
:1038D000ADADADADADADADADADADADADADADADAD18
:1038E000ADADADADADADADADADADADADADADADAD08
:1038F000ADADADADAD5B5B5B5B5B5BADADADADADE4
:10390000ADADADADADADADADADADADADADADADADE7
:10391000ADADADADADADADADADADADADADADADADD7
:10392000ADADADADAD5B5B5B5B5B5BADADADAD5B05
:103930005BADAD09ADAD5BADADADADADADADADADFF
:10394000ADADADADADADADADADADADADADADADADA7
:10395000ADADADADADADADAD5B5B5B5BAD5B5B5BD5
:10396000AD5BAD5B5BADADADADADADADADADADAD7D
:10397000ADADADADADADADADADADADADADADADAD77
:10398000ADADADADAD5B5B5B5B5B5BADADADADAD53
:10399000AD09ADADADADADADADADADAD5BADADAD4D
:1039A000ADADADADADADADADADADADADADADADAD47
:1039B000ADADADADAD5B5B5B5B5B5BADADADADAD23
:1039C000ADADADADADADAD5B5B5B5B5B5B5B5B5B09
:1039D0005B5B5BADAD5B5B5B5BADADADADAD5BADA7
:1039E000ADADADADAD5B5B5B5B5B5BADADADADADF3
:1039F000ADADADADAD09AD0909090909095B5B5B69
:103A00005B5B5B5B5B5B5B5B5B5B5B5B5B5B5BADB4
:103A10005B5B5B5B5BADAD5B5B5B5B5BADAD5B5BAE
:103A20005BAD5BADAC5B5B0909090909095B5B5BDD
:103A30005B5B5B5B5B5B5B5B5B5B5B5B5B5B5B5BD6
:103A40005B5B5B5B5B5B5B5B5B5B5B5B5B5B5B5BC6
:103A50005B5B5B5B5B5B5B0909090909095B5B5BA2
:103A60000909095B5B5B5B5B095B5B5B5B5B5B5BEE
:103A70005B5B5B5B5B5B5B5B5B5B5B5B5B5B5B5B96
:103A80005B5B5B5B5B5B5B09090909090909090968
:103A90000909090909090909095B5B5B0909095B4E
:103AA0005B5B5B5B5B5B5B5B5B5B5B5B5B5B5B5B66
:103AB0005B5B5B5B5B5B5B09090909090909090938
:103AC0000909090909090909090909090909095B14
:103AD0005B5B5B5B5B5B5B5B5B5B5B5B5B5B5B5B36
:103AE0005B5B5B5B5B5B5B09090909090909090908
:103AF0000909090909090909090909090909095BE4
:103B00005B090909095B5B5B5B09095B5B5B5B5BF1
:103B1000095B5B5B5B5B0009090909090909090984
:103B20000909090909090909090909090909090905
:103B300009090909090909090909090009090909FE
:103B40000900000009090909090909090009090909
:103B500009090009090909090009090909090009F0
:103B600009090909000909090909000909090909D7
:103B700000090909090900090909090909090909C7
:103B800009090909090909090909090909090909A5
:103B900009090909000909090000000909000000D4
:103BA00000090000000000090909090909090909BB
:103BB00009000009090000000000000000000000EA
:103BC00000000000000000000000000000000000F5
:103BD0000000000000000009000000005B00000081
:103BE00000005B00000000005B00000000005B00C4
:103BF000000000005B00000000005B00000000000F
:103C00005B0000000000005B5B5B5B5B5B5B5B5B26
:103C10005B5B5B5B5B5B5B5B5B5B5B5B5B5B5B5BF4
:103C20005B5B5B5B5B5B5B5B5B5B5B5B5B5B5B5BE4
:103C30005B5B5B5B5B5B5B5B5BAD5BAD095B5BAD30
:103C40005BADAD5B5BAD5BADAD5B5BAD5BADAD5B34
:103C50005BAD5BADAD5B5BAD5BADAD5B5BAD5BAD24
:103C6000AD5B5BAD5BADAD0909ADADADAD09ADAD66
:103C7000ADADADADADADADADADADADADADADADAD74
:103C8000ADADADADADADADADADADADADADADADAD64
:103C9000ADADADADADADADADADADADADADADADAD54
:103CA000ADADADADADADADADADADADADADADADAD44
:103CB000ADADADADADADADADADADADADADADADAD34
:103CC000ADADADADADADADADADADADADADADADAD24
:103CD000ADAD01ADADADADAD01ADADADADAD01AD18
:103CE000ADADADAD01ADADADADAD01ADADADADAD5C
:103CF00001ADADADADADADADADADADADAD0101ADF8
:103D0000ADADADADAD01ADAD01ADAD01AD01AD013F
:103D100001ADAD0101ADAD01AD01ADADAD01AD0187
:103D2000ADADADADADADADADADADADADAD01ADAD6F
:103D300001ADADAD01AD01ADADAD01AD0101AD0167
:103D400001AD01AD01AD01AD01ADADAD01AD01AD57
:103D5000ADADADADADADADADADADADADAD01AD01EB
:103D600001010101AD01ADAD0101AD01ADADAD018F
:103D7000AD01AD010101AD01ADAD0101AD0101012B
:103D800001ADADADADADADADADADADADADAD010167
:103D900001ADADAD01ADADADADAD01ADADADADAD57
:103DA0000101ADADADAD01ADADADADAD010101AD4B
:103DB000ADADADADADADADAD090909AD5BADAD0915
:103DC000ADAD5BADADADADAD5BADADADADAD5BAD19
:103DD000ADADADAD5BADADADADAD5BADADADADADB7
:103DE0005BADADADADAD5B5BAD5B5BAD095BAD5BE5
:103DF0005BADAD5BAD5B5BADAD5BAD5B5BADAD5B83
:103E0000AD5B5BADAD5BAD5B5BADAD5BAD5B5BAD72
:103E1000AD5BAD5B5BADADADADADADADADADAD0174
:103E20000101ADADAD01ADAD01ADAD01ADAD01ADCA
:103E3000AD01ADAD01ADAD01ADAD01ADAD01010166
:103E4000ADADADADADADADADADADADADADAD01AD4E
:103E500001ADADAD01AD01ADADAD01ADAD01ADADEE
:103E600001ADAD01ADAD01ADADAD01AD01ADADADDE
:103E700001ADADADADADADADADADADADADAD01ADCA
:103E8000010101AD01AD01ADAD01ADAD01ADAD01C2
:103E9000ADAD0101ADADADAD01ADADADADAD0101AE
:103EA00001ADADADADADADADADAD090909ADADADDA
:103EB000AD09ADADADADADADADADADADADADADADD6
:103EC000ADADADADADADADADADADADADADADADAD22
:103ED000ADADADADADADADAD5BADAC5B5BAD5BAD5B
:103EE000AC5B5BAD5BADAC5B5BAD5BADAC5B5BAD95
:103EF0005BADAC5B5BAD5BADAC5B5BAD5BADAC5B85
:103F00005BAD5BADAC5B5B5B5B5B5B5B005B5B5B67
:103F10005B5B005B5B5B5B5B005B5B5B5B5B005B02
:103F20005B5B5B5B005B5B5B5B5B005B5B5B5B00F2
:103F3000005B5B5B00000009090909090900000931
:103F4000090909000000000909000000000009003B
:103F50000000000000000000000000000000000061
:103F60000000000000000009090909090009090909
:103F700009090009090909090009090909090000D5
:103F800009090909000000090909000000000909E0
:103F90000000000009090000000000000900000006
:103FA00000000900000000000900000000000900F6
:103FB0000000000000000000000000000000000001
:103FC00000000000000000090000000000090000DF
:103FD00000000009000000000009090000000009BD
:103FE0000909000000090909090000000909090977
:103FF00000000000000909005B5B5B5B5B00005B8D
:104000005B5B5B000000005B5B00000000000000E9
:1040100000000000000000000000000000000000A0
:10402000000000000000005B5B5B5B5B5B5B5B5B5D
:104030005B5B5B5B5B5B5B5B5B5B5B5B5B5B5B002B
:10404000005B5B5B5B0000005B5B5B0000000000F3
:10405000000000000000005B5B5B5B5B5B5B5B5B2D
:104060005B5B5B5B5B5B5B5B5B5B5B5B5B5B5B5BA0
:104070005B5B5B5B5B5B5B5B5B5B5B5B5B5B5B5B90
:104080005B0000005B5B5B5B5BAD5BADAD5B5BAD49
:104090005BADAD5B5BAD5BADAD5B5BAD5BADAD5BE0
:1040A0005BAD5BADAD5B5BAD5BADAD5B5BAD5BADD0
:1040B000AD5B5BAD5BADADADADADADAD5BADADAD78
:1040C000ADAD5BADADADADAD5BADADADADAD5BAD16
:1040D000ADADADAD5BADADADADAD5BADADADADADB4
:1040E0005BADADADADAD5B5BAD5B5BADAD5BAD5B3E
:1040F0005BADAD5BAD5B5BADAD5BAD5B5BADAD5B80
:10410000AD5B5BADAD5BAD5B5BADAD5BAD5B5BAD6F
:10411000AD5BAD5B5BADAD5B5B5B5B5B5B5B5B5BA7
:104120005B5B5B5B5B5B5B5B5B5B5B5B5B5B5B5BDF
:104130005B5B5B5B5B5B5B5B5B5B5B5B5B5B5B5BCF
:104140005B5B5B000000005B5B5B5B5B5B5B5B5B2B
:104150005B5B5B5B5B5B5B5B5B5B5B5B5B5B5B5BAF
:104160005B5B5B5B5B5B5B5B5B00005B00000000C1
:10417000000000000000005B5B5B5B5B5B5B5B5B0C
:104180005B5B5B5B5B5B5B00005B5B000000005BA1
:10419000000000000000000000000000000000001F
:1041A000000000000000005B5B0000000000000059
:1041B00000000000000000000000000000000000FF
:1041C00000000000000000000000000000000000EF
:1041D00000000000000000000000000000000000DF
:1041E00000000000000000000000000000000000CF
:1041F000000000000000000000000900000909099B
:104200000900090909000000000009090000000078
:10421000090900000009090900000909090000094D
:104220000909090000090909000000000000000058
:10423000000000000000000909090000000000095A
:104240000909090000000009090000000000000041
:10425000000000000000000000000000000000005E
:104260000000000000000000000000000009000045
:1042700000000009090900000000000909090900FF
:10428000000000090900000000000000000000001C
:10429000000000000000000000000000000000001E
:1042A0000000000000000000000000000000000905
:1042B00009090900000000090909090000000000BF
:1042C00009000000000000000000000000000000E5
:1042D00000000000000000000000000000000000DE
:1042E00000000000000000000000000909090000B3
:1042F00000000000090909000000000000000000A3
:1043000000000000000000000000000000000000AD
:10431000000000000000000000000000000000009D
:104320000009000000000000005B5B5B5B00000018
:10433000000000000000000000000000000000007D
:10434000000000000000000000000000000000006D
:10435000000000000000005B5B5B5B5B5B0000003B
:10436000000000000000000000000000000000004D
:10437000000000000000000000000000000000003D
:10438000000000000000005B5BAD5BADAD005BAD0D
:104390005BADAD005BAD5BAD09005BAD5BADAD0092
:1043A0005BAD5B5BAD005BADAD5B5B005BADADADD5
:1043B000AD005BADAD5B5BADADADADADAD09ADAD74
:1043C000ADADAD0909ADADADAD09ADADADADADAD09
:1043D000ADADADADAD5B5B5B5B5B5BADADADADADF9
:1043E000AD5B5B5B5B5B5BADADADADADADADADADE9
:1043F000ADADADADADADADADADADADADADADADADED
:10440000ADADADADAD5B5B5B5B5B5BADADADADADC8
:10441000AD5B5B5B5B5B5BADADADADAD5BADAD09AE
:10442000ADAD5BAD090909AD5BADAD09ADAD5BAD42
:10443000ADADAD5B5B5B5B5B5B5BADADADADADADEA
:10444000AD5B5B5B5B5B5B5BAD5B5BADAD5BAD5B22
:104450005BADAD5BAD5B5BAD095BAD5B5BADADAD6E
:10446000ADAD5B5BADADADADAD5B5BADADADADADC4
:10447000AD5B5B5B5B5B5BADADADADADADADADAD58
:10448000AD09ADADADAD090909ADADADAD09ADAD90
:10449000ADADADADAD5B5B5B5B5B5BADADADADAD38
:1044A000AD5B5B5B5B5B5BAD5BADAC0000AD5BAD27
:1044B000AC0000AD5BADAC0000AD5BADAC00005B33
:1044C0005BADAC00005BADADAC0000ADADADAC0024
:1044D000005BADADAC00000000000000000000007B
:1044E00000000000000000000000000000000000CC
:1044F00000000000000000000000000000000000BC
:1045000000000000000009000000000000000000A2
:10451000000000000000000000000000000000009B
:104520000000000000000000000000000000090979
:104530000909090900000000000000000000000057
:10454000000000000000000000000000000000006B
:10455000000000090900090909090009000000001C
:10456000000000000000000000000000000000004B
:1045700000000000000000090909090909090909EA
:104580000900000000000000000000000000000022
:1045900000000000000000000000090909000909EE
:1045A00009090909090000000000000000000000DE
:1045B00000000000000000000000000000000000FB
:1045C00000000000000000090900000000000000D9
:1045D00000000000000000000000000000000000DB
:1045E00000000000000000000000000000000000CB
:1045F00000000000000000000000000000000000BB
:1046000000000000000000000000000000000000AA
:1046100000000000AD00000000AD5B00000000AD38
:104620005B00000000AD5B00000000000000000027
:10463000000000000000000000000000000000ADCD
:10464000ADADADADAD5B5B5B5B5B5B0000000000E7
:104650000000000000000000090909090000000036
:10466000000909000000000000000000000000AD8B
:10467000ADADADADAD5B5B5B5B5B5B0000000000B7
:10468000000000000000000000000000000909090F
:10469000090909000000000000000000000000AD52
:1046A000ADADADADAD5B5B5B5B5B5B000000000087
:1046B00000000000000000000000000000090909DF
:1046C000090909000000000000000000000000AD22
:1046D000ADADAD00005B5B5B5BAD000000005BADB2
:1046E000000000005BAD00005BAD5B5BAD095BAD46
:1046F0005BADAD005BAD5BAD09005BAD5BADAD002F
:104700005BAD5BADAD005BAD5BADAD005BAD5BAD1F
:10471000AD005BAD5BADADADADADADADAD09ADADBE
:10472000ADADAD0909ADADADAD09ADADADADADADA5
:10473000ADADADADADADADADADADADADADADADADA9
:10474000ADADADADADADADADADADADADADADADAD99
:10475000AD09ADADADAD090909ADADADAD09ADADBD
:10476000ADADADADADADADADADADADADADADADAD79
:10477000ADADADADADADAD5B5BADAC0909AD5BADA8
:10478000AC0000AD5BADAC0000AD5BADAC0000AD0E
:104790005BADAC0000AD5BADAC0000AD5BADAC00A3
:1047A00000AD5BADAC000009090909090900000072
:1047B00000000000000000000000ADADADADADADEB
:1047C0005B5B5B5B5BAD5B00000000AD5B00000012
:1047D00000AD5B000000000909090909090000009B
:1047E000000000000000000000ADADADADADAD5B60
:1047F0005B5B5B5B5B0000000000000000000000F2
:1048000000000000000000000000000000000000A8
:10481000000000000000000000ADADADADADAD5B2F
:104820005B5B5B5B5B0000000000000000000000C1
:104830000000000000000000000000000000000078
:10484000000000000000000000ADADADADADAD5BFF
:104850005B5B5B5B5B00000000005B000000000036
:104860005B00000000005B00000000000000000092
:10487000000000000000000000000000000000AD8B
:104880000000000000AD0000000000AD00000000CE
:1048900000AD00000000000000005BAD0000000063
:1048A0005BAD000000005BAD000000005BAD0000F0
:1048B00000005BAD000000005BAD000000005BADE0
:1048C000000000005BAD00005BAD5BADAD005BAD1B
:1048D0005BADAD005BAD5BADAD005BAD5BADAD00A9
:1048E0005BAD5BADAD005BAD5BADAD005BAD5BAD3E
:1048F00009005BAD5BADADADADADADADADADADADDD
:10490000ADADADADADADADADADADADADADADADADD7
:10491000ADADADADAD09ADADADADAD0909ADADADB3
:10492000AD09ADADADADADADADADADADADADADAD5B
:10493000AD0101ADADADAD01ADADADADAD01ADAD57
:10494000ADADAD01ADADADADAD01ADADADADAD019B
:1049500001ADADADADADADADADADADADAD01ADADDF
:10496000ADAD01AD01ADAD01ADAD01AD01ADADADD3
:1049700001AD010101AD01AD01ADAD01ADAD01ADC7
:10498000ADADADADADADADADADADADADADADAD0103
:10499000ADAD0101AD01ADAD0101AD0101AD010153
:1049A000AD01AD010101AD01ADAD0101AD01ADAD97
:1049B00001ADADADADADADADADADADADADAD01012B
:1049C0000101ADAD01ADAD01ADAD01ADADADADAD73
:1049D00001AD0101ADAD01ADAD01ADAD0101010113
:1049E000ADADADADADADADADADADADADAD010101FB
:1049F000AD010101ADADAD01AD01ADADAD01AD019B
:104A000001ADAD010101ADADAD01AD010101AD01E2
:104A1000ADADADADADADADADADADADADAD01ADAD72
:104A2000ADADADAD01ADADADADAD01ADADADAD01BA
:104A3000ADADADADADAD01ADADADADAD01ADADADFE
:104A4000ADADADADADADADADADADADADADADADAD96
:104A5000ADADADADADADADADADADADADADADADAD86
:104A6000ADADADADADADADADAD09ADADADAD090962
:104A700009ADADADAD09ADAD5BADAC0000AD5BADAD
:104A8000AC0000AD5BADAC0000AD5BADAC0000AD0B
:104A90005BADAC0000AD5BADAC0000AD5BADAC00A0
:104AA00000AD5BADAC0000AD5B00000000AD5B0095
:104AB000000000AD5B00000000AD5B00000000AD39
:104AC0005B00000000AD5B00000000AD5B0000007B
:104AD00000AD5B0000000000000000005B00000073
:104AE00000005B00000000005B00000000005B00B5
:104AF000000000005B00000000005B000000000000
:104B00005B00000000005BAD0000000000AD000095
:104B1000000000AD0000000000AD0000000000AD8E
:104B20000000000000AD0000000000AD000000002B
:104B300000AD0000000000005BAD5B5BAD005BAD55
:104B4000AD5B5B005BADADADAD005BADADADAD00E4
:104B50005BADADADAD005BADADADAD005BADADADD5
:104B6000A4005BADADADA4ADADADADADAD5B5B5B7C
:104B70005B5B5BADADADADADADADADACACACACAD5F
:104B80005B5B5B5B5B5BADADADADAD5BADADADAD93
:104B9000AD5BADADADADADADADADADADAD5B5B5B8D
:104BA0005B5B5BADADADADADADACACACACACAC5B83
:104BB0005B5B5B5B5BADADADADADADADADADADADBF
:104BC000ADADADADADADADADADADADADAD5B5B5B0B
:104BD0005B5B5BADADADADADADACACACADADAD5B50
:104BE0005B5B5B5BADADADADADAD5BADADADADAD8F
:104BF0005BADADADADAD5B5B5BADAC00005BADADDA
:104C0000AC0000ADADADAC0000ADADADAC0000ADE5
:104C1000ADADAC0000ACADADAC0000ACADADAC002A
:104C200000ACADADAC0000005BADADADA4005BADC4
:104C3000ADADA4005BADADADA4005BADADADA4006A
:104C40005BADADADA4005BADADADA4005BADADADF6
:104C5000A4005BADADADA45BADADADADAD5BADAD39
:104C6000AD07075BADADADADAD5BADADAD07075B02
:104C7000ADADAD07075BADADADADAD5BADADADAD54
:104C8000AD5BADADADAD5BADADADADADAD0707AD44
:104C9000070707AD07AD07ADAD07ADAD07ADAD0774
:104CA00007AD070707ADADADADADAD646464646439
:104CB000645B5B5B5B5B5BADADADADADAD0707ADA5
:104CC000ADADADAD07ADADADADAD07ADADADAD0706
:104CD00007ADADADADADADADADADAD646464646417
:104CE000645B5B5B5B5B5BADADADADADADADADAD29
:104CF000ADADAD0707AD07ADADAD0707ADADAD07C8
:104D000007AD07ADADADADADADADAD64646464648C
:104D1000645B5B5B5B5B5BADADADADADADADADADF8
:104D2000ADAD00ADADADADAD00ADADADADAD00ADBA
:104D3000ADADADAD00ADADADADADAD6464646464BD
:104D4000645B5B5B5B5B5BADADADADADAD000000CF
:104D5000000000AD00AD00AD00ADADADADADADAD91
:104D6000ADADADADADADADADADADAD6464646464E0
:104D7000645B5B5B5B5B5BADADADADADAD0000009F
:104D8000000000AD00AD00AD00AD00ADADADADAD0E
:104D900000ADADADADADADADADADAD64646464645D
:104DA000645B5B5B5B5B5BADADADADADAD0000006F
:104DB000000000AD00AD00AD00ADADAD00ADADADDE
:104DC000ADAD00ADADADADADADADAD64646464642D
:104DD000645B5B5B5B5B5BADADADADADAD0000003F
:104DE000000000AD07AD00AD00AD07ADADAD00AD4D
:104DF00007ADADAD00AD07ADADADAD646464646449
:104E0000645B5B5B5B5B5BADADADADADAD0000000E
:104E100000ADADAD00AD00ADADADADAD00ADADAD76
:104E2000ADAD00ADADADADADADADAD6464646464CC
:104E3000645B5B5B5B5B5BADADADADADADADADADD7
:104E4000ADADADADADADADADADADADADADADADAD92
:104E5000ADADADADADADADADADADAD6464646464EF
:104E6000645B5B5B5B5B5BADADADADAD5BADADADF9
:104E7000ADAD5BADADADADAD5BADADADADAD5BAD58
:104E8000ADADADAD5BADADADADAD5BADADADADADF6
:104E90005B5BADADADAD5BACADADAC0000ACADAD95
:104EA000AC0000ACADADAC0000ACADADAC0000AC46
:104EB000ADADAC0000ACADADAC0000ACADADAC0088
:104EC00000ACADADAC00005BADADADA4A35BADADD2
:104ED000ADA4A35BADADADA4A35BADADADA4A35B31
:104EE000ADADADA4A35BADADADA4A35BADADADA4C5
:104EF000A35BADADADA4A35B64ADADAD5B5B64ADD9
:104F0000ADAD5B5B64ADADAD5B5B64ADADAD5B5B4F
:104F100064ADADAD5B5B64ADADAD5B5B64ADADADE4
:104F20005B5B64ADADAD5B5BADADADA4A35BADADA7
:104F3000ADA4A35BADADADA4A35BADADADA4A35BD0
:104F4000ADADADA4A35BADADADA4A35BADADADA464
:104F5000A35B000000A4A300000000AD5B00000004
:104F600000AD5B00000000AD5B00000000AD5B0029
:104F7000000000AD5B00000000AD5B00000000AD74
:104F80005B0000000000AD00000000000000000019
:104F90000000000000000000000000000000000011
:104FA00000000000000000000000005B5B5B5B5B3A
:104FB0005BADADADADADAD0000005BAD0000000080
:104FC0005BAD000000005BAD000000005BAD0000C9
:104FD00000005BAD000000005BAD005B5B5B5BADA8
:104FE00000ADADADAD00005B00ADADA4A35B0000B6
:104FF000ADA4A35B00ADADA4A35B0000ADA4A35B17
:1050000000ADADA4A35B0000ADA4A35B00ADADA457
:10501000A35B000000A4A3AD5B00000000AD5B003B
:10502000000000AD5B00000000AD5B00000000ADC3
:105030005B00000000AD5B00000000AD5B5B5B5BF4
:105040005B00ADADADADAD00000000005B00000049
:1050500000005B00000000005B00000000005B003F
:10506000000000005B00000000005B5B5B5B5B5BC3
:105070005BADADADADADADAD0000000000AD00006D
:10508000000000AD0000000000AD0000000000AD19
:105090000000000000AD0000000000AD00000000B6
:1050A0000000000000000000000000000000000000
:1050B00000000000000000000000000000000000F0
:1050C00000000000000000000000000000000000E0
:1050D000005B5B5B5B5B5B005BADADADA4005BADA0
:1050E000ADADA4005BADADADA4005BADADADA400B6
:1050F0005BADADADA4005B5B5B5B5B005BADADAD81
:10510000A45BADADADADA45B00ADADA4A35B0000F1
:10511000ADA4A35B00ADADA4A35B0000ADA4A35BF5
:1051200000ADADA4A35B0000ADA4A35B00ADADA436
:10513000A35B000707A4A3ACADADAC0000ACADAD64
:10514000AC0000ACADADAC0000ACADADAC00005BF4
:105150005B5BAC0000ACADADAC0000ACADADACACDD
:10516000ACACADADADADAD00000000000000000086
:10517000000000000000000000000000000000002F
:105180000000000000000000000000ACACACACACC3
:10519000ACADADADADADAD00000000000000000055
:1051A00000000000000000000000000000000000FF
:1051B00000000000000000000000000000000000EF
:1051C00000ACACACACACAC000000000000000000D7
:1051D00000000000000000000000000000000000CF
:1051E000000000005B00000000005B000000000009
:1051F0005B00000000005B000000000000000000F9
:105200005B5BAD005B5BADADAD5B5BADADADADAD67
:10521000ADADADADADADADAD09ADADADAD0909094E
:10522000ADADADAD09ADAD5B5B5B5B5B5BADADAD3E
:10523000ADADADADADADADADADADADADADADADAD9E
:10524000ADADADADADADADADADADADADADADADAD8E
:10525000ADADADADADADADADADADADADA4ADADAD87
:10526000ADADA4ADADADADADA4ADADADADADA4AD89
:10527000ADADADADA4ADADADADADA4ADADADADAD70
:10528000A4ADADADADADA4ACADADADADADACADAD62
:10529000ADADADACADADADADADACADADADADADAC41
:1052A000ADADADADADACADADADADADACADADADAD30
:1052B000ADACADADADADADACACAC000000ADADAD29
:1052C000ACAC00ADADADADADACADADAD09ADADAD62
:1052D000AD090909ADADADAD09ADADADADADADAD8E
:1052E000ADADADADADADAD00000000000000000003
:1052F000000000000000000000AC00000000005BA7
:1053000000000000005B00000000005B00000000E7
:10531000005B00000000005B00000000005B00007C
:105320000000005B00000000005B00000000005B6C
:1053300000000000005B00000000005B00000000B7
:10534000005B000000000000000000000000000002
:10535000000000000000000000005B5B5B5B5B0185
:1053600001010101015B5B5B5B5B5B0909090909E9
:10537000095B5B5B5B5B5B00000000000000000002
:105380000000000000000000005B5B5B5B5B5B01FA
:1053900001010101015B5B5B5B5B5B0909090909B9
:1053A000095B5B5B5B5B5B00000000005B00000077
:1053B00000005B00000000005B5B5B5B5B5B5B0114
:1053C000010101015B5B5B5B5B5B5B09090909092F
:1053D0005B5B5B5B5B5B5B5B00000000005B00009A
:1053E0000000005B00000000005B5B5B5B5B5B5BE5
:1053F00001010101015B5B5B5B5B5B5B0909090907
:10540000095B5B5B5B5B5B00000000000000000071
:105410000000000000000000005B5B5B5B5B0001C4
:1054200001010101015B5B5B5B5B5B090909090928
:10543000095B5B5B5B5B5B0808080808085B5B5B00
:105440005B5B5B5B5B5B5B5B5B5B5B5B5B5B5B08FF
:1054500008080808085B5B5B5B5B5B0909090909D5
:10546000095B5B5B5B5B5B08080808085B5B5B5B7D
:105470005B5B5B5B5B5B5B5B5B5B5B5B5B5B5B08CF
:10548000080808085B5B5B5B5B5B5B090909090952
:105490005B5B5B5B5B5B5B5B08080808085B5B5BFB
:1054A0005B5B5B5B5B5B5B5B5B5B5B5B5B5B5B5B4C
:1054B00008080808085B5B5B5B5B5B5B0909090923
:1054C000095B5B5B5B5B5B010101010101005B5BF5
:1054D0005B5B5B00000000000000000000000000BB
:1054E00000000000000000000000000000000000BC
:1054F000000000000000000101010101015B5B5B95
:105500005B5B5B000000000000000000000000008A
:10551000000000000000000000000000000000008B
:105520000000000000000001010101015B5B5B5B0A
:105530005B5B5B00000000005B00000000005B00A4
:10554000000000005B00000000005B0000000000A5
:105550005B000000000000ADADADADADADADADADDB
:10556000ADADADADADADADADADADADADADADADAD6B
:10557000ADADADADADADADAD09ADADADAD090909EB
:10558000ADADADAD09ADADADAD000000ADAD000050
:10559000A400000000A4A4A40000A4A4A4A4A40047
:1055A00000A4A4A400AD0000A40000ADAD00000064
:1055B000ADADADADADADADADADADADADA4ADADAD24
:1055C000ADADA400ADADADADA400ADADADADA4002D
:1055D000ADADADADA4ADADADADADA4ADADADADAD0D
:1055E000A4ADADADADADAD5BADADADADA35BADADA2
:1055F000ADADAD5BADADADADAD5BADADADADAD5BD1
:10560000ADADADADAD5BADADADADAD5BADADADAD6E
:10561000AD5BADADADADADA3A3A3A3A3A3A4A4A463
:10562000A4A4A4ADADADADADADADADADADADADADC5
:10563000ADADADADADADADADADADADADADADADAD9A
:10564000ADADADADADADADA3ADADADAD5BADADADE6
:10565000ADAD5BADADADADAD5BADADADADAD5BAD70
:10566000ADADADAD5BADADADADAD5BADADADADAD0E
:105670005BADADADADAD5BACADADADAD00ACADADAD
:10568000AD0000ACADAD0000A4ACADAD00A4A4ACC9
:10569000ADAD0000A4ACADADAD0000ACADADADADF9
:1056A00000ACADADADADAD0000ADADADADA4000095
:1056B000ADADADA4A40000ADADA4A4A400ADADA457
:1056C000A40000ADADA40000ADADAD0000ADADAD2A
:1056D000ADADADADADADADADADADADADADADADADFA
:1056E000ADADADADADADADADADADADADADADADADEA
:1056F000ADADADADADADAD09ADADADAD090909AD6A
:10570000ADADAD09ADADAD5B01010101015B5B5B11
:105710005B5B5B5B00000000005B00000000005B67
:1057200000000000005B00000000005B00000000C3
:10573000000000000000000101010101015B5B5B52
:105740005B5B0000000000000000000000000000A3
:105750000000000000000000000000000000000049
:105760000000000000000000ADADADADAD0000AD2B
:10577000ADADAD0000000000000000000000000022
:105780000000000000000000000000000000000019
:1057900000000000000000ADADADADADADADADADF4
:1057A000ADADAD00000000000000000000000000F2
:1057B00000000000000000000000000000000000E9
:1057C00000000000000000AD5B5B5B5B5BADADAD5E
:1057D000ADADAD00000000000000000000000000C2
:1057E00000000000000000000000000000000000B9
:1057F000000000000000005B5B5B5B5BADADADAD2E
:10580000ADADAD0000000000000000000000000091
:105810000000000000000000000000000000000088
:1058200000000000000000ADADADADAD00ADADAD10
:10583000AD000000000000000000000000000000BB
:105840000000000000000000000000000000000058
:105850000000000000000000000000000000000048
:10586000000000000000000000000000000000AD8B
:10587000AD000000005B5BAD000000005BAD000010
:1058800000005BAD000000005BAD000000005BAD00
:10589000000000005BAD000000005BAD00000000F8
:1058A0005BAD000000005BAD000000005BAD0000E0
:1058B00000005BAD00000000000000AD5B000000D8
:1058C00000AD5B00000000AD5B0000000000AD001B
:1058D00000000000000000000000000000000000C8
:1058E00000000000000000000000000000000000B8
:1058F0000000005B5B5B5B5B5BADADADADADAD0078
:105900000000000000000000000000000000000097
:1059100000000000000000005BAD000000005BAD77
:105920000000005B5BAD000000ADAD0000000000BA
:105930000000000000000000000000000000000067
:105940000000000000000000000000000000000057
:105950000000000000000000000000000000000047
:1059600000000000000000000048480000000000A7
:105970000000000000000000000000000000000027
:105980000000000000000000000000000000000017
:105990000000000000484848484848000000000057
:1059A0000048484848484800000000000000000047
:1059B00000000000000000000000000000000000E7
:1059C0000000484848484848000000004848484807
:1059D0004848000000000000000000000000000037
:1059E0000000000000000000000000000000484827
:1059F00048484848480000000000004848484848D7
:105A0000480000000000000000000000000000004E
:105A1000000000000000000000484848484848488E
:105A200048484848480000000000004848484848A6
:105A300048004848484848000000000000000000B6
:105A4000000000000000000000480000000048487E
:105A50004848484848000048484848484848484856
:105A6000484848484848480000000000000000003E
:105A7000000000000000000000484848484848482E
:105A80004848484848484848484848484848484896
:105A9000484848484848480000000000000000000E
:105AA00000000000000000000048484848484848FE
:105AB00048484848484848484848480000585858C6
:105AC000584848585848580000000000000000009E
:105AD00000000000000000000000000048484848A6
:105AE0004848484848484848484848584858484816
:105AF000485858585858480000000000000000005E
:105B0000000000000000000000484848484848489D
:105B10004848484848484848484848484848484805
:105B200048004848484848000000000000000000C5
:105B300000000000000000000048484848480048B5
:105B4000000000000048484848484848484848483D
:105B5000484848484848480000000000000000004D
:105B60000000000000000000000000000000000035
:105B700000484848484848484848484848484848ED
:105B8000484848484848480000000000000000001D
:105B900000000000000000000000000000000048BD
:105BA000484800000048484848484848484848484D
:105BB00048484848484848000000000000000000ED
:105BC00000000000000000000000000000000000D5
:105BD0004848484848480000004848484848480065
:105BE0000048484848484800000000000000000005
:105BF000000000000000000000000000000000485D
:105C000048480000004848484848484848484848EC
:105C1000480000484848480000000000000000001C
:105C20000000000000000000000000000000000074
:105C30004848484800480000000000484848484894
:105C4000484848484848480000000000000000005C
:105C50000000000000000000000000000000000044
:105C600000000048480000484800004800000000CC
:105C70000048484848000000000000000000000004
:105C80000000000000000000000048484848484864
:105C9000000000000000004848484848480000480C
:105CA00048000000484848000000000000000000D4
:105CB00000000000000000000048484800004800C4
:105CC0000000484800484848000000484848484804
:105CD00048484848484848000000000000000000CC
:105CE0000000000000000000004848480000480094
:105CF000000000000000000000004848484848003C
:105D000000484848484848000000000000000000E3
:105D1000000000000000000000484848484800001B
:105D20000000000048480000000000000000484853
:105D30000048000048484800000000000000000043
:105D4000000000000000000000000000004848487B
:105D50004848484848000000484848004848000073
:105D60000048000048484800000000000000000013
:105D70000000000000000000004848480000004803
:105D800048484848484848484848480000000000FB
:105D90004848484848480000000000000000000053
:105DA00000000000000000000000000000000000F3
:105DB000004848484848480000484848484848483B
:105DC000480000000000000000000000000000008B
:105DD0000000000000000000000048484848484813
:105DE000000000000048484848484848484848489B
:105DF0004800480000000000000000000000000013
:105E000000000000000000000048484848484800E2
:105E1000000000000048484848484848484848486A
:105E2000480000000000000000000000000000002A
:105E30000000000000000000004848480000480042
:105E400000000000004848484848484848480000CA
:105E5000000000004848480000000000000000006A
:105E60000000000000000000004848484800000012
:105E70000000000000484800000000000000000092
:105E80000048484848484800000000000000000062
:105E900000000000000000000000004848484800E2
:105EA0000000000000484848484848000000000042
:105EB00000484848000048000000000000000000C2
:105EC0000000000000000000004848484848480022
:105ED00000000000004800000048480000000000EA
:105EE000004800000000000000000000000000006A
:105EF0000000000000000000004848484800000082
:105F000000000000004848484848480000000000E1
:105F10000000000000000000004848484800004819
:105F20004848480000000048480000000000000009
:105F30000048484848000000000000000000000041
:105F40000000484848484800000000000048484811
:105F500048484848484848484800000000000000B9
:105F60000000000000000048484848000048484839
:105F700048484848484848004848484848484848E9
:105F800048484848484848484800000000004848F9
:105F90004848484848484848484848484848484881
:105FA0004848484848484848484848484848484871
:105FB0004848484848484848484848484848484861
:105FC0004848484848484848484848484848484851
:105FD0004848484848585848484848484848484821
:105FE0004848484848484848484848484848484831
:105FF0004848484848484848484848484848484821
:1060000048585858585858484848484848484848B0
:106010004848484848484848484848484848484800
:106020004848484848484848484848484848480038
:106030004858585848585848484848484848484890
:1060400048484848484848484848484848484848D0
:1060500048484848484848484848484848484848C0
:1060600048585848004848485858585858005858B0
:1060700058585848485858585848485858585848F0
:1060800048585858584848585858584848585858E0
:1060900058484858585858585858585858585858A0
:1060A00058585800485858585800484858585800A8
:1060B0004800585858484848585858004848585870
:1060C0005800484858585848484848484858004890
:1060D0000048585800485858585848585858585820
:1060E0005858585848584848000048584848585840
:1060F0005858586060606048484848484858584870
:10610000484848585858584800585858585848000F
:10611000585858585848585858585858585858580F
:106120005858606060584848484848484848484877
:1061300058584858585858585858585858585858EF
:1061400058584848485858584800005858585858BF
:106150005858586058585848484848484848484847
:1061600048484848580048484858584800484858FF
:10617000584800484848484800484848484848481F
:1061800048585858484848484800484848484848A7
:10619000484848484848484848484848484848487F
:1061A000484848484848484848484848484848486F
:1061B0004848484848484800484848484848000037
:1061C0004848484848480048484848484848484897
:1061D000484848484848484848484848484848483F
:1061E0004848484848484848484800000048484807
:1061F000484848484848484848484848484848481F
:10620000484848484848484848484848484848480E
:10621000484848484848484848484848480000488E
:106220004848484848000048480000000000000076
:1062300000000000004800000000004800000000CE
:10624000004800000000004848484848484848487E
:10625000484848484848484848000000000048006E
:10626000000000000000000000000000000000002E
:106270000000000000000048484848484848484896
:1062800048484848484848484848484848484800D6
:1062900000000000000000000000000000000000FE
:1062A0000000000000000048000000004848484886
:1062B00048484848484848484848484848484800A6
:1062C00000000000000000000000000000000000CE
:1062D0000000000000000048484848484848484836
:1062E0004848484848484848484848484848480076
:1062F00048484848480000484848000000004848CE
:10630000000000004848484848484848484848482D
:1063100048484848000000000048484848484800AD
:106320000000000048000000000000000000000025
:10633000000000000000484848484848484848488D
:10634000480000000000004848484848484848487D
:10635000484848484800000000000000000000488D
:106360004800004848484848484848484800000015
:106370000000004848484848484848484848484875
:10638000484848484800000000000048484848483D
:106390004848484848484848484848484800000055
:1063A0000000004848484848484848484848484845
:1063B00048484848480048484848484848484848A5
:1063C00048484848484848484848480000000000B5
:1063D00000484848000000004848000048000048C5
:1063E0004848000000484800000000484848484825
:1063F0004848484800000000000000000048000035
:1064000000000048480000000000000000000048B4
:106410004848480000000000000000484848480084
:106420000000000000004800000000000000000024
:10643000000000000000000000000000000000005C
:106440000000000000000000000000004800000004
:1064500000480000000000000000000000000000F4
:1064600000004800000000000000000000000000E4
:1064700000000000000000000000000000000048D4
:1064800048000000000000000048484848000000A4
:1064900048484800000000004800000000000000DC
:1064A0000000000000000000004848484848000084
:1064B000000000000048004848484848484848480C
:1064C00048484848484848484800000000484800B4
:1064D000004848484848480000484800000000007C
:1064E0004848484848484848484800585848484854
:1064F000005858484848005858484848484858485C
:1065000048484848584848484848584848484848EB
:10651000584848484848585858585858585858584B
:1065200058585858585858585858585858585858EB
:1065300058585858585858585858585858585848EB
:1065400048585858585858585858485858585858EB
:1065500058585858585858585858585858585858BB
:1065600048485858584848480058580048484858DB
:106570005848484848585858585858004858584853
:1065800048584858585858585858585858585858AB
:10659000585858586058585858606058585858605B
:1065A00060585858606060484858585858004858D3
:1065B000585860005860606060485860606060488B
:1065C00058585858584848484848000048480059C2
:1065D00060004800616060484858606060606060CA
:1065E00060606060606060606060606060605858BB
:1065F000585858480058586060606060606060603B
:1066000060606060606060606060605808606060EA
:106610006058005960606060600061606060604860
:106620000059585848605858004848606060606198
:106630000060606060606148606060600059606038
:1066400060606060606060606060606060605900B1
:1066500048584848484848484848484848484848AA
:106660004800484848006000004848585860606149
:1066700000485960606060586060606060606008F9
:1066800059606060604800000000584860606060C9
:1066900060606060606060585858004848606058AA
:1066A000484848606060004848606048484848582A
:1066B0000048484848485858480048606060606052
:1066C00060606060606060484848484848484848A2
:1066D0004848484848484848484848484848004882
:1066E0004848484848484848484848004848585852
:1066F00048605848605858484848484848484848BA
:106700004848484848480048484848485848585821
:106710004848585858585858585858585858585819
:1067200048585858585848484848484848480048E1
:106730004848484800484848484800484848485859
:106740000048484848484800484848484848484859
:1067500048484848484848484848484848484848B9
:1067600048484848484848484848484848484848A9
:106770004848484848484848484848484848484899
:106780004848484848484048000000000048000089
:106790000000004800000000004800000000004821
:1067A0000000000000480000000000490000000058
:1067B00000000000000000000000000000000000D9
:1067C00000000000000000000000000000000000C9
:1067D0000000000000000000000000400000000079
:1067E00000000000004000000000004848000000D9
:1067F0000000000000000000480000000000480009
:106800000000000048000000000000000000000040
:1068100000000000000000484848484848000000C8
:106820000000000048484848480048484848484850
:106830000048484848000000000000484800484818
:106840004800480048480048000048484800000008
:106850000000004800004848004800004848004840
:106860000000484800000000000000000000004850
:1068700000000000000000484848480000000000F8
:106880000000004848484848484848484848484860
:1068900048484848000000000000004848484800B8
:1068A00048484848480048000000000048000000F0
:1068B0000000000048484800480048480048484850
:1068C00048480048480000004848484848004848B0
:1068D00048480048484848484800484848484848C8
:1068E0004848004800484848484848480000004890
:1068F0000000484848484848000000484848484880
:1069000048484848484848484848484800004800DF
:106910000000004848000000000048484848484837
:10692000480000000048000000480000000000008F
:10693000000000000000004848484848480000485F
:1069400048484800484848484800000000004800BF
:1069500048484848480000004848484800484848D7
:106960004800000000000048484848484848484857
:106970004848484848484848484848484848484897
:106980004848484848484848484848484848484887
:1069900048004848484848484848484858484848AF
:1069A0004848584848484848584848484848584837
:1069B0004848484858484848484858484848484837
:1069C0005848484848485858585858585858585897
:1069D0005858585858585858585858585858585837
:1069E0005858585858585858585858585858585827
:1069F0005858585858585848484848585848485877
:106A00005858585858585858585858585858585806
:106A10005858585858585858585858484858585816
:106A2000580048484858585858606060005860609E
:106A300060600058605858484858585800484858AE
:106A4000580048484858606060480058606060607E
:106A50005858586058606048005960606048005954
:106A600060606048596060606000606060606048BD
:106A70006060606060486060606060596060606035
:106A80006060606060606060606060606060606006
:106A9000606060606060605860606060004848608E
:106AA0006060004800606059004800606060004815
:106AB0004860605800484860606060606060606086
:106AC00060606060606060606060606060606060C6
:106AD00060606060606060606060606060606060B6
:106AE00060606060606060610048006060605800E5
:106AF0006160606060005860606060486060606015
:106B0000605960606060606060606060606060608C
:106B10006060606060606060606060606060606075
:106B200060606060606060606060606060600060C5
:106B300060606060486060606048486060606058A5
:106B4000486060606058486060606060606060607D
:106B500060606060606060606000596060606048B4
:106B6000006060606048486060606048006060602D
:106B7000604848606060606060606060586060604D
:106B8000606058606060605858606060580058608D
:106B9000605858485860606060485860606060485D
:106BA00058606060600058584858585848585858BD
:106BB0005858585858585858585858585858585855
:106BC0005858585858585848585858585858585855
:106BD00048585858585848484848484848585858B5
:106BE00048484858585848484858585848484858B5
:106BF0005848484848484848484848484848484805
:106C00004848484848484848484848484848484804
:106C100048484848484848484848484848484848F4
:106C200048484848404848484848484848484848EC
:106C3000484848484848484000000000000000001C
:106C40000000000000000000000000000000000044
:106C50000000000000000000000000000000000034
:106C60000000000000000000484800000000000094
:106C70000000000000000000000000000000000014
:106C80000000000000000000000000000000000004
:106C900000000000000000004848484848484848B4
:106CA0004848484848484048484840484848484874
:106CB00048484848484048484040480048484840BC
:106CC0004800484848484000000000000048484844
:106CD00048484848484848000048484848484848C4
:106CE000000000000048484848484848484848488C
:106CF0004848484848484800404840484800000044
:106D0000000000000048000000484848000048001B
:106D10000000000000484800000048480000000053
:106D2000480000000000000000000000000000001B
:106D300000000000000000000048480000000000C3
:106D400000000000004800000000004800000000B3
:106D500000000000000000480048484848000000CB
:106D6000000000000000484848484800484848489B
:106D7000480048484848480048484800000000008B
:106D800000480000000048484848484848000000C3
:106D90000000484848484848484848484848484803
:106DA000484848484848484848484800000048483B
:106DB0004848484848484848484848485848484843
:106DC000484858484848480058484848484858485B
:106DD000484848485848484848485848484800584B
:106DE00058484848005858585858585848585858BB
:106DF0005858484858585858485848585858585853
:106E00005858585858585848585858585858585812
:106E10005858485848585848484848485848484892
:106E20004848584848480058580000005858585892
:106E300058585858585858585858585858585858D2
:106E400058585858585858585860606060585858A2
:106E50006060605858586060605858585860605872
:106E600058585858585858585858584858585858B2
:106E700048585858585800606060606060606060B2
:106E8000606060606060606060606060606060481A
:106E9000586060606048586060606048005860609A
:106EA000604848485858606060604848486060588A
:106EB00000484860606000484860606000480060CA
:106EC0006060480048606060606060606060606052
:106ED00060606058606060606060606060606060BA
:106EE00060606060606060606060606060606060A2
:106EF000606058606060606060606060606060609A
:106F00006060606060606060606060606060606081
:106F10006060606060606060606060606060606071
:106F20006048606060606000606060605848486011
:106F300060584848486060606060605848606060C1
:106F400060584860606060584860606060584860A1
:106F500060606060006060606060586058606060A1
:106F60006060606060606048486060606048486081
:106F700060606048486060606048006060606048D1
:106F80000060605858486060605860606060605899
:106F90005860605858585860606060005860606081
:106FA00060004860606058484860605858485860C1
:106FB0005858584848585858484800585858004851
:106FC00048585848484848585858585848585858A1
:106FD0004858485858584858485858585858485881
:106FE0005858585848485858585848484858584881
:106FF00048585858584848484048484848404848E1
:1070000048484848484848484800000000000048B0
:1070100048000000004848484800004048484848A8
:1070200000404848484800004048484800000048A0
:107030004848480000484848480000000000000058
:107040000000000000000000000000000000000040
:1070500000000000000000484848484000484848F8
:107060004848004048484848480000000000484060
:1070700040000000000000000000000000000000D0
:107080000000000000000000000000000000000000
:1070900000000048480000000048480000000000D0
:1070A00000000000000000000000000000000000E0
:1070B00000000000000000000000000000000000D0
:1070C0000000000000000000000040000000000080
:1070D00000000000000000000000000000000000B0
:1070E0000000000000000000484800484800000080
:1070F0000000004848484848480000000000480098
:107100004848484848000000000000000000000017
:10711000000000000000004848484848480048482F
:1071200048484848484848484848484848484848DF
:10713000484848484800000000000048484848487F
:107140004800000000004848484848484848484827
:1071500048484848484848484848484848484848AF
:10716000484848484800004848484848484848482F
:1071700048484848484848484848005858484848B7
:10718000484848484848484848484848484848487F
:10719000484848484848484848484848484848486F
:1071A00048484848484848585858585858484848FF
:1071B000585858484848484848484848484848481F
:1071C000484848484848484848484848484848483F
:1071D00040484848404848585858585858585858AF
:1071E00058585848484848484848484848484848EF
:1071F0004848484848484848404040484848484827
:10720000484848484840405858584800484848006E
:1072100048484848484848484848484848484848EE
:1072200048484848484848404848484848484848E6
:10723000484000004040404848484858584848485E
:1072400048485848484848484848484848484848AE
:1072500048484848484848484848484848484848AE
:10726000484040404040005848585860605858587E
:1072700058606000004848485848484848484848CE
:10728000484848484848484800000048000000482E
:107290004800000000000060586060605858586066
:1072A00058484848000048484848484848484848DE
:1072B0004848484848000000000000480048484846
:1072C000480000000000000048484848604848481E
:1072D000484848484848484848484848484848482E
:1072E00048484848480000000000004848484848CE
:1072F000480000000000006060585858585858482E
:1073000058585848004858585848484848484848E5
:1073100048484848480000000000004800484848E5
:10732000480000000000005858585858585858480D
:10733000585858584848484848484848484848488D
:1073400048484848480000000000004848484800B5
:1073500048000000000000584848484800480048DD
:10736000484848484848484848484848484848489D
:10737000484848484800000000000048484848483D
:1073800048000000000000485858584848484848FD
:1073900048484848004848484848484848484848B5
:1073A0004848484848000000000000484840484815
:1073B00048000000000000484848484848484848FD
:1073C00048484848484800000048484800004848A5
:1073D00048000048480000004040484800484848ED
:1073E00048000000000000484848484848000000A5
:1073F000000000004848484848484848404048483D
:1074000048484848484848484848484848484848FC
:107410004800000000000048484848484800000074
:107420004848480048000000000048484840000024
:107430004848484048004848484848004848484864
:107440004800484848484848484848484848484804
:10745000484848484848484848000000484048488C
:107460004800004848484848000000484848484804
:10747000484848484800004848484848484848481C
:10748000484848484848484848484848484848487C
:1074900048484848484848484848480000000000D4
:1074A00000000000000000484848484000484800EC
:1074B0004840004848484848004848484800004874
:1074C000484840480048000000000000000000005C
:1074D000000000404000000000000000000000002C
:1074E000000000000000000000000000000000009C
:1074F000000000000000000000000000000000008C
:10750000000040404040400000000000000000003B
:10751000000000000000000000000000000000402B
:1075200040400000000000404040000000000040DB
:10753000000000000000400000000000000000000B
:10754000000000000000000000000000000000003B
:1075500000000000000000000000400000000000EB
:10756000004040400000000000000000000000005B
:10757000000000000000000000000000000000000B
:10758000000000000040400000000040404040007B
:107590000000404040400000484848404000000093
:1075A000000040000000000000000000000000009B
:1075B00000000000000000000000000000000000CB
:1075C0000000000000000048484848484040404053
:1075D000400000404040404000000000404040006B
:1075E000000000004000000000000000000000401B
:1075F00000000000000000484848484848000000DB
:10760000000000000000000000000000000000007A
:10761000000000000000000000000000000000006A
:1076200000000000000040484848484848004040EA
:10763000400000000000000000000000000000000A
:10764000000000000000000000000000000000003A
:1076500000404040400000484848484848404040BA
:107660004848480000000000000000000000000042
:1076700000000000000000000000000000004000CA
:10768000000000404048404848484848484848486A
:107690004848480000000000000000000000000012
:1076A000000000000000400000000000000000009A
:1076B000000040000000004840484848484848480A
:1076C00048484800000000000000000000000000E2
:1076D000000000000000000000000040000000006A
:1076E000000000000000004848484848004848485A
:1076F00048004800000000000000000000000000FA
:107700000000000000000000000000000000000079
:1077100000000000000000484848484848484848E1
:107720004848480000000000000000000000000081
:107730000000000000000000000000000000000049
:107740000000000000000048004848484848004049
:107750004040480000000000000000000000000061
:107760000000000000000000000000000000000019
:107770000000000000000048004848484848004811
:107780004848480000000000000000000000000021
:1077900000000000000000000000000000000000E9
:1077A0000000000000000048484848004848484899
:1077B0004800480000000000000000000000000039
:1077C00000000000000000000000000000000000B9
:1077D0000000000000000048484048484048404839
:1077E0004848480040400000000000000000000041
:1077F0000000000000000000000000000000000089
:1078000000000000000000480040404040480048A0
:107810004848480000000000400000000000000050
:107820000000000000000000000000000000000058
:1078300000000000000000404040404040484848F0
:107840004848480000000000000000000000000060
:107850000000000000000000000000000000000028
:107860000000000000000000404048484800484830
:1078700048404800000040400000000000000000B8
:1078800000000000000000000000000000000000F8
:107890000000000000000048484840000048404008
:1078A0004000004040404840400000000000000010
:1078B00000000000000000000000000000000000C8
:1078C00000000000000000000000000000000000B8
:1078D0000000004000400000000000000000000028
:1078E0000000000000000000004000000000000058
:1078F0004000000000404000000000404000000048
:107900000000000000000000000000000000000077
:10791000004040404000000040004840400000401F
:107920004040004040000040400000004000404017
:1079300040404000000040004000000000000040C7
:107940004000000000484040004800484840404097
:107950000040404848404040400000000000404097
:107960004040004040000040404040404000404017
:107970000000404040404000000000404000000047
:1079800000404040400000000000000000000000F7
:107990000000000000000000004040000000004027
:1079A0004040000000404040404000004040404017
:1079B0004000004040404040404040000000404007
:1079C00000400000404040004000000040404000B7
:1079D00000404040000000004040400000000040E7
:1079E000404048004040400000404040400000000F
:1079F000004040000000000040000000000048403F
:107A0000000000004800400000000040004000006E
:107A10000040404000000000000000000040000066
:107A200000000040400000000040404048484848F6
:107A3000484000484800484040404800000040405E
:107A40004000000000404000000000000000000076
:107A500000000048484800000048484848000048E6
:107A600048484848484848484848484800484848DE
:107A70004840484848484800000000000000000016
:107A800000000000000000000000000000004000B6
:107A90004848000000484848000048004848484816
:107AA000484848480048000000000000000000006E
:107AB0000000000000000000004040404000004086
:107AC00040404040000000404040404800404048A6
:107AD000480048004040480000000000000000004E
:107AE0000000000000000000000000000000000096
:107AF0000000400000404800004040404040480036
:107B0000404848404848480000000000000000008D
:107B10000000000000000000000000000000000065
:107B200000004848004848484848484048484800FD
:107B300048004040484800000000000000000000ED
:107B40000000000000000000000000000000000035
:107B5000480000000000000000000048480000004D
:107B60000000000000000000000000000000000015
:107B700000004800000000000000000000000000BD
:107B80000000004800000000000000000000004865
:107B9000000000000040000048484048484848486D
:107BA000484848000000000048000000000000486D
:107BB00048484848480000000000004848484848F5
:107BC00048000000000000484848484848484848E5
:107BD00048484800000000000048484848484848D5
:107BE00048484848480000000000004848484848C5
:107BF00048000000000000404048484848404040DD
:107C0000404048004040404848484040404848487C
:107C1000484848484800004848484848480000004C
:107C200000000000000000484848404040484048EC
:107C300048404048484848484848484848484848D4
:107C400048404048484848484000000000000000C4
:107C50000000000000000000404040404840404814
:107C60004840404040484048484848484000004854
:107C700048484848484848484848480000000000EC
:107C80000048484848484840400000000040404004
:107C9000000000404040404040484840404040488C
:107CA00048484840404848404848480000484848FC
:107CB000484848484848480000000000004040400C
:107CC00000000048404040000000404040000040AC
:107CD0004048400000404048400000484048404084
:107CE00000484848484040000000000000000000F4
:107CF0000000000000000000000000000000000084
:107D0000004000000000004040404800004040406B
:107D10004000004040404000000000000000000023
:107D20000000000000000000000000000000000053
:107D30004040400000484848484848484848404873
:107D40004840484848484800000000000000000043
:107D500000000000000000000040000000000040A3
:107D60004040404000484040404040484848404033
:107D70004048484848404000000000000000000023
:107D800000000000000000000000000000000000F3
:107D9000004040404000000040404040400040481B
:107DA000404040484040400000000000000000000B
:107DB00000000000000000000000000000000000C3
:107DC00040400000000000404040404000000048AB
:107DD00048484040484848000000000000000000BB
:107DE0000000000000000000000000000000000093
:107DF0000000000000000040404040404040484833
:107E000048484800404048000000000000000000D2
:107E10000000000000000000000000000000000062
:107E20000000000000404040404040484040404882
:107E30004048484848404000000000000000000062
:107E400000000000000000000000000000400000F2
:107E5000000040404840404000404040000000409A
:107E6000404840404048480000000000000000003A
:107E70000000000000000000000000000000000002
:107E80000000000000400000000000404000000032
:107E9000004048404048480000000000000000004A
:107EA00000000000000000000000000000000000D2
:107EB00000000000000000000000004040000048FA
:107EC00048484848484848000000000000000000BA
:107ED0000000000000000000400000000000000062
:107EE0000000000000000000000000484848484032
:107EF0004048484848484800000000000000000092
:107F00000000004000000000004040400000000071
:107F10004040404000000040404040404048484011
:107F200040484848484840000000404040000000A9
:107F30000000000000000000000000000000000041
:107F40000000000000004040404000000040404071
:107F50004040000040404040400040400040404021
:107F600040404000004040404000000000404000D1
:107F70000000000040000000000000000048000079
:107F800040404848484848004040480000004800F9
:107F90004000004000000040004000000000404061
:107FA0000000000000404000000000404040404011
:107FB0004048484048484840404040404000004019
:107FC0004040400040404040004048484840404019
:107FD0004848484800484848484848484848484869
:107FE0004848484848484800000000400040000019
:107FF0000040404040000000404040404000004001
:1080000040004040404840404800404848484848B8
:108010004848484848484840404800404048484848
:108020000000404048484848004040004848480058
:108030004040000000404040404040484848004028
:1080400040484848484848404040400000400040C0
:108050004040404040404040404840404040404810
:108060004840404040004848404000004848484898
:108070000048484048484800000000004800000010
:1080800000000040400000000040000000004840A8
:108090004000000000404040000048404000000018
:1080A0004800404040000040400000000000400008
:1080B0000040000000000000004800000000000038
:1080C0000000004848484848484848484848484808
:1080D00048000000000000004848484848000000F0
:1080E0000000004800400040480000000000004838
:1080F00000000040404800004048004800000000E8
:10810000400000000000004848000000000048480F
:10811000484800400000000000000000000000008F
:1081200000484848484000004848000000004848CF
:108130004800000000000000000000000000484867
:1081400048000000000000000000000000000000E7
:108150000000000000004848484848004848484897
:10816000484848480000000000404000000000006F
:108170004000000000000000004848484848000057
:10818000000000000000000000484848484848003F
:10819000480048484848484848000000000000009F
:1081A00000000000000000000000000000000000CF
:1081B0000000000000000000000000480000000077
:1081C0000048000000000000000000000000000067
:1081D000000048000000000048000000004848007F
:1081E00000000000000000000048480000000000FF
:1081F000000000000048480000000000000048485F
:108200000048004848484848480000000000000076
:1082100000000000004848484848000000000000F6
:10822000484848000000000000000000004848489E
:1082300048484848484848484800000000000000B6
:10824000000000000000000000000000000000002E
:10825000484848484848480000484848484848482E
:10826000484848484848484848004848484848001E
:10827000000048484800484800000048484848482E
:10828000484848000000004848484848484848488E
:108290004848484840484848484848484848484866
:1082A00048484848480000000048484848484800B6
:1082B000000000000000004848484848480048487E
:1082C00000004848484848484848484848484848BE
:1082D000484848484848484848484800000000483E
:1082E00048000000000000484848484848484848BE
:1082F00048484848484848484848484848484848FE
:1083000048484848484848484848484848484848ED
:108310004800000000000048484848484048484895
:1083200048484848484848484848484848484848CD
:108330004848484848484848000000484848484895
:108340004800000000000040404840404048404095
:108350004040404848480000484848484848484845
:1083600048484848480048484848484800000000F5
:108370000000000000000048484848484848484875
:10838000484848484848484848484848484848486D
:108390004848484848484848484848000000484835
:1083A0004800484800000048484848484048484875
:1083B000484848484848484848484848484848483D
:1083C00048484848484848484800004848484848BD
:1083D00048000000000000404040484848484848E5
:1083E0004848484848484848484848484848004855
:1083F0004848484848004848484848480000000065
:1084000000000000000000484840484848484848EC
:108410004848484848484848480048484848484824
:10842000000000484848484848000000480000480C
:10843000480000000000004848484848484848486C
:1084400048484848484848484848484848484848AC
:108450000000484848000000004848484800000024
:108460000000484848480048484848484840404874
:10847000484848484848004848484848004848480C
:108480004848004848484848480048000000000064
:10849000480000484800004848484040484848488C
:1084A0004848404848484848484848484848484854
:1084B000484848484848484848484848484848483C
:1084C00048000000000000484848484848404040F4
:1084D000484848484848484848484848484848481C
:1084E000484800484848484848004848484848489C
:1084F000000000004848484848484848484848481C
:1085000048484848484848484848484848484848EB
:1085100048004848484848480048484848484800B3
:10852000480048484848004848484848484848485B
:10853000484848484800004848484848484848484B
:1085400048484848484848484848484848480048F3
:1085500048484848480048484848484048484848EB
:10856000484848484848484848484848484848488B
:10857000484848484848484848484848484848487B
:108580004800000000000040404840484848404043
:108590004048484848484848484848484848484863
:1085A000484848484848484848484848484848484B
:1085B00048000000000000484848484848484848EB
:1085C0004848484848484800484848484848484873
:1085D0004848484848484848484848404848484823
:1085E00048000000000000484848484848484848BB
:1085F0004848484800484848484848484848484843
:1086000048484848484848484848484848484848EA
:10861000484040404000404848484848484848484A
:1086200048484848484848484848484848484848CA
:1086300048484848484848484848484848484848BA
:10864000480000004048484848484848484848488A
:10865000484848484848484848484848484848489A
:10866000484848484848484848404048484848489A
:10867000484848480000004848480000004848482A
:10868000484848484848484848484848484848486A
:1086900048484848484040404000004800000048E2
:1086A0004800404848480000000000000048484892
:1086B0004848484848484848484848484848004882
:1086C000480000484800004848484848404040406A
:1086D0004000000000000000000000000048484882
:1086E000484848484848484848000000000048407A
:1086F0004040000048484848484848400040400042
:108700000000000000004000000000000048484851
:108710004848484848484848484800000000004841
:108720004848000000484848484848000000000009
:108730004040484848484800000000000048484879
:1087400048484848484848484800000000000000A1
:108750000000000000484848484848404848484809
:108760004848484848484800000000000048484839
:108770004848484848480000000000000000000049
:1087800000000000004848484848484848484848D1
:108790004848484800000000000000000048000071
:1087A0000000000048484848480000000000000061
:1087B00000000000000000000000004848480040A1
:1087C0000000000000004800000000000000000061
:1087D0000000000048000000000000000000000051
:1087E0000000000000000000000000400000000049
:1087F000000048000000000002060000FB00FF002F
:1088000000F405030C05040C05030C05040C050518
:108810000000FF00083803005901085401083F0018
:10882000050000FF00084203006301084A010853E5
:1088300000050000FF00010A0000E202010501013D
:108840000301010102050000FF0000E702030C0420
:10885000050000FF0000F100085A020403020404AE
:1088600002040502040602050000FF0002060008DB
:10887000320000DD00FF00020600082D080504009C
:1088800000E208050400FF0001000007A00000EC62
:108890000100FE00010100FF0001030000E20301EE
:1088A0000604010903050000FF0002010107C801D9
:1088B00006000100EC00FF0002040000F10400F9D2
:1088C00000FF00020300077F0008320104060104D4
:1088D0000601040601070003077F000832010406B1
:1088E0000104060104060107000308320007200105
:1088F000040601040601040601040601070003083A
:108900003200070F010406010406010406010406F3
:1089100001070001050000FF0000C4000209020475
:108920000400FF00077F0002030000FF000837017A
:108930000404010404010404010404010404010406
:108940000401040401040401040403076400083260
:1089500001040401040401040401040401040401E9
:108960000404010404010404010404030750000882
:108970002D0104040104040104040104040104049D
:108980000104040104040104040104040307320087
:10899000082801040401040401040401040401047E
:1089A000040104040104040104040104040307286D
:1089B00000082D010404010404010404010404015D
:1089C0000404010404010404010404010404030771
:1089D0001400083201040401040401040401040425
:1089E0000104040104040104040104040104040159
:1089F000050000FF0007FF0001090000F60207FF65
:108A00000000F100010602010100FF000209000060
:108A1000F100FF0007FF0002030000FC000828012E
:108A20000405010404010403010402010401000916
:108A300090000A6002040102040102040102040120
:108A40000204010204010204010204010204010201
:108A5000040102040102040102040102050000FFF6
:108A60000002020106000100E000FF000201010611
:108A7000000100E000FF0002080106000100E00024
:108A8000FF0002050106000100E000FF00020901ED
:108A900006000100E000FF0002030007000009409B
:108AA000000A1E0100140500000106000100FB0180
:108AB000FF000700000940000A1E01001405000025
:108AC0000106000100FB01FF000000F78700000025
:108AD00000000000FF870000000000000013880075
:108AE00000000000000024880000000001000035A4
:108AF000880000000000000049880000000000001D
:108B0000005488000000000000006B880000000096
:108B10000000007688000000000100008788000047
:108B20000000010000988800000000000000A988F3
:108B300000000000000000B78800000000000000F6
:108B4000C28800000000000000188900000000003A
:108B50000000238900000000000000F489000000EC
:108B6000000000000B8A00000000000000138A00D3
:108B7000000000000000608A000000000000006BA0
:108B80008A00000000000000768A0000000000005B
:108B900000818A000000000000008C8A00000000B4
:108BA000000000978A000000000200A9B18A0000BE
:108BB000000120003E3E2050524553532042205495
:108BC0004F20474F204241434B203C3C00414E4404
:108BD00020474554205448452046524545204741AA
:108BE0004D45204D4F44555321005452592054486F
:108BF00045204E45585420444946464943554C5417
:108C0000204C4556454C004841524400415645527F
:108C1000414745004541535900444946464943555B
:108C20004C54204C4556454C3A00544F54414C202E
:108C300053554E4B2053484950533A00594F5520F5
:108C4000574F4E20544845204C4556454C21002B4B
:108C50002B2B2B2B2B2B2B2B2B2B2B2B2B2B2B2B64
:108C60002B2B2B2B00434F4E47524154554C415414
:108C7000494F4E204350542E003E3E205052455303
:108C800053204220544F20474F204241434B203C29
:108C90003C004F4E20594F5552204E455854204DC0
:108CA000495353494F4E2100414E442054525920BC
:108CB000544F2053554E4B204D4F52452053484959
:108CC000505300504C415945522C20504C45415373
:108CD00045204C4F4F4B20464F525741524400576E
:108CE0004954482054484520424552454156454440
:108CF000210054484520555A45424F5820434F4D76
:108D00004D554E495459204D4F55524E5300544FD6
:108D100054414C2053554E4B2053484950533A0030
:108D200054484520454E454D5920464F5243452015
:108D30005741532048415244210054484520454E54
:108D4000454D5920464F52434520574153204156E7
:108D50004552414745210054484520454E454D590F
:108D600020464F52434520574153204541535921F6
:108D7000004D414E5920534F554C5320464F5220E1
:108D800054484520474F44204F46205448452057DB
:108D9000415445522100414E442048452053554EF0
:108DA0004B205448452048414C4620454E454D599E
:108DB00020464C45455421004954205741532054E6
:108DC000484520574152204F4620544845205041A5
:108DD00043494649432100414E44204845205355CC
:108DE0004E4B2041204C4F54204F46205348495071
:108DF0005321004E4557204D4554414C20464F527B
:108E000020544845204F4345414E2100414E4420C7
:108E100048452053554E4B204D414E59205348490B
:108E20005053210042555420544F4F204C4553532A
:108E300020544F204D454E54494F4E2100414E4441
:108E40002048452053554E4B20412046455720533E
:108E5000484950532100544F4F204C455353205400
:108E60004F204D454E54494F4E2100414E4420481D
:108E7000452053554E4B204E4F20534849505321C7
:108E8000004E455645522046494E4420534F4D45CD
:108E90004F4E45204C494B452048494D21004845FF
:108EA00020574153205448452042455354204F46B3
:108EB00020544845204245535421212100414E442D
:108EC000204845204449454420534F20594F554E92
:108ED00047210048452057415320412047524541F2
:108EE00054204649474854455221004954275320AD
:108EF0005245414C4C592053414420544841542040
:108F00004845275320474F4E4521004845205741AB
:108F10005320414E204153504952494E4720475516
:108F2000592100484520464F554E4453205448454A
:108F300020444541544820564552592051554943F3
:108F40004B2100495420574153204E4F542048494B
:108F500053204441592100434F4D4D414E44455209
:108F6000204F46205448452053554E4B454E2053E4
:108F700055424D4152494E45210054484520552EF9
:108F80005A2E452E204E4156592043484F495220D3
:108F9000484F4E4F525320544845002B2B2B2B2B20
:108FA0002B2B2B2B2B2B2B2B2B2B2B2B2B2B00481F
:108FB0004F4E4F52494E4720544845204352455743
:108FC000003E3E205052455353204220544F2047EC
:108FD0004F204241434B203C3C00484152443A2000
:108FE0004C4556454C203800415645524147453A7C
:108FF000204C4556454C20313000454153593A20CC
:109000004C4556454C20313500594F555220474F5D
:10901000414C3A0053544152542B53454C3A204250
:1090200041434B20544F204D41494E204D454E5514
:1090300000593A204C4F4144494E472047414D4545
:1090400000583A20534156494E472047414D45006C
:10905000534C3A20535552464143494E47005352D0
:109060003A20444956494E4700413A204649524524
:1090700020544F525045444F00422B55502F444FDF
:10908000574E3A20494E43522F44454352204259AD
:10909000203130300055502F444F574E3A20534521
:1090A000542044495354414E4345205748454E208F
:1090B000494E2052414E4745004C4546542F524997
:1090C0004748543A205455524E494E472053434F37
:1090D000504500434F4E54524F4C533A00594F5550
:1090E00052204D495353494F4E2049533A2053493A
:1090F0004E4B20414C4C20534849505321212121B3
:10910000212100434F4E5441435420414E442041BD
:109110004C4C20594F55204841564520544F20442F
:109120004F20494E00534541212043555252454E50
:10913000544C59205448455245275320454E454DDF
:109140005920434F4E544143542100594F5520411B
:109150005245204120434F4D4D414E444552204FF2
:10916000462041205355424D4152494E45204154DD
:10917000002B2B2B2B2B2B2B2B2B2B00425249451F
:1091800046494E4700465245452047414D4500005F
:1091900011241FBECFEFD0E1DEBFCDBF14BE88E1EA
:1091A0000FB6F89480936000109260000FBE11E03B
:1091B000A0E0B1E0EEEFF6EE02C005900D92A23114
:1091C000B107D9F71CE0A2E1B1E001C01D92A43FB4
:1091D000B107E1F70E94BA4C882311F40E948A4D2E
:1091E000F894EDEEF9E080E881939BE0E93FF90720
:1091F000D9F78DEE99E09093FA0B8093F90B1092CA
:10920000FB0B1092FE0B1092040C10920A0C1092A1
:10921000100C1092D6091092D80982E18093D709D8
:1092200080EE8093E0098093DE0984E18093DF097A
:109230008093DD091092E4091092E3091092E80985
:109240001092E70981E08093FD0B0E94005820E90D
:1092500030E0F90185919491FC01F07090832E5FCC
:109260003F4F80E02E3B3807A1F778940E94395990
:109270000E947C600C947D730C94000030EE3A9553
:109280000C944249E1F70C944549C2E1D1E000EE6B
:10929000A02E662776E035D13BE23A95F1F70E94A1
:1092A000784931E13A95F1F7AA9489F0C895639528
:1092B000683029F033E03A95F1F70000ECCF6627EB
:1092C000002430E5C30FD01DC8950000E4CF35E081
:1092D0003A95F1F70000000014D1E091D80942E07E
:1092E000E427E160E093D809E2E0E09336000895D6
:1092F000DE014D915D91679FC001480F591FFA0132
:1093000028E2059108B94D91059108B95D91059143
:1093100008B900C0059108B9480F591F059108B94F
:109320000591FA012A9508B961F7C895002708B98F
:1093300008950F921F92EF93FF93EFB7EF93E09191
:109340008400E251F1E0EF1700F0F395FA30D8F322
:109350000C94AA49E091D709EA95E093D709F091D6
:10936000D609F0FD57C0EC3098F0F3E0F093890097
:10937000FDE8F0938800E0FB289826F4E1E00E94E5
:109380007A4BB8C0E5E1EA95F1F70000289AB2C03F
:10939000E63038F100C000C02898E0FBE4E016F4A5
:1093A0000E947A4BE4E0E0933600E6E0E0936F0041
:1093B000A1C0EF93EFB7EF93E0918400ED55E1305A
:1093C00000F0E23000F0E33000F0E43000F0E5308F
:1093D00000F0289AE2E0E0936F00EF91EFBFEF9189
:1093E000189500C0E0FB289826F4E1E00E947A4B33
:1093F00005C0E5E1EA95F1F70000289AE091D70968
:10940000E03009F077C0EDEFE093D709E1E0E093B9
:10941000D60970C0E7E0E0938900EBE1E0938800B3
:1094200000C02898E2E000C00E947A4BFDEF009057
:10943000DD09F019E091D709EF17E0F4FDEF009096
:10944000DD09F0190090DE09F019EF1798F0EDE151
:10945000FF2700800F92EA95E1F70FE10A95F1F7F7
:10946000000000000E943E49E1E0FF270F900192BA
:10947000EE31E0F3E091D709E03009F03BC02F93E3
:109480003F934F935F936F937F938F939F93AF938C
:10949000BF9378941124EE27E093D609E2E1E0939C
:1094A000D709F091DF09F093DD09F091E009F0931D
:1094B000DE09E091D909F091DA09E115F10509F029
:1094C00009950E94A94C0E9456580E948C4A11246A
:1094D000E091DB09F091DC09E115F10509F009954E
:1094E000BF91AF919F918F917F916F915F914F91BC
:1094F0003F912F91EF91EFBFFF91EF911F900F9050
:1095000018952898E2E000C00E947A4BE091D709B4
:10951000EA95E093D7090895E091FD0BE0FD0E94E4
:10952000434F0090FB0B002019F4ADEEB9E002C0F0
:10953000A3EFBAE021E002260092FB0B22E0209389
:10954000FC0BE091FD0BE0FF08952F923F924F92AC
:109550005F926F927F928F929F92AF92BF92CF92C3
:10956000DF92EF92FF920F931F93CF93DF9350916F
:10957000100C6091140C7091150C8091130C40909C
:10958000110C5090120C66248090180C9090190CBD
:10959000A090160CB090170C1D01C3E8840D651D3A
:1095A000761D6815790508F0B501FB014491450366
:1095B0001D92840D651D761D6815790508F0B501AD
:1095C000FB01449145031D92CA9541F7D1012090BA
:1095D000FF0B3090000C4090020C5090030C6090F8
:1095E000010C1091FE0B7090050C8090060C909071
:1095F000070CA090080CB090090C2091040CC090AE
:109600000B0CD0900C0CE0900E0CF0900F0C009115
:109610000D0C30910A0C9FEFCC91DD27C7FDDFEFD9
:10962000620C431CF201449141030008C10DD01D9E
:10963000970CA81CF501449142030008C10DD01DF0
:109640000C0DED1CF701449143030008C10DD01D22
:109650000024C038D0050CF0CFE70A94C038D005FC
:109660000CF4C0E8C058CD939A9509F0D5CF40913D
:10967000FC0B4A954093FC0B97E009F0CDCF60922C
:10968000010C4092020C9092070CA092080C0093DF
:109690000D0CE0920E0C5093100C6093140C709310
:1096A000150C8093130CDF91CF911F910F91FF90B8
:1096B000EF90DF90CF90BF90AF909F908F907F9072
:1096C0006F905F904F903F902F900895E091F90B2D
:1096D000F091FA0B019100000093B3000BE0E93F19
:1096E000F0070DEE19E008F0F801E093F90BF093A4
:1096F000FA0B08950F931F932F93EF93E091F90BBB
:10970000F091FA0B01910093B3000BE0E93FF007F1
:109710000DEE19E008F0F801E093F90BF093FA0B65
:10972000E8E0EA95F1F7EF912F911F910F91E0FD9D
:10973000289AE0FF01C00895F4E1FA95F1F700C01E
:10974000E1FD289AE1FF00C0089599277727E8E016
:10975000F4EA660F771FE60FF71FA591B491EEEFBD
:10976000FBE026E0289FE00DF11DA183B2831124C8
:10977000089599277727EEEFFBE026E0289FE00D7C
:10978000F11D76EA760F75831124089599277727BE
:10979000EEEFFBE026E0289FE00DF11D6083112431
:1097A0000895E0E6F4E0A2E1B1E06091D2097091A1
:1097B000D3096D937D933197E1F71124089599278B
:1097C000552728E2220F629F880F080E191EA2E17A
:1097D000B1E0A00DB11D6091D2097091D30920E3D1
:1097E000429F600D711D6D937C93112408959927FC
:1097F000772728E2220F629F880F080E191EA2E128
:10980000B1E0A00DB11D6091D4097091D50920E39C
:10981000429F600D711D529F700D6D937C931124BA
:1098200008958093D2099093D30908958093D40921
:109830009093D50908958091D80981700895209159
:10984000D8092E7F2093D8090895882329F4809180
:10985000E1099091E20908958091E5099091E60966
:109860000895F999FECF92BD81BD60BDF894FA9A32
:10987000F99A78940895F999FECF92BD81BDF89434
:10988000F89A80B5789408958093EA099093EB094B
:1098900008950F931F9380E694E0A2E1B1E0E09178
:1098A000EA09F091EB0940E30091D4091091D50940
:1098B00065917591649F9001749F300D200F311F49
:1098C0002D933D930197A1F711241F910F910895B6
:1098D000129AC895C895C895C895129820E030E0AE
:1098E00080E090E040E03695279596958795C8955D
:1098F000C895C895C8951398009B3068019B9068DF
:10990000139AC895C895C895C8954F5F403159F7C7
:109910003093E2092093E1099093E6098093E509E9
:109920008091E1099091E2090F9731F08091E5096A
:109930009091E6090F9761F428E088E190E00FB676
:10994000F894A895809360000FBE20936000FFCF2D
:10995000089510921F0C009903C081E080931F0CA2
:10996000019905C080911F0C826080931F0C0E949A
:10997000684C08951F9380E090E00E943B4C182FA4
:1099800081E090E00E943B4C90E0382F20E0210FD6
:10999000311D2A55354509F491E0892F1F9108950D
:1099A000A0E0B0E0E6EDFCE40C94B4726C01062F8C
:1099B000B72E0E94BA4C882309F440C08FEFC81616
:1099C0008FEFD80611F481E03CC0EE24FF24C701DC
:1099D0000E943B4C182FC70101960E943B4CD82F88
:1099E000C0E0CE01810F911D8C159D0531F49FEFD4
:1099F000E9169FEFF90659F423C080E290E0E80EE3
:109A0000F91E90E0E91694E0F90609F719C0802FD5
:109A10009B2D9C01E90170E2C72ED12CC20ED31EF2
:109A200087010F5F1F4FC7010E943B4C8993CC15E4
:109A3000DD0511F480E005C07801F2CF84E001C0BB
:109A400083E0CDB7DEB7E9E00C94D072A0E0B0E0DF
:109A5000ECE2FDE40C94B4726C010E94BA4C8823D1
:109A600011F484E04EC0F60180819181FFEF8F3FB9
:109A70009F0709F445C08A55954509F441C001E0A6
:109A800010E0F0E2EF2EF12CC7010E943B4CB82E03
:109A9000C70101960E943B4CD82FC0E09E012B0DC0
:109AA000311DF601808191812817390719F411239E
:109AB000B1F00EC02F5F3F4F19F4112309F4102F9E
:109AC0000F5F80E290E0E80EF91E0034E9F61EC058
:109AD000E12EFF24E5E0EE0CFF1CEA95E1F7C0E083
:109AE000D0E0F601EC0FFD1FCE018E0D9F1D6081B1
:109AF0000E94314C2196C032D10599F780E001C017
:109B000081E0CDB7DEB7E9E00C94D072112301F704
:109B100082E0F7CFCF93DF93C0E0D0E0FE01E059C1
:109B2000FF4FE491CE016E2F0E94314C2196C0323E
:109B3000D105A1F7C0E2D0E0CE016FEF0E94314C19
:109B4000CE0101966FEF0E94314CA09688E0C030A4
:109B5000D80791F7DF91CF910895FC0145870895CB
:109B60000895FC0180818F7580830895FC018081B8
:109B7000806480830895FC0144870895FC01478335
:109B80000895FC01408708951F93CF93DF93EC0164
:109B9000162F898190E0FC01EE0FFF1FE85FFB4567
:109BA00025913491E42FFF27E7FDF095E80FF91F89
:109BB000EE0FFF1FE85FFB45859194916091270CA4
:109BC000821B930B70E00E9476729B0161157105F8
:109BD00011F421E030E0812F90E0FC01EE0FFF1F37
:109BE000E80FF91FEE0FFF1FE250F44F81819281C1
:109BF000820F931F928381833B832A8388818860AD
:109C000088838981840F8C83DF91CF911F91089580
:109C10004093270C089590937D0C80937C0C8FE6E5
:109C200080937F0C1092EC09E2E2FCE090E18FEF70
:109C300028E1908313868187828716862087958303
:109C400076963CE0EA37F307A1F708959C01E2E23B
:109C5000FCE080818F77808376968CE0EA37F80786
:109C6000C1F7C90101969093840C8093830C909363
:109C7000210C8093200C9093860C8093850C10927D
:109C8000810C1092800C10927B0C10927A0C109226
:109C90007E0C1092820C81E08093EC0908958AEF8B
:109CA00080932F0C8093450C80935B0C8093710CF8
:109CB0001092EC090895DC01ED91FC911197AF0130
:109CC0004F5F5F4F11965C934E93E4912E2F30E0DF
:109CD000E7FF13C02F7730703695322F2227379544
:109CE0002795FA014F5F5F4FE4918E2F8F77280FF2
:109CF000311DE7FDF1CF4D935C93C9010895862F87
:109D0000642F0E94B94B0895EF92FF920F931F9317
:109D1000CF93DF93182F062FE22E86E1189FE001E4
:109D20001124CE5DD34FF8801A8A1D869FEF9C8741
:109D30004B871B8A8F2D8062877B88831F82998740
:109D40002983133049F51092130C89E0689FC001F4
:109D5000112420917C0C30917D0C280F391FF901C2
:109D60003196459154915093150C4093140CF90180
:109D7000359685919491840F951F9093170C80933D
:109D8000160CF901379685919491480F591F5093FD
:109D9000190C4093180C04C0812F60E00E94B94B4D
:109DA000812F6E2D0E94A54BF7FE02C00F8701C0C8
:109DB0000E8789E0089FC0011124E0917C0CF0918E
:109DC0007D0CE80FF91F339625913491211531054B
:109DD00019F41D8A1C8A07C0F9018491898B2F5FB1
:109DE0003F4F3D8B2C8BCDB7DEB7E6E00C94D372A2
:109DF0001F93782F142FA82FB0E086E190E0A89F42
:109E0000F001A99FF00DB89FF00D1124EE5DF34F06
:109E10003081532F35FF02C037FD33C02223F9F4C0
:109E200086E190E0A89FF001A99FF00DB89FF00D8A
:109E30001124EE5DF34F8585882311F456FF1386B8
:109E400086E190E0A89FF001A99FF00DB89FF00D6A
:109E50001124EE5DF34F80818F7B808312C086E1F9
:109E600090E0A89FF001A99FF00DB89FF00D11247C
:109E7000EE5DF34F3F773083872F422F212F0E94D3
:109E8000844E1F910895AF92BF92DF92EF92FF929E
:109E90000F931F93CF93DF93A2E2BCE0CFEFDBE001
:109EA0001D968C911D978823B9F0282F332727FD05
:109EB00030951C968C911C97280F311D2F3F310532
:109EC00019F014F02FEF30E0C90137FF02C080E035
:109ED00090E01C968C931C978C9183FF26C0129661
:109EE0004D915C91139728813981240F351F398357
:109EF000288314968C911497E82FF0E0EE0FFF1F43
:109F0000E85FFB45859194911416150624F42817F3
:109F1000390730F40AC0452B41F08217930728F027
:109F2000998388838C91877F8C93569626964CE0F4
:109F3000AA37B40709F0B4CF8091EC09882309F05F
:109F4000DEC0F1C0E091830CF091840CCF0101964A
:109F50009093840C8093830C44914F3F69F5AC013E
:109F60004F5F5F4F5093840C4093830CFC018491AE
:109F70008F3219F41092EC09D0C0863009F0B2C0CB
:109F8000FA013196CF0101969093840C8093830C53
:109F9000E491E33529F49093860C8093850CA2C05C
:109FA000E53409F09FC08091850C9091860C9093C8
:109FB000840C8093830C96C047FF02C040937E0CB4
:109FC00020917E0C322F3F7047FF08C0019690937E
:109FD000840C8093830C0197FC014491822F90E0C4
:109FE000807F9070803B910531F1803C910509F4B0
:109FF0006DC08039910509F075C0E091830CF09136
:10A00000840C3196F093840CE093830C3197E491A7
:10A01000832F90E08C9FD0018D9FB00D9C9FB00D41
:10A020001124AE5DB34FEE0F832F1E966C912E2F31
:10A030000E94F84E57C0E091830CF091840C319649
:10A04000F093840CE093830C31972491473071F4A2
:10A05000832F90E08C9FF0018D9FF00D9C9FF00D61
:10A060001124EE5DF34F220F22873CC04B3071F478
:10A07000832F90E08C9FF0018D9FF00D9C9FF00D41
:10A080001124EE5DF34F220F21872CC04C3571F463
:10A09000832F90E08C9FF0018D9FF00D9C9FF00D21
:10A0A0001124EE5DF34F220F27831CC04436D1F4F8
:10A0B000832F90E08C9FF0018D9FF00D9C9FF00D01
:10A0C0001124EE5DF34F220F20870CC0832F90E008
:10A0D0008C9FF0018D9FF00D9C9FF00D1124EE5D83
:10A0E000F34F468783E89CE00E945B4E9093810C7F
:10A0F0008093800C10927B0C10927A0C02C0C6E107
:10A10000D0E020917A0C30917B0C8091800C909162
:10A11000810C2817390709F415CF2F5F3F4F309373
:10A120007B0C20937A0CC2E2DCE00EEF1BE0FF24F4
:10A13000EFEFAE2EB12CDC2EED2E888186FD3DC0DA
:10A140008C899D89892B09F435C09A89898998174A
:10A1500068F530C0EC89FD89CF0101969D8B8C8B11
:10A1600024912F3F31F488818F7788831D8A1C8A40
:10A1700021C001969D8B8C8B0197FC014491822F0D
:10A1800090E0880F991F82549F4FFC0125913491D4
:10A190008D2D9E2D6F2DF9010995EC89FD89319644
:10A1A000FD8BEC8B3197E491E98B1A8A9A89898926
:10A1B000981781F28A898F5F8A8B888185FD03C019
:10A1C00020E030E070C08B898F3F11F08F5F8B8B68
:10A1D000888187FF02C08FEF01C08A859B85992304
:10A1E00009F45BC02C85222309F457C0882309F4A5
:10A1F00054C040917F0C442309F44FC0899FC00193
:10A20000112480509F4F892F992730E0B901869FF4
:10A210009001879F300D969F300D112420503F4FA5
:10A22000232F3327898590E0FC012E9FC0012F9FAB
:10A23000900D3E9F900D112480509F4F892F99279C
:10A24000242F30E0AC01429FC001439F900D529FEC
:10A25000900D112480509F4F292F33278F81882301
:10A26000F1F0EE81F0E0E050FA45E491E058E89F2B
:10A27000C001112480509F4F892F9927B501681B79
:10A28000790B629FC001639F900D729F900D112406
:10A2900080509F4F292F332702C020E030E08E816D
:10A2A0009885890F8E83F8012083F39466960A5F60
:10A2B0001F4FF4E0FF1609F03ECFDF91CF911F91C1
:10A2C0000F91FF90EF90DF90BF90AF900895582FBF
:10A2D000762F89E0589FC0011124E0917C0CF09109
:10A2E0007D0CE80FF91F9491892F8150823010F472
:10A2F00043E021C0923011F444E01DC08091380C3D
:10A3000087FF16C08091470C851711F4442381F410
:10A3100080914E0C87FF0EC080915D0C851711F463
:10A32000442341F490914B0C8091610C891710F4F7
:10A3300041E001C042E0242F30E086E190E0289F18
:10A34000F001299FF00D389FF00D1124EE5DF34FC1
:10A35000808180688083842F652F472F20E50E94AD
:10A36000844E0895FF920F931F938C01862FF42E35
:10A37000642F0E94A54BF801F1828081877F808342
:10A380001F910F91FF900895FC01862F6181641B3E
:10A3900061830E94A54B0895FC01862F9181490F8E
:10A3A0004183642F0E94A54B089500000000000027
:10A3B000000000000000000000000000000000009D
:10A3C000000000000000000000000000000000008D
:10A3D000000000000000000000000000000000007D
:10A3E000000000000000000000000000000000006D
:10A3F000000000000000000000000000000000005D
:10A4000080E08093FD0B08952200240026002800A0
:10A410002B002D0030003300360039003D00400095
:10A42000440048004C00510056005B00600066008C
:10A430006C00730079008100880090009900A200F0
:10A44000AC00B600C100CC00D800E500F30001016B
:10A45000100121013201440157016C018101980171
:10A46000B001CA01E5010202210241026402880230
:10A47000AE02D7020303300361039403CB03050448
:10A4800042048304C70410055D05AF050506610697
:10A49000C206290796070908830805098E09200ABC
:10A4A000BA0A5D0B0A0CC10C840D510E2B0F121051
:10A4B00007110A121D1340147415BA1614188319C3
:10A4C000071BA31C571E24200E22142439267F2884
:10A4D000E82A752D293006330F364539AD3C494001
:10A4E0001B442848734CFE50CF55EA5A51600C6605
:10A4F0001D6C8B725A79928037885090E598FDA137
:10A500009FABD3B5A3C00000000000000000000016
:10A51000000000000000000000000000000000003B
:10A52000000000000000000000000000000000002B
:10A53000000000000000000000000000000000001B
:10A54000000000000000000000000000000000000B
:10A5500000000000000000000000000000000000FB
:10A5600000000000000000000000000000000000EB
:10A5700000000000000000000000000000000000DB
:10A5800000000000000000000000000000000000CB
:10A5900000000000000000000000000000000000BB
:10A5A00000000000000000000000000000000000AB
:10A5B000000000000000000000000000000000009B
:10A5C000000000000000000000000000000000008B
:10A5D000000000000000000000000000000000007B
:10A5E000000000000000000000000000000000006B
:10A5F000000000000000000000000000000000005B
:10A60000000306090C101316191C1F2225282B2ED7
:10A61000313336393C3F414447494C4E51535558EC
:10A620005A5C5E60626466686A6B6D6F70717374A9
:10A63000757678797A7A7B7C7D7D7E7E7E7F7F7F62
:10A640007F7F7F7F7E7E7E7D7D7C7B7A7A79787648
:10A6500075747371706F6D6B6A68666462605E5C5E
:10A660005A585553514E4C494744413F3C39363373
:10A67000312E2B2825221F1C191613100C09060336
:10A6800000FDFAF7F4F0EDEAE7E4E1DEDBD8D5D23D
:10A69000CFCDCAC7C4C1BFBCB9B7B4B2AFADABA808
:10A6A000A6A4A2A09E9C9A9896959391908F8D8C2B
:10A6B0008B8A888786868584838382828281818152
:10A6C0008181818182828283838485868687888A4C
:10A6D0008B8C8D8F9091939596989A9C9EA0A2A416
:10A6E000A6A8ABADAFB2B4B7B9BCBFC1C4C7CACDE1
:10A6F000CFD2D5D8DBDEE1E4E7EAEDF0F4F7FAFDFE
:10A70000808182838485868788898A8B8C8D8E8FD1
:10A71000909192939495969798999A9B9C9D9E9FC1
:10A72000A0A1A2A3A4A5A6A7A8A9AAABACADAEAFB1
:10A73000B0B1B2B3B4B5B6B7B8B9BABBBCBDBEBFA1
:10A74000C0C1C2C3C4C5C6C7C8C9CACBCCCDCECF91
:10A75000D0D1D2D3D4D5D6D7D8D9DADBDCDDDEDF81
:10A76000E0E1E2E3E4E5E6E7E8E9EAEBECEDEEEF71
:10A77000F0F1F2F3F4F5F6F7F8F9FAFBFCFDFEFF61
:10A78000000102030405060708090A0B0C0D0E0F51
:10A79000101112131415161718191A1B1C1D1E1F41
:10A7A000202122232425262728292A2B2C2D2E2F31
:10A7B000303132333435363738393A3B3C3D3E3F21
:10A7C000404142434445464748494A4B4C4D4E4F11
:10A7D000505152535455565758595A5B5C5D5E5F01
:10A7E000606162636465666768696A6B6C6D6E6FF1
:10A7F000707172737475767778797A7B7C7D7E7FE1
:10A8000000020406080A0C0E10121416181A1C1E58
:10A8100020222426282A2C2E30323436383A3C3E48
:10A8200040424446484A4C4E50525456585A5C5E38
:10A8300060626466686A6C6E70727476787A7C7E28
:10A840007F7D7B79777573716F6D6B696765636108
:10A850005F5D5B59575553514F4D4B4947454341F8
:10A860003F3D3B39373533312F2D2B2927252321E8
:10A870001F1D1B19171513110F0D0B0907050301D8
:10A88000FFFDFBF9F7F5F3F1EFEDEBE9E7E5E3E1C8
:10A89000DFDDDBD9D7D5D3D1CFCDCBC9C7C5C3C1B8
:10A8A000BFBDBBB9B7B5B3B1AFADABA9A7A5A3A1A8
:10A8B0009F9D9B99979593918F8D8B898785838198
:10A8C00080828486888A8C8E90929496989A9C9E98
:10A8D000A0A2A4A6A8AAACAEB0B2B4B6B8BABCBE88
:10A8E000C0C2C4C6C8CACCCED0D2D4D6D8DADCDE78
:10A8F000E0E2E4E6E8EAECEEF0F2F4F6F8FAFCFE68
:10A900007F7F7F7F7F7F7F7F7F7F7F7F7F7F7F7F57
:10A910007F7F7F7F7F7F7F7F7F7F7F7F7F7F7F7F47
:10A920007F7F7F7F7F7F7F7F7F7F7F7F7F7F7F7F37
:10A930007F7F7F7F7F7F7F7F7F7F7F7F7F7F7F7F27
:10AC00000309131E28313A40464C5054585B5E618C
:10AC1000636567696B6C6E6F70717273747576774C
:10AC2000777879797A7A7B7B7C7C7C7D7D7D7E7E72
:10AC30007E7E7F7F7F7F7F7F7F7F7F7F7F7F7F7F26
:10AC40007F7F7F7F7F7F7F7F7F7F7F7F7F7E7E7E17
:10AC50007E7D7D7D7C7C7C7B7B7A7A797978777749
:10AC6000767574737271706F6E6C6B696765636112
:10AC70005E5B5854504C46403A31281E130903007D
:10AC8000C6CCD5DBDFE3E5E7E9EAEBECEDEEEFEF91
:10AC9000F0F0F0F1F1F1F1F2F2F2F2F2F2F2F2F39D
:10ACA000F3F3F3F3F3F3F3F3F3F3F3F3F3F3F3F374
:10ACB000F3F3F3F3F3F3F3F3F3F3F3F3F3F3F3F364
:10ACC000F3F3F3F3F3F3F3F3F3F3F3F3F3F3F3F354
:10ACD000F3F3F3F3F3F3F3F3F3F3F3F3F3F3F3F344
:10ACE000F2F2F2F2F2F2F2F2F1F1F1F1F0F0F0EF51
:10ACF000EFEEEDECEBEAE9E7E5E3DFDBD5CCC60010
:10AD000000283D42302D2C2B2C2D2E2F3032333568
:10AD100037393B3D3F414345484A4C4E50535557C8
:10AD2000595B5D5F61636567696B6C6E70717374AD
:10AD3000757778797A7B7C7D7D7E7E7F7F7F7F7F54
:10AD40007F7F7F7F7F7F7E7E7D7D7C7B7A7978773A
:10AD500075747371706E6C6B69676563615F5D5B61
:10AD600059575553504E4C4A484543413F3D3B3956
:10AD700037353332302F2E2D2C2B2C2D30423D28C1
:10AD800000E9E5FED4D7D7D7D6D4D2D0CECCCAC826
:10AD9000C6C3C1BFBDBAB8B6B4B1AFADABA9A7A564
:10ADA000A3A19F9E9C9A999795949391908F8D8C37
:10ADB0008B8A898888878685858484848383838336
:10ADC0008383838383848484858586878888898A2E
:10ADD0008B8C8D8F909193949597999A9C9E9FA11F
:10ADE000A3A5A7A9ABADAFB1B4B6B8BABDBFC1C337
:10ADF000C6C8CACCCED0D2D4D6D7D7D7D4FEE5E9F0
:10AE0000F9F8F9F5EBE1DDDEE0E2E4E5E6E5E4E2C0
:10AE1000DED9D2CAC1B7ACA299918A8683818080DB
:10AE20008182838586888A8C8D8F90929395969760
:10AE300098999A9B9B9C9D9D9D9E9E9E9F9F9F9F48
:10AE40009F9F9F9E9E9E9D9D9D9C9B9B9A99989740
:10AE500096959392908F8D8C8A8886858382818047
:10AE6000808183868A9199A2ACB7C1CAD2D9DEE229
:10AE7000E4E5E6E5E4E2E0DEDDE1EBF5F9F8F90032
:10AE80000708070B151F2322201E1C1B1A1B1C1E44
:10AE900022272E363F49545E676F767A7E7F7F7F0A
:10AEA0007F7E7D7B7A7876747371706E6D6B6A6964
:10AEB000686766656564646363626262616161615B
:10AEC0006161616262626363636465656667686944
:10AED0006A6B6D6E7071737476787A7B7D7E7F7F1E
:10AEE0007F7F7E7A766F675E54493F362E27221E1B
:10AEF0001C1B1A1B1C1E2022231F150B07080700F2
:10AF00001F313D444E5354565A5F64696E747679CE
:10AF10007C7F7F7F7F7F7F7F7F7F7F7F7F7F7F7F44
:10AF20007F7F7F7F7F7F7F7F7F7F7F7F7F7F7F7F31
:10AF30007F7F7F7F7F7F7F7F7F7F7F7F7F7F7F7F21
:10AF40007F7F7F7F7F7F7F7F7F7F7F7F7F7F7F7F11
:10AF50007F7F7F7F7F7F7F7F7F7F7F7F7F7F7F7F01
:10AF60007F7F7F7F7F7F7F7F7F7F7F7F7F7F7F7FF1
:10AF70007F7F7F7F7F7F7F7F7F7F7F7C7871684C43
:10AF80002C1C120C0A0B0A05FDF3E9DFD4CAC0B76A
:10AF9000AEA69E97918B86858280808080808080FF
:10AFA00080808080808080808080808080808080A1
:10AFB0008080808080808080808080808080808091
:10AFC0008080808080808080808080808080808081
:10AFD0008080808080808080808080808080808071
:10AFE0008080808080808080808080808080808061
:10AFF000808080808087919DACC4CBD4DDF2FAFA4A
:10B000000895982F882319F48FEF87B9089581E068
:10B0100080938B0C8093880C9093870C10928A0CF1
:10B020008093890C662321F08091890C8823E1F7B5
:10B030000895982F882311F417B808958CE0809311
:10B040008B0C8FEF8093880C9093870C10928A0C56
:10B0500081E08093890C662321F08091890C8823FC
:10B06000E1F708958091890C8823F9F080918A0C8A
:10B070008823C1F48091870C80938A0C80918B0C7B
:10B08000E82FF0E0ED55F74FE491E7B99091880C87
:10B09000980F90938B0C992311F09D3031F41092FE
:10B0A000890C0895815080938A0C08950E9432582B
:10B0B00008950F931F93CF93DF938C01C0E0D0E0EE
:10B0C00007C00E941B4C8823E1F30E941F4C21966D
:10B0D000C017D107B4F3DF91CF911F910F9108955D
:10B0E00040520E94DF4B0895FF920F931F93CF931E
:10B0F000DF938C01F62EEA01FE0144912196442350
:10B1000049F0802F0F5F1F4F4F7740526F2D0E94E5
:10B11000DF4BF2CFCDB7DEB7E5E00C94D472EF92FF
:10B12000FF920F931F93CF93DF93F62E042FE22EFF
:10B13000EC0110E0002311F4112349F4802F6AE0A0
:10B140000E945672905F8C2F6F2D492F09C0EE2000
:10B1500021F08C2F6F2D40E103C08C2F6F2D40E02C
:10B160000E94DF4B1F5F2197133031F0802F6AE080
:10B170000E945672082FDECFCDB7DEB7E6E00C9402
:10B18000D372A0E0B0E0E7ECF8E50C94B572C62EFF
:10B1900079018A01EC01DD24E114F10401051105B6
:10B1A00011F4DD2069F4C801B7012AE030E040E085
:10B1B00050E00E948972462F405F8C2F6C2D03C097
:10B1C0008C2F6C2D40E00E94DF4BD39421978AE0B6
:10B1D000D81669F0C801B7012AE030E040E050E03D
:10B1E0000E948972C901DA017C018D01D5CFCDB7EA
:10B1F000DEB7E8E00C94D172A0E0B0E0E2E0F9E55F
:10B200000C94B072782E862EEA01FA01C590D49083
:10B21000FA013296A590B49000E016C0FC01EE0D44
:10B22000FF1D3296EE0FFF1FEC0FFD1F459154914D
:10B23000812F870D692D0E94F74B1F5F812F90E0B2
:10B240008C159D055CF30F5F802F90E08A159B05A0
:10B250005CF48C9D70018D9DF00C9C9DF00C112474
:10B2600010E0902E980CEACFCDB7DEB7EDE00C944D
:10B27000CC720F931F938FEE90E00E940B4E08EF5D
:10B2800010E0C8010E94164CC8010E94114C0E9497
:10B29000D14B8EE190E00E94595880E06FEF41E081
:10B2A0000E94675108E418E082E16CE0A8010E9466
:10B2B000FC5883E090E00E94595882E16CE04CE732
:10B2C00058E00E94FC5882E090E00E94595882E1C8
:10B2D0006CE0A8010E94FC5880E490E00E9459585C
:10B2E0000E94D14B84E190E00E9459581F910F9128
:10B2F0000895A0E2B0E0EFE7F9E50C94BB7282E1BB
:10B3000090E09A838983BE016F5F7F4F0E94D04C8B
:10B310008FE190E063E170E042EB5BE80E947458DB
:10B320008B81813061F480910A0190910B0101972A
:10B3300031F48FE163E142E450E00E94F74B8885ED
:10B34000813061F480910A0190910B01029731F4F0
:10B350008FE163E142E450E00E94F74B8D8581303C
:10B3600061F480910A0190910B01892B31F48FE1F6
:10B3700063E142E450E00E94F74B8B81813061F43D
:10B380008885813049F48D85813031F481E090E009
:10B390009093BB0C8093BA0CA096E2E00C94D77209
:10B3A0008BE064E042E050E00E94F74B8CE064E008
:10B3B00043E050E00E94F74B08951F931CE0812F5B
:10B3C0006BE041E050E00E94F74B1F5F1B31B9F783
:10B3D00085E090E00E9459581CE0812F6CE041E02C
:10B3E00050E00E94F74B1F5F1B31B9F783E090E0FC
:10B3F0000E9459581CE0812F6DE041E050E00E940E
:10B40000F74B1F5F1B31B9F783E090E00E9459585A
:10B410001CE0812F6EE041E050E00E94F74B1F5F7F
:10B420001B31B9F71F9108951F930E94337368E68B
:10B4300071E00E947672AA2797FDA095BA2F80939B
:10B44000020190930301A0930401B09305010E94AF
:10B45000387388E090E09093910C8093900C0E9458
:10B4600033736CEB72E00E94767288539F4FAA2769
:10B4700097FDA095BA2F8093F00C9093F10CA093B8
:10B48000F20CB093F30C0E9438731CE0812F6EE035
:10B4900040E050E00E94F74B1F5F1B31B9F71CE002
:10B4A000812F6FE040E050E00E94F74B1F5F1B319F
:10B4B000B9F785E090E00E9459581CE0812F6DE0BB
:10B4C00040E050E00E94F74B1F5F1B31B9F783E06B
:10B4D00090E00E9459581CE0812F6CE040E050E061
:10B4E0000E94F74B1F5F1B31B9F783E090E00E9489
:10B4F00059581CE0812F6BE040E050E00E94F74B70
:10B5000082E167E044E050E00E94F74B83E167E0AE
:10B5100045E050E00E94F74B1F5F1B3159F71F9128
:10B52000089580E162E141E150E00E94F74B86E13D
:10B5300062E142E150E00E94F74B87E090E00E9418
:10B5400059588DE060E941E00E94675181E161E175
:10B5500041E150E00E94F74B85E161E142E150E0BA
:10B560000E94F74B88E090E00E9459588DE060E916
:10B5700041E00E94675182E160E141E150E00E94B8
:10B58000F74B84E160E142E150E00E94F74B89E033
:10B5900090E00E9459588DE060E941E00E946751B7
:10B5A00082E167E044E050E00E94F74B83E167E00E
:10B5B00045E050E00E94F74B80911D0C90911E0CCD
:10B5C000892B09F0E7C02091920C3091930C809167
:10B5D000CE0C9091CF0C2817390709F04EC08091FE
:10B5E000900C8E5F6EE04FE050E00E94F74B80E1E0
:10B5F00062E140E050E00E94F74B86E162E140E00A
:10B6000050E00E94F74B86E090E00E9459588FE08E
:10B6100060E941E00E9467518091900C8E5F6EE07E
:10B6200040E150E00E94F74B81E161E140E050E0F1
:10B630000E94F74B85E161E140E050E00E94F74B4A
:10B6400086E090E00E9459588FE060E941E00E9456
:10B6500067518091900C8E5F6EE041E050E00E9457
:10B66000F74B82E160E140E050E00E94F74B84E15B
:10B6700060E140E050E00E94F74B2091920C309145
:10B68000930C8091CE0C9091CF0C2817390709F4B8
:10B6900081C08091900C8F5F6EE04BE050E00E9483
:10B6A000F74B8091900C8E5F6EE04CE050E00E9472
:10B6B000F74B80E162E140E050E00E94F74B86E109
:10B6C00062E140E050E00E94F74B86E090E00E948B
:10B6D00059588FE060E941E00E9467518091900CD9
:10B6E0008F5F6EE04DE050E00E94F74B8091900C30
:10B6F0008E5F6EE04EE050E00E94F74B81E161E129
:10B7000040E050E00E94F74B85E161E140E050E00D
:10B710000E94F74B86E090E00E9459588FE060E964
:10B7200041E00E94675182E160E140E050E00E9408
:10B73000F74B84E160E140E050E00E94F74B8091DC
:10B74000900C6EE041E050E00E94F74B8091900C2D
:10B750008F5F6EE041E050E00E94F74B8091900CCB
:10B760008E5F6EE041E050E00E94F74B8091900CBC
:10B770008D5F6EE041E050E00E94F74B82E167E0B0
:10B7800044E050E00E94F74B83E167E045E050E081
:10B790000E94F74B80911D0C90911E0C019709F0AF
:10B7A000E7C02091920C3091930C8091CE0C909137
:10B7B000CF0C2817390709F04EC08091900C8E5F8E
:10B7C0006EE041E350E00E94F74B80E162E140E02F
:10B7D00050E00E94F74B86E162E140E050E00E94B9
:10B7E000F74B86E090E00E9459588FE060E941E015
:10B7F0000E9467518091900C8E5F6EE042E350E0B2
:10B800000E94F74B81E161E140E050E00E94F74B7C
:10B8100085E161E140E050E00E94F74B86E090E076
:10B820000E9459588FE060E941E00E946751809181
:10B83000900C8E5F6EE041E050E00E94F74B82E199
:10B8400060E140E050E00E94F74B84E160E140E0BD
:10B8500050E00E94F74B2091920C3091930C809114
:10B86000CE0C9091CF0C2817390709F481C0809134
:10B87000900C8F5F6EE04DE250E00E94F74B80919C
:10B88000900C8E5F6EE04EE250E00E94F74B80E13C
:10B8900062E140E050E00E94F74B86E162E140E067
:10B8A00050E00E94F74B86E090E00E9459588FE0EC
:10B8B00060E941E00E9467518091900C8F5F6EE0DB
:10B8C0004FE250E00E94F74B8091900C8E5F6EE04B
:10B8D00040E350E00E94F74B81E161E140E050E03D
:10B8E0000E94F74B85E161E140E050E00E94F74B98
:10B8F00086E090E00E9459588FE060E941E00E94A4
:10B90000675182E160E140E050E00E94F74B84E142
:10B9100060E140E050E00E94F74B8091900C6EE0B7
:10B9200041E050E00E94F74B8091900C8F5F6EE0F9
:10B9300041E050E00E94F74B8091900C8E5F6EE0EA
:10B9400041E050E00E94F74B8091900C8D5F6EE0DB
:10B9500041E050E00E94F74B82E167E044E050E0B4
:10B960000E94F74B83E167E045E050E00E94F74B0F
:10B970000E94337368E671E00E947672AA2797FDF1
:10B98000A095BA2F8093020190930301A093040124
:10B99000B09305010E94387388E090E09093910C79
:10B9A0008093900C0E9433736CEB72E00E9476726D
:10B9B00088539F4FAA2797FDA095BA2F8093F00C2C
:10B9C0009093F10CA093F20CB093F30C0E94387397
:10B9D0001092930C1092920C10921B0C10921A0C55
:10B9E0001092970C1092960C8091E40C9091E50CBB
:10B9F00001969093E50C8093E40C8091BA0C9091A1
:10BA0000BB0C892B61F480918C0C90918D0C85304E
:10BA1000910529F0019790938D0C80938C0C809167
:10BA2000EC0C9091ED0C01969093ED0C8093EC0C46
:10BA30000297B1F48091E80C9091E90C01969093F3
:10BA4000E90C8093E80C1092ED0C1092EC0C8091B4
:10BA5000CE0C9091CF0C01979093CF0C8093CE0C8D
:10BA60008091CE0C9091CF0C892B79F484E090E0FA
:10BA70009093CF0C8093CE0C8091C00C9091C10C10
:10BA800001979093C10C8093C00C8091C00C909151
:10BA9000C10C019761F483E090E09093CF0C809308
:10BAA000CE0C84E090E09093C10C8093C00C809108
:10BAB0000201909103010E9438730E94337368E67B
:10BAC00071E00E947672AA2797FDA095BA2F809305
:10BAD000020190930301A0930401B09305010E9419
:10BAE000387388E090E09093910C8093900C809153
:10BAF000F00C9091F10C0E9438730E9433736CEB40
:10BB000072E00E94767288539F4FAA2797FDA095F6
:10BB1000BA2F8093F00C9093F10CA093F20CB09399
:10BB2000F30C0E9438731092930C1092920C1092A6
:10BB30001B0C10921A0C1092970C1092960C80917C
:10BB40001D0C90911E0C019690931E0C80931D0C61
:10BB500008951F9383E060E941E00E9467511CE073
:10BB6000812F6BE041E050E00E94F74B1F5F1B31DB
:10BB7000B9F789E090E00E94595883E060E941E01C
:10BB80000E9467511CE0812F6CE041E050E00E9470
:10BB9000F74B1F5F1B31B9F786E090E00E945958C0
:10BBA00083E060E941E00E9467511CE0812F6DE075
:10BBB00041E050E00E94F74B1F5F1B31B9F786E070
:10BBC00090E00E94595882E060E941E00E9467518C
:10BBD0001CE0812F6EE041E050E00E94F74B1F5FB8
:10BBE0001B31B9F71092DD0C1092DC0C1F910895F7
:10BBF0001F930E94337368E671E00E947672AA2751
:10BC000097FDA095BA2F8093020190930301A09312
:10BC10000401B09305010E94387388E090E090938E
:10BC2000910C8093900C0E9433736CEB72E00E9435
:10BC3000767288539F4FAA2797FDA095BA2F8093BD
:10BC4000F00C9093F10CA093F20CB093F30C0E94C3
:10BC5000387383E060E941E00E9467511CE0812F66
:10BC60006EE040E050E00E94F74B1F5F1B31B9F7D8
:10BC70001CE0812F6FE040E050E00E94F74B1F5F17
:10BC80001B31B9F789E090E00E94595882E060E9E1
:10BC900041E00E9467511CE0812F6DE040E050E0E0
:10BCA0000E94F74B1F5F1B31B9F786E090E00E94BE
:10BCB000595882E060E941E00E9467511CE0812F01
:10BCC0006CE040E050E00E94F74B1F5F1B31B9F77A
:10BCD00086E090E00E94595882E060E941E00E94CD
:10BCE00067511CE0812F6BE040E050E00E94F74B71
:10BCF00082E167E044E050E00E94F74B83E167E0B7
:10BD000045E050E00E94F74B1F5F1B3159F78091CF
:10BD1000E60C9091E70C05979093E70C8093E60C66
:10BD20001F9108958091CC0C9091CD0C0196909329
:10BD3000CD0C8093CC0C069761F48AE164E045E178
:10BD400050E00E94F74B8BE164E046E150E00E9436
:10BD5000F74B8091CC0C9091CD0C0C9789F48AE133
:10BD600064E043E150E00E94F74B8BE164E044E182
:10BD700050E00E94F74B81E060E941E00E9467518A
:10BD80008091CC0C9091CD0C429721F41092CD0C67
:10BD90001092CC0C08958091D60C9091D70C0196FE
:10BDA0009093D70C8093D60C069761F482E167E0FC
:10BDB00044E050E00E94F74B83E167E045E050E04B
:10BDC0000E94F74B8091D60C9091D70C0C9789F478
:10BDD00082E167E042E050E00E94F74B83E167E0D8
:10BDE00043E050E00E94F74B81E060E941E00E94AF
:10BDF00067518091D60C9091D70C429721F4109204
:10BE0000D70C1092D60C089583E160E14AE150E02E
:10BE10000E94F74B89E090E00E9459588DE060E95C
:10BE200041E00E94675183E160E140E050E00E9400
:10BE3000F74B83E161E14BE150E00E94F74B88E072
:10BE400090E00E9459588DE060E941E00E946751FE
:10BE500083E161E140E050E00E94F74B83E162E161
:10BE60004CE150E00E94F74B87E090E00E94595867
:10BE70008DE060E941E00E94675182E061E00E944C
:10BE8000195880E061E00E94015883E162E140E0DE
:10BE900050E00E94F74B8FE060E941E00E9467515B
:10BEA0000E94145A1092DD0C1092DC0C1092930C2C
:10BEB0001092920C10921B0C10921A0C0E94DD59D9
:10BEC0001092970C1092960C1092D50C1092D40CE4
:10BED00082E167E044E050E00E94F74B83E167E0D5
:10BEE00045E050E00E94F74B20911D0C30911E0C54
:10BEF0002115310531F48091E60C9091E70C0F97F4
:10BF000008C02130310549F48091E60C9091E70C8E
:10BF100049979093E70C8093E60C2F5F3F4F309347
:10BF20001E0C20931D0C08951F930E94D14B8AE094
:10BF300060E14DE150E00E94F74B1BE0812F60E192
:10BF400041E250E00E94F74B1F5F1032B9F780E2E8
:10BF500060E14EE150E00E94F74B8AE061E143E28C
:10BF600050E00E94F74B8AE062E143E250E00E9419
:10BF7000F74B8AE063E143E250E00E94F74B8AE02E
:10BF800064E143E250E00E94F74B8AE065E14FE153
:10BF900050E00E94F74B80E261E144E250E00E94F1
:10BFA000F74B80E262E144E250E00E94F74B80E20E
:10BFB00063E144E250E00E94F74B80E264E144E236
:10BFC00050E00E94F74B80E265E140E250E00E94C1
:10BFD000F74B1BE0812F65E142E250E00E94F74BF6
:10BFE0001F5F1032B9F78DE090E061E170E045EF3E
:10BFF00058E00E9474588DE090E062E170E048E102
:10C0000059E00E9474588091BA0C9091BB0C019732
:10C0100041F481E190E06FE070E045E851E90E9471
:10C02000745880910A0190910B01019741F48DE0C1
:10C0300090E063E170E043E559E00E94745880911C
:10C040000A0190910B01029741F48DE090E063E1C9
:10C0500070E046E659E00E94745880910A01909180
:10C060000B01892B41F48DE090E063E170E049E73A
:10C0700059E00E94745880910C0190910D01892B18
:10C0800041F48DE090E064E170E042EB59E00E9401
:10C09000745880910C0190910D01029741F48DE04C
:10C0A00090E064E170E04FE959E00E94745880919B
:10C0B0000C0190910D01019741F48DE090E064E155
:10C0C00070E04CE859E00E94745885E090E068E127
:10C0D00070E04CE50E94705887E090E068E170E005
:10C0E00040EB58E00E94745883E063E041EB50E27B
:10C0F0000E94FC581F910895A0E0B0E0E2E8F0E64D
:10C100000C94AD721092BD0C1092BC0C80E00E9499
:10C11000254C86E090E00E9459581092DD0C109258
:10C12000DC0C84E090E09093CF0C8093CE0C909345
:10C13000C10C8093C00C1092CB0C1092CA0C1092C0
:10C14000E50C1092E40C84E690E09093E70C809369
:10C15000E60C88E691E0909301018093000188E667
:10C1600091E0A0E0B0E08093020190930301A093DE
:10C170000401B093050184EF91E0A0E0B0E080936A
:10C18000060190930701A0930801B0930901109252
:10C190001C0C8DE49CE00E94114C87E493E20E9409
:10C1A000164C81EF97E10E94444C0E9479590E94FD
:10C1B000945F8BE061E147E150E00E94F74B8CE037
:10C1C00061E148E150E00E94F74B84E090E06DE0CF
:10C1D00070E04CEC58E00E9474588091D00C909123
:10C1E000D10C892B41F488EC9AE80E940B4E85EC27
:10C1F00099E00E94264E8091D00C9091D10C01972D
:10C2000021F41092D10C1092D00C0E94795954E074
:10C21000652E712C45E0842E912C36E0A32EB12C96
:10C220002EE1C22ED12C9DE2E92EF12C0CE310E080
:10C2300083E0482E512C0E94337368E671E00E941F
:10C240007672AA2797FDA095BA2F8093020190934A
:10C250000301A0930401B093050180E00E94254CE6
:10C26000EC0188709170892B09F4F0C08091BC0CAE
:10C270009091BD0C892B09F049C080E00E94254CAB
:10C28000892BD9F780910201909103010E943873A4
:10C2900083E061E00E94195885EC99E00E944F4EBE
:10C2A00080910A0190910B018130910529F410933E
:10C2B0008D0C00938C0C0EC08230910529F4F09205
:10C2C0008D0CE0928C0C06C0892B21F4D0928D0C41
:10C2D000C0928C0C80910C0190910D0181309105E0
:10C2E00029F4B092990CA092980C0EC0823091055E
:10C2F00029F49092990C8092980C06C0039721F42F
:10C300007092990C6092980C0E943E698091BC0CCE
:10C310009091BD0C019711F40E9498718091BC0C12
:10C320009091BD0C029709F046C080910A0190914E
:10C330000B01019690930B0180930A01019761F420
:10C340008DE090E063E170E043E559E00E947458AD
:10C3500010938D0C00938C0C80910A0190910B012D
:10C36000029761F48DE090E063E170E046E659E009
:10C370000E947458F0928D0CE0928C0C80910A010E
:10C3800090910B01039781F48DE090E063E170E000
:10C3900049E759E00E947458D0928D0CC0928C0CE1
:10C3A00010920B0110920A0180E00E94254C892B0B
:10C3B000D9F70E9479598091BC0C9091BD0C0397DC
:10C3C00009F044C080910C0190910D010196909369
:10C3D0000D0180930C01019761F48DE090E064E120
:10C3E00070E04CE859E00E947458B092990CA09209
:10C3F000980C80910C0190910D01029761F48DE0F1
:10C4000090E064E170E04FE959E00E947458909226
:10C41000990C8092980C80910C0190910D010397DA
:10C4200081F48DE090E064E170E042EB59E00E941D
:10C4300074587092990C6092980C10920D011092A1
:10C440000C0180E00E94254C892BD9F79E01207CAD
:10C4500009F44FC08091BC0C9091BD0C029709F07B
:10C4600046C080910A0190910B01019690930B01B7
:10C4700080930A01019761F48DE090E063E170E040
:10C4800043E559E00E94745810938D0C00938C0C76
:10C4900080910A0190910B01029761F48DE090E088
:10C4A00063E170E046E659E00E947458F0928D0C0A
:10C4B000E0928C0C80910A0190910B01039781F41A
:10C4C0008DE090E063E170E049E759E00E94745824
:10C4D000D0928D0CC0928C0C10920B0110920A011C
:10C4E00080E00E94254C892BD9F70E947959C6FD1E
:10C4F00002C0C7FF4BC08091BC0C9091BD0C03974C
:10C5000009F044C080910C0190910D010196909327
:10C510000D0180930C01019761F48DE090E064E1DE
:10C5200070E04CE859E00E947458B092990CA092C7
:10C53000980C80910C0190910D01029761F48DE0AF
:10C5400090E064E170E04FE959E00E9474589092E5
:10C55000990C8092980C80910C0190910D01039799
:10C5600081F48DE090E064E170E042EB59E00E94DC
:10C5700074587092990C6092980C10920D01109260
:10C580000C0180E00E94254C892BD9F7CE018073E5
:10C590009070892B09F44FCE6091BC0C6F5E8BE0DC
:10C5A00049E150E00E94F74B6091BC0C6F5E8CE05B
:10C5B00049E150E00E94F74B81E060E941E00E94D0
:10C5C0006751C4FF0DC08091BC0C9091BD0C0097C9
:10C5D00029F45092BD0C4092BC0C17C0019711C0B9
:10C5E000C472D070CD2B89F08091BC0C9091BD0CA1
:10C5F0008330910529F41092BD0C1092BC0C05C03B
:10C6000001969093BD0C8093BC0C6091BC0C6F5E46
:10C610008BE047E150E00E94F74B6091BC0C6F5EED
:10C620008CE048E150E00E94F74B80E00E94254CEE
:10C63000892BD9F700CEA0E2B0E0E1E2F3E60C945A
:10C64000B77285EC99E00E94264E0E94D14B8BE098
:10C6500090E062E070E045E65CE80E9474588AE091
:10C6600090E063E070E04FE45CE80E9474588BE077
:10C6700090E067E070E04CE35CE80E94745889E069
:10C6800090E068E070E04AE25CE80E9474588DE156
:10C6900090E068E070E04091E40C21E00E948F5847
:10C6A00087E090E06AE070E049E15CE80E9474583D
:10C6B00080910A0190910B01019741F489E190E08A
:10C6C0006AE070E044E15CE80E94745880910A01DD
:10C6D00090910B01029741F489E190E06AE070E0EB
:10C6E0004CE05CE80E94745880910A0190910B0123
:10C6F000892B41F489E190E06AE070E047E05CE872
:10C700000E94745884E090E06CE070E04AEE5BE8D0
:10C710000E94745889E090E06DE070E04DEC5BE8B9
:10C720000E94745888E090E069E170E044EB5BE8B7
:10C730000E94745882E190E09A838983BE016F5F02
:10C740007F4F0E94D04C80910A0190910B01813063
:10C75000910519F481E08B830AC08230910519F4A8
:10C7600081E0888704C0892B11F481E08D87CE0198
:10C7700001960E94264D01E010E06EE0E62EF12CBD
:10C7800080E00E94254C80FFFBCF10930D010093A9
:10C790000C0110930B0100930A011093D10C00932C
:10C7A000D00C86E090E00E9459581092CB0C109269
:10C7B000CA0CF0928F0CE0928E0C1092DD0C10924D
:10C7C000DC0C0E947C60DCCF0F931F93CF93DF9330
:10C7D00085EC99E00E94264E0E94D14B8BE090E0C0
:10C7E00062E070E04FEA5FE80E9474588AE090E0EF
:10C7F00063E070E04BE95FE80E94745881E090E0EC
:10C8000066E070E04AE75FE80E94745881E090E0DB
:10C8100067E070E047E55FE80E9474588091E80C9B
:10C820009091E90C039784F481E090E069E070E076
:10C8300043E45FE80E94745881E090E06AE070E0B1
:10C8400043E25FE80E9474588091E80C9091E90CF3
:10C850000397089780F481E090E069E070E04BE096
:10C860005FE80E94745881E090E06AE070E04BEE6F
:10C870005EE80E9474588091E80C9091E90C0B9747
:10C880000A9780F481E090E069E070E043ED5EE8B3
:10C890000E94745881E090E06AE070E04DEB5EE841
:10C8A0000E9474588091E80C9091E90C459784F0AF
:10C8B00081E090E069E070E04EE95EE80E94745823
:10C8C00081E090E06AE070E041E85EE80E94745820
:10C8D0008091E40C9091E50C892B81F481E090E04B
:10C8E0006BE070E04BE65EE80E94745881E090E0F7
:10C8F0006CE070E046E55EE80E9474588091E40CBC
:10C900009091E50C0B9784F481E090E06BE070E08F
:10C910004DE35EE80E94745881E090E06CE070E0C6
:10C9200044E25EE80E9474588091E40C9091E50C1A
:10C930000B970F9780F481E090E06BE070E04CE0A3
:10C940005EE80E94745881E090E06CE070E043EF94
:10C950005DE80E9474588091E40C9091E50C4A9730
:10C960000A9780F481E090E06BE070E047ED5DE8CD
:10C970000E94745881E090E06CE070E048EB5DE864
:10C980000E9474588091E40C9091E50C849784F097
:10C9900081E090E06BE070E046E95DE80E94745849
:10C9A00081E090E06CE070E041E75DE80E9474583F
:10C9B00080910A0190910B01019741F481E090E090
:10C9C0006DE070E047E55DE80E94745880910A01CF
:10C9D00090910B01029741F481E090E06DE070E0EE
:10C9E0004AE35DE80E94745880910A0190910B011E
:10C9F000892B41F481E090E06DE070E040E25DE879
:10CA00000E94745881E090E06EE070E04EE05DE8D6
:10CA10000E94745885E190E06EE070E04091E40C73
:10CA200021E00E948F5881E090E060E170E042EFE9
:10CA30005CE80E94745881E090E061E170E04FEDA5
:10CA40005CE80E94745881E090E062E170E043ECA1
:10CA50005CE80E94745881E090E063E170E048EA8D
:10CA60005CE80E94745881E090E064E170E042E983
:10CA70005CE80E94745888E090E069E170E049E762
:10CA80005CE80E947458C1E0D0E00EE010E080E065
:10CA90000E94254C80FFFBCFD0930D01C0930C0169
:10CAA000D0930B01C0930A01D093D10CC093D00C4A
:10CAB00086E090E00E9459581092CB0C1092CA0C5C
:10CAC00010938F0C00938E0C1092DD0C1092DC0CE6
:10CAD0000E947C60DCCF1F938AE164E045E150E076
:10CAE0000E94F74B8BE164E046E150E00E94F74B77
:10CAF0001CE0812F6CE049E150E00E94F74B812F50
:10CB00006BE049E150E00E94F74B812F6DE049E175
:10CB100050E00E94F74B812F6EE049E150E00E9407
:10CB2000F74B812F6FE049E150E00E94F74B812FD6
:10CB300060E149E150E00E94F74B812F61E149E15A
:10CB400050E00E94F74B812F62E149E150E00E94E2
:10CB5000F74B1F5F1B3169F68EE090E06DE070E0EF
:10CB60004EE259E00E9474588EE090E06FE070E071
:10CB70004AE359E00E94745880E00E94254C887076
:10CB80009170892B89F081E060E941E00E94675152
:10CB900081E090E09093CB0C8093CA0C86E090E00B
:10CBA0000E9459580E94E4631F910895A0E2B0E0EA
:10CBB000ECEDF5E60C94B37280E00E94254C8C01FC
:10CBC000A12CF4E0BF2EA822B92292FF1BC080FF47
:10CBD0004EC390FF4CC38091E60C9091E70C8036D9
:10CBE00091050CF044C305969093E70C8093E60CF6
:10CBF0003EC38091E80C9091E90C01969093E90C6A
:10CC00008093E80CC8018C7090700C97A9F488E0B0
:10CC100060E941E00E94675181E090E09093CB0C85
:10CC20008093CA0C1092DD0C1092DC0C86E090E030
:10CC30000E9459580E947C6006FFF2C08091BE0C91
:10CC40009091BF0C01969093BF0C8093BE0C87E02F
:10CC500060E941E00E9467512091920C3091930C61
:10CC60008091CE0C9091CF0C2817390709F4D8C0C9
:10CC7000809100019091010118161906DCF40197CA
:10CC800090930101809300018091DC0C9091DD0C68
:10CC9000892B49F48091D20C9091D30C01969093FA
:10CCA000D30C8093D20C81E090E09093C90C8093D8
:10CCB000C80C06C088E691E09093010180930001C2
:10CCC0008091900C9091910C8B31910541F08830BE
:10CCD000910529F001969093910C8093900C80918E
:10CCE000900C9091910C0897D9F48091000190914B
:10CCF0000101AA2797FDA095BA2F2091DE0C309153
:10CD0000DF0C4091E00C5091E10C82179307A407CF
:10CD1000B50731F489E090E09093910C8093900CEA
:10CD20008091900C9091910C4B97D9F480910001D7
:10CD300090910101AA2797FDA095BA2F2091DE0CB2
:10CD40003091DF0C4091E00C5091E10C8217930779
:10CD5000A407B50731F487E090E09093910C80939D
:10CD6000900C8091D20C9091D30C039711F5809187
:10CD7000EA0C9091EB0C8D31910541F088309105D2
:10CD800029F001969093EB0C8093EA0C8091EE0CC5
:10CD90009091EF0C8D31910541F08830910529F08B
:10CDA00001969093EF0C8093EE0C1092D30C10929E
:10CDB000D20C8091BE0C9091BF0C089769F48091C1
:10CDC0008E0C90918F0C019690938F0C80938E0C0B
:10CDD0001092BF0C1092BE0C8091EA0C9091EB0C5B
:10CDE0004B9761F489E090E09093EB0C8093EA0C10
:10CDF0008AE16BE041E050E00E94F74B8091EE0C3D
:10CE00009091EF0C4B9761F48AE090E09093EF0CD7
:10CE10008093EE0C8AE16CE041E050E00E94F74B19
:10CE200007FFE3C08091BE0C9091BF0C01969093D8
:10CE3000BF0C8093BE0C87E060E941E00E9467511F
:10CE40002091920C3091930C8091CE0C9091CF0C4C
:10CE50002817390709F4C9C0809100019091010198
:10CE600021E088369207CCF40196909301018093DB
:10CE700000018091DC0C9091DD0C892B49F48091AC
:10CE8000D20C9091D30C01969093D30C8093D20C3A
:10CE90001092C90C1092C80C04C01092010110929B
:10CEA00000018091900C9091910C8830910541F097
:10CEB0008B31910529F001979093910C8093900C00
:10CEC0008091900C9091910C4B97D9F48091000136
:10CED00090910101AA2797FDA095BA2F2091D80C17
:10CEE0003091D90C4091DA0C5091DB0C82179307EA
:10CEF000A407B50731F48AE190E09093910C8093F8
:10CF0000900C8091900C9091910C0897D9F480919D
:10CF1000000190910101AA2797FDA095BA2F2091B9
:10CF2000D80C3091D90C4091DA0C5091DB0C82175F
:10CF30009307A407B50731F48AE190E09093910C30
:10CF40008093900C8091D20C9091D30C039711F5A3
:10CF50008091EA0C9091EB0C8B31910541F0883077
:10CF6000910529F001979093EB0C8093EA0C809146
:10CF7000EE0C9091EF0C8B31910541F089309105C9
:10CF800029F001979093EF0C8093EE0C1092D30C44
:10CF90001092D20C8091BE0C9091BF0C089769F44E
:10CFA00080918E0C90918F0C019790938F0C8093B1
:10CFB0008E0C1092BF0C1092BE0C8091EA0C9091D6
:10CFC000EB0C089731F48AE190E09093EB0C80939E
:10CFD000EA0C8091EE0C9091EF0C099731F48AE104
:10CFE00090E09093EF0C8093EE0C8091900C9091D8
:10CFF000910C419709F094C0E0E1EE2EF12CE02273
:10D00000F12204FF20C088E060E941E00E946751FE
:10D010008091060190910701A0910801B09109014A
:10D02000883E23E0920720E0A20720E0B2075CF4EC
:10D030000196A11DB11D8093060190930701A09355
:10D040000801B093090170E2C72ED12CC022D12271
:10D0500005FF1DC088E060E941E00E9467518091B2
:10D06000060190910701A0910801B09109011816DD
:10D0700019061A061B065CF40197A109B1098093F1
:10D08000060190930701A0930801B0930901E114F0
:10D09000F10419F100FF21C088E060E941E00E943D
:10D0A00067518091060190910701A0910801B0910C
:10D0B0000901843823E0920720E0A20720E0B207AC
:10D0C00064F48D599F4FAF4FBF4F809306019093EB
:10D0D0000701A0930801B0930901C114D10401F123
:10D0E00000FF1EC088E060E941E00E946751809126
:10D0F000060190910701A0910801B09109018536C0
:10D100009105A105B10564F083569040A040B04060
:10D110008093060190930701A0930801B093090141
:10D1200013FF0EC08091DC0C9091DD0C892B41F433
:10D1300081E090E09093DD0C8093DC0C0E94F85D20
:10D14000A114B104A1F08091DC0C9091DD0C019749
:10D1500071F41092DD0C1092DC0C1092930C109272
:10D16000920C10921B0C10921A0C0E94A95D01FFE8
:10D1700036C080E00E94254C892BD9F78DE060E90C
:10D1800041E00E94675181E190E09A8389830E9487
:10D19000BA4C882309F46EC081E190E0BE016F5F54
:10D1A0007F4F0E94D04C882309F064C08B8180930C
:10D1B000E60C1092E70C8F898093E40C1092E50C3A
:10D1C0008D858093E80C1092E90C88858093980CEB
:10D1D0001092990C8A8980938C0C10928D0C11FFFF
:10D1E00021C080E00E94254C892BD9F78DE060E9B1
:10D1F00041E00E94675181E190E09A8389838091A8
:10D20000E40C8F8B8091E60C8B838091E80C8D87EA
:10D2100080918C0C8A8B8091980C8887CE01019626
:10D220000E94264D10FF26C0209106013091070173
:10D2300040910801509109018091F00C9091F10CFE
:10D24000A091F20CB091F30C281739074A075B073D
:10D2500019F40E94915A0EC080E00E94254C892B3F
:10D26000D9F78EE060E941E00E94675103C010FDEC
:10D27000C0CCC8CCA096EAE00C94CF72EF92FF929B
:10D280000F931F93CF93DF930EE010E010938F0C5A
:10D2900000938E0C85EC99E00E944F4E81E090E067
:10D2A0009093E90C8093E80C1092DD0C1092DC0C4A
:10D2B00010921C0C88E090E09093910C8093900C5D
:10D2C0001093EB0C0093EA0C86E190E09093EF0C46
:10D2D0008093EE0C0E9433736CEB72E00E947672C6
:10D2E00088539F4FAA2797FDA095BA2F8093F00CE3
:10D2F0009093F10CA093F20CB093F30C0E9438734E
:10D3000080E061E00E9401580E94494C8BE064E09B
:10D3100044E050E00E94F74B8CE064E045E050E0D0
:10D320000E94F74B82E167E044E050E00E94F74B37
:10D3300083E167E045E050E00E94F74B8AE164E05A
:10D3400045E150E00E94F74B8BE164E046E150E09C
:10D350000E94F74B8091EA0C6BE045E250E00E949E
:10D36000F74B8091EA0C8F5F6BE046E250E00E9441
:10D37000F74B8091EA0C8E5F6BE047E250E00E9431
:10D38000F74B8091EE0C6CE045E250E00E94F74BC9
:10D390008091EE0C8F5F6CE047E250E00E94F74B0B
:10D3A0000FE010E0ACE0EA2EF12C80918E0C909111
:10D3B0008F0C0B9721F410938F0C00938E0C80919F
:10D3C0008E0C90918F0C409721F4F0928F0CE0928C
:10D3D0008E0C8091DC0C9091DD0C892B09F0B3C090
:10D3E00080918E0C6FE043E350E00E94F74B8091F8
:10D3F0008E0C8F5F6FE044E350E00E94F74B80910A
:10D400008E0C8E5F6FE045E350E00E94F74B8091F9
:10D410008E0C8D5F6FE046E350E00E94F74B8091E9
:10D420008E0C8C5F6FE047E350E00E94F74B8091D9
:10D430008E0C8B5F6FE048E350E00E94F74B8091C9
:10D440008E0C8A5F6FE049E350E00E94F74B8091B9
:10D450008E0C895F6FE04AE350E00E94F74B8091A9
:10D460008E0C885F6FE04BE350E00E94F74B809199
:10D470008E0C875F6FE04CE350E00E94F74B809189
:10D480008E0C865F6FE04DE350E00E94F74B809179
:10D490008E0C855F6FE04EE350E00E94F74B809169
:10D4A0008E0C90918F0C0F9731F48CE06FE04EE36F
:10D4B00050E00E94F74B80918E0C90918F0C40971A
:10D4C00061F48DE06FE04EE350E00E94F74B8CE09A
:10D4D0006FE04DE350E00E94F74B80918E0C9091ED
:10D4E0008F0C419791F48EE06FE04EE350E00E9484
:10D4F000F74B8DE06FE04DE350E00E94F74B8CE07E
:10D500006FE04CE350E00E94F74B80918E0C9091BD
:10D510008F0C0D9731F48AE16FE043E350E00E94F5
:10D52000F74B80918E0C90918F0C0C9761F489E1F0
:10D530006FE043E350E00E94F74B8AE16FE044E381
:10D5400050E00E94F74B8091CA0C9091CB0C892B34
:10D5500009F0C6C68091980C9091990C0E94595878
:10D5600080911D0C90911E0C029721F410921E0CBC
:10D5700010921D0C8091E60C9091E70C181619067C
:10D580009CF01092E70C1092E60C81E090E09093F2
:10D59000CB0C8093CA0C9093DD0C8093DC0C81E063
:10D5A00080931C0C0E946B658091BA0C9091BB0C0F
:10D5B000892B51F580910A0190910B01019741F45B
:10D5C0008091E80C9091E90C0F9711F40E941B6375
:10D5D00080910A0190910B01029741F48091E80C2F
:10D5E0009091E90C0A9711F40E941B6380910A0143
:10D5F00090910B01892B41F48091E80C9091E90CFA
:10D60000089711F40E941B6360918C0C70918D0C33
:10D6100080911A0C90911B0C0E9476727093930C5F
:10D620006093920C8091020190910301A0910401FA
:10D63000B09105010E97A109B1098093D80C909380
:10D64000D90CA093DA0CB093DB0C4196A11DB11D4F
:10D650008093DE0C9093DF0CA093E00CB093E10C70
:10D660008091DC0C9091DD0C019711F40E94925E88
:10D670008091DC0C9091DD0C892B09F055C58AE175
:10D6800064E045E150E00E94F74B8BE164E046E145
:10D6900050E00E94F74B2091920C3091930C8091B6
:10D6A000CE0C9091CF0C2817390709F077C0E09184
:10D6B000D40CF091D50C60918C0C70918D0CCF0135
:10D6C0000E9476727093970C6093960C2091C00C18
:10D6D0003091C10C6217730729F03196F093D50C85
:10D6E000E093D40C0E94CB5E80911D0C90911E0C97
:10D6F000892B39F58091900C6EE041E050E00E945A
:10D70000F74B8091900C8F5F6EE041E050E00E94FB
:10D71000F74B8091900C8E5F6EE041E050E00E94EC
:10D72000F74B8091900C8D5F6EE041E050E00E94DD
:10D73000F74B8091900C8E5F6EE04AE050E00E94C3
:10D74000F74B80911D0C90911E0C019739F580913B
:10D75000900C6EE041E050E00E94F74B8091900CFD
:10D760008F5F6EE041E050E00E94F74B8091900C9B
:10D770008E5F6EE041E050E00E94F74B8091900C8C
:10D780008D5F6EE041E050E00E94F74B8091900C7D
:10D790008E5F6EE04CE250E00E94F74B2091960CB9
:10D7A0003091970C8091C00C9091C10C28173907CB
:10D7B00031F40E94045F1092970C1092960C209105
:10D7C000920C3091930C8091CE0C9091CF0C281735
:10D7D000390709F4A9C48091C80C9091C90C892B10
:10D7E00009F04DC22091900C3091910C27313105F8
:10D7F0000CF0ADC080911D0C90911E0C892B09F08E
:10D800004FC0822F8C5F6EE041E050E00E94F74BEA
:10D810002091900C3091910CC9010897059738F030
:10D82000822F81506EE041E050E00E94F74B209142
:10D83000900C3091910CC9010897049730F0822F19
:10D840006EE046E050E00E94F74B2091900C309142
:10D85000910CC9010897039738F0822F8F5F6EE013
:10D8600047E050E00E94F74B2091900C3091910CD2
:10D87000C9010897029738F0822F8E5F6EE048E06A
:10D8800050E00E94F74B8091900C9091910C883061
:10D89000910531F08D5F6EE049E050E00E94F74B5A
:10D8A00080911D0C90911E0C019709F050C0809141
:10D8B000900C8C5F6EE041E050E00E94F74B2091AD
:10D8C000900C3091910CC9010897059738F0822F80
:10D8D00081506EE041E050E00E94F74B2091900CA7
:10D8E0003091910CC9010897049730F0822F6EE0B7
:10D8F00048E250E00E94F74B2091900C3091910C3F
:10D90000C9010897039738F0822F8F5F6EE049E2D4
:10D9100050E00E94F74B2091900C3091910CC9017E
:10D920000897029738F0822F8E5F6EE04AE250E04F
:10D930000E94F74B8091900C9091910C883091054A
:10D9400031F08D5F6EE04BE250E00E94F74B80912A
:10D95000EA0C9091EB0C883191050CF03EC08D5F84
:10D960006BE041E050E00E94F74B2091EA0C3091CF
:10D97000EB0CC9010997049730F0822F6BE041E06E
:10D9800050E00E94F74B2091EA0C3091EB0CC9015A
:10D990000997039730F0822F6BE045E250E00E9438
:10D9A000F74B2091EA0C3091EB0CC90109970297D3
:10D9B00038F0822F8F5F6BE046E250E00E94F74B19
:10D9C0008091EA0C9091EB0C8930910531F08E5FDB
:10D9D0006BE047E250E00E94F74B8091EE0C909193
:10D9E000EF0C893191050CF58E5F6CE041E050E061
:10D9F0000E94F74B2091EE0C3091EF0CC9010A9771
:10DA0000029730F0822F6CE045E250E00E94F74B25
:10DA10008091EE0C9091EF0C8A30910531F08F5F80
:10DA20006CE047E250E00E94F74B80911D0C909112
:10DA30001E0C892B09F060C08091900C9091910C84
:10DA40004A9731F48AE16EE046E050E00E94F74BDD
:10DA50008091900C9091910C499771F489E16EE05E
:10DA600046E050E00E94F74B8091900C8F5F6EE093
:10DA700047E050E00E94F74B8091900C9091910C00
:10DA80004897B1F488E16EE046E050E00E94F74B21
:10DA90008091900C8F5F6EE047E050E00E94F74B62
:10DAA0008091900C8E5F6EE048E050E00E94F74B52
:10DAB0008091900C9091910C4797F1F487E16EE082
:10DAC00046E050E00E94F74B8091900C8F5F6EE033
:10DAD00047E050E00E94F74B8091900C8E5F6EE023
:10DAE00048E050E00E94F74B8091900C8D5F6EE013
:10DAF00049E050E00E94F74B80911D0C90911E0C64
:10DB0000019709F060C08091900C9091910C4A9718
:10DB100031F48AE16EE048E250E00E94F74B8091D8
:10DB2000900C9091910C499771F489E16EE048E274
:10DB300050E00E94F74B8091900C8F5F6EE049E2BD
:10DB400050E00E94F74B8091900C9091910C489777
:10DB5000B1F488E16EE048E250E00E94F74B80911A
:10DB6000900C8F5F6EE049E250E00E94F74B80918D
:10DB7000900C8E5F6EE04AE250E00E94F74B80917D
:10DB8000900C9091910C4797F1F487E16EE048E298
:10DB900050E00E94F74B8091900C8F5F6EE049E25D
:10DBA00050E00E94F74B8091900C8E5F6EE04AE24D
:10DBB00050E00E94F74B8091900C8D5F6EE04BE23D
:10DBC00050E00E94F74B8091EA0C9091EB0C4A9741
:10DBD00031F48AE16BE045E250E00E94F74B80911E
:10DBE000EA0C9091EB0C499771F489E16BE045E206
:10DBF00050E00E94F74B8091EA0C8F5F6BE046E2A9
:10DC000050E00E94F74B8091EA0C9091EB0C489702
:10DC1000B1F488E16BE045E250E00E94F74B80915F
:10DC2000EA0C8F5F6BE046E250E00E94F74B809178
:10DC3000EA0C8E5F6BE047E250E00E94F74B809168
:10DC4000EE0C9091EF0C4A9731F48AE16CE045E2DA
:10DC500050E00E94F74B8091EE0C9091EF0C4997A9
:10DC600071F489E16CE045E250E00E94F74B80914D
:10DC7000EE0C8F5F6CE047E250E00E94F74B809122
:10DC8000C80C9091C90C019709F04EC22091900CDC
:10DC90003091910C2D3031050CF4ADC080911D0CEC
:10DCA00090911E0C892B09F04FC0822F81506EE09D
:10DCB00041E050E00E94F74B2091900C3091910C84
:10DCC000C9014797059738F0822F8C5F6EE041E0DD
:10DCD00050E00E94F74B2091900C3091910CC901BB
:10DCE0004897049738F0822F8D5F6EE049E050E04E
:10DCF0000E94F74B2091900C3091910CC9014997EB
:10DD0000039738F0822F8E5F6EE048E050E00E946B
:10DD1000F74B2091900C3091910CC9014A970297D2
:10DD200038F0822F8F5F6EE047E050E00E94F74BA3
:10DD30008091900C9091910C8B31910529F06EE0BF
:10DD400046E050E00E94F74B80911D0C90911E0C14
:10DD5000019709F050C08091900C81506EE041E035
:10DD600050E00E94F74B2091900C3091910CC9012A
:10DD70004797059738F0822F8C5F6EE041E050E0C6
:10DD80000E94F74B2091900C3091910CC90148975B
:10DD9000049738F0822F8D5F6EE04BE250E00E94D6
:10DDA000F74B2091900C3091910CC9014997039742
:10DDB00038F0822F8E5F6EE04AE250E00E94F74B0F
:10DDC0002091900C3091910CC9014A97029738F03C
:10DDD000822F8F5F6EE049E250E00E94F74B809106
:10DDE000900C9091910C8B31910529F06EE048E2F6
:10DDF00050E00E94F74B8091EA0C9091EB0C8D3033
:10DE000091050CF43FC081506BE041E050E00E946E
:10DE1000F74B2091EA0C3091EB0CC901489704971D
:10DE200038F0822F8D5F6BE041E050E00E94F74BAD
:10DE30002091EA0C3091EB0CC9014997039738F017
:10DE4000822F8E5F6BE047E250E00E94F74B2091FB
:10DE5000EA0C3091EB0CC9014A97029738F0822FF7
:10DE60008F5F6BE046E250E00E94F74B8091EA0C36
:10DE70009091EB0C8B31910529F06BE045E250E07D
:10DE80000E94F74B8091EE0C9091EF0C8D30910534
:10DE90000CF181506CE041E050E00E94F74B209182
:10DEA000EE0C3091EF0CC9014A97029738F0822F9F
:10DEB0008F5F6CE047E250E00E94F74B8091EE0CE0
:10DEC0009091EF0C8B31910529F06CE045E250E028
:10DED0000E94F74B80911D0C90911E0C892B09F02C
:10DEE00060C08091900C9091910C099731F48CE076
:10DEF0006EE049E050E00E94F74B8091900C9091C9
:10DF0000910C0A9771F48CE06EE048E050E00E94BA
:10DF1000F74B8091900C8D5F6EE049E050E00E94DD
:10DF2000F74B8091900C9091910C0B97B1F48CE091
:10DF30006EE047E050E00E94F74B8091900C8D5FBF
:10DF40006EE049E050E00E94F74B8091900C8E5FAC
:10DF50006EE048E050E00E94F74B8091900C909169
:10DF6000910C0C97F1F48CE06EE046E050E00E94DA
:10DF7000F74B8091900C8F5F6EE047E050E00E947D
:10DF8000F74B8091900C8D5F6EE049E050E00E946D
:10DF9000F74B8091900C8E5F6EE048E050E00E945D
:10DFA000F74B80911D0C90911E0C019709F060C0F9
:10DFB0008091900C9091910C099731F48CE06EE077
:10DFC0004BE250E00E94F74B8091900C9091910CA5
:10DFD0000A9771F48CE06EE04AE250E00E94F74B41
:10DFE0008091900C8D5F6EE04BE250E00E94F74B09
:10DFF0008091900C9091910C0B97B1F48CE06EE0B5
:10E0000049E250E00E94F74B8091900C8D5F6EE0EA
:10E010004BE250E00E94F74B8091900C8E5F6EE0D7
:10E020004AE250E00E94F74B8091900C9091910C45
:10E030000C97F1F48CE06EE048E250E00E94F74B60
:10E040008091900C8F5F6EE049E250E00E94F74BA8
:10E050008091900C8D5F6EE04BE250E00E94F74B98
:10E060008091900C8E5F6EE04AE250E00E94F74B88
:10E070008091EA0C9091EB0C0A9731F48CE06BE004
:10E0800047E250E00E94F74B8091EA0C9091EB0C34
:10E090000B9771F48CE06BE046E250E00E94F74B86
:10E0A0008091EA0C8E5F6BE047E250E00E94F74BF4
:10E0B0008091EA0C9091EB0C0C97B1F48CE06BE042
:10E0C00045E250E00E94F74B8091EA0C8F5F6BE0D5
:10E0D00046E250E00E94F74B8091EA0C8E5F6BE0C5
:10E0E00047E250E00E94F74B8091EE0C9091EF0CCC
:10E0F0000B9731F48CE06CE047E250E00E94F74B64
:10E100008091EE0C9091EF0C0C9771F48CE06CE028
:10E1100045E250E00E94F74B8091EE0C8F5F6CE07F
:10E1200047E250E00E94F74B20910001309101013D
:10E13000442737FD4095542F88E190E066E170E078
:10E140000E94C15889E190E066E170E047E20E94D8
:10E1500070588DE090E066E170E04CEE58E00E946F
:10E1600074582091060130910701409108015091A7
:10E17000090184E290E068E170E00E94C15888E102
:10E1800090E068E170E047E059E00E94745882E056
:10E1900090E068E070E041E259E00E94745884E049
:10E1A00090E069E070E04091E60C21E00E948F5819
:10E1B00086E090E069E070E045E20E94705880914E
:10E1C000D80C9091D90C9093C30C8093C20C82E030
:10E1D00090E06BE070E046E459E00E94745884E0FF
:10E1E00090E06CE070E04091C20C21E00E948F58FA
:10E1F00085E090E06CE070E047E20E9470588FE1AB
:10E2000090E068E070E048E259E00E94745882E2D1
:10E2100090E069E070E04091E40C21E00E948F58AA
:10E220008FE190E06BE070E042E159E00E947458A9
:10E2300082E290E06CE070E04091E80C21E00E9406
:10E240008F588091900C9091910C419721F52091DD
:10E25000F00C3091F10C4091F20C5091F30C8FE0E6
:10E2600090E068E170E00E94C1580E94D05920916E
:10E27000920C3091930C8091CE0C9091CF0C28177A
:10E28000390749F080911A0C90911B0C01969093DC
:10E290001B0C80931A0C8091900C9091910C4197DB
:10E2A000A9F08FE090E068E170E04091C40C21E0BB
:10E2B0000E948F588BE064E044E050E00E94F74BEE
:10E2C0008CE064E045E050E00E94F74B82E090E093
:10E2D00068E170E04BEF58E00E9474580E94D665E8
:10E2E00080911C0C882309F460C8C1E0D0E0D09371
:10E2F000CB0CC093CA0C80E00E94254C88709170B2
:10E30000892B09F452C881E060E941E00E9467511D
:10E31000D093CB0CC093CA0C1092DD0C1092DC0C85
:10E3200086E090E00E9459580E94E4630C94D569FD
:10E33000CF93DF930E94D14B8FE090E061E070E0DB
:10E340004CE751E90E9474588EE090E062E070E082
:10E3500041E751E90E94745881E090E064E070E088
:10E360004BE451E90E94745881E090E065E070E070
:10E3700045E251E90E94745881E090E066E070E067
:10E3800043E051E90E94745881E090E067E070E05A
:10E390004DED50E90E94745881E090E069E070E032
:10E3A00043ED50E90E94745881E090E06AE070E02B
:10E3B00049EB50E90E94745881E090E06BE070E016
:10E3C00045E950E90E94745881E090E06CE070E00B
:10E3D00049E750E90E94745881E090E06DE070E0F8
:10E3E00049E650E90E94745881E090E06EE070E0E8
:10E3F0004EE550E90E94745881E090E06FE070E0D3
:10E4000040E550E90E94745881E090E060E170E0DE
:10E4100041E450E90E94745881E090E060E170E0CE
:10E4200041E350E90E94745881E090E061E170E0BE
:10E4300044E150E90E94745881E090E063E170E0AB
:10E4400049E050E90E94745881E090E064E170E096
:10E450004AEF5FE80E94745881E090E065E170E067
:10E4600048EE5FE80E94745881E090E066E170E059
:10E470004AED5FE80E94745888E090E069E170E03E
:10E4800041EC5FE80E947458C1E0D0E080E00E9457
:10E49000254C80FFFBCF86E090E00E945958D09336
:10E4A000D10CC093D00C0E947C60F0CF991B79E016
:10E4B00004C0991F961708F0961B881F7A95C9F714
:10E4C00080950895AA1BBB1B51E107C0AA1FBB1F63
:10E4D000A617B70710F0A61BB70B881F991F5A95F0
:10E4E000A9F780959095BC01CD01089597FB092E61
:10E4F00007260AD077FD04D0E5DF06D000201AF405
:10E50000709561957F4F0895F6F7909581959F4F8F
:10E510000895A1E21A2EAA1BBB1BFD010DC0AA1F64
:10E52000BB1FEE1FFF1FA217B307E407F50720F07C
:10E53000A21BB30BE40BF50B661F771F881F991FF7
:10E540001A9469F760957095809590959B01AC0140
:10E55000BD01CF0108952F923F924F925F926F922B
:10E560007F928F929F92AF92BF92CF92DF92EF9263
:10E57000FF920F931F93CF93DF93CDB7DEB7CA1BE4
:10E58000DB0B0FB6F894DEBF0FBECDBF09942A880F
:10E59000398848885F846E847D848C849B84AA84B7
:10E5A000B984C884DF80EE80FD800C811B81AA8144
:10E5B000B981CE0FD11D0FB6F894DEBF0FBECDBF0F
:10E5C000ED010895A0E0B0E0E8EEF2E70C94B3723C
:10E5D000EC01A880B980CA80DB80A114B104C10419
:10E5E000D10441F484E2A82E89EDB82E8BE5C82E23
:10E5F00087E0D82EC601B5012DE133EF41E050E0B0
:10E600000E94627327EA31E440E050E00E944373C5
:10E610007B018C01C601B5012DE133EF41E050E0F3
:10E620000E946273CA01B9012CEE34EF4FEF5FEF25
:10E630000E9443736E0D7F1D801F911F97FF04C0C2
:10E640006150704080409048688379838A839B83BF
:10E650009B013F77C901CDB7DEB7EAE00C94CF72DA
:10E660000E94E27208958EE091E00E94E2720895A5
:10E67000A0E0B0E080930E0190930F01A0931001F1
:10E68000B09311010895629FD001739FF001829FA2
:10E69000E00DF11D649FE00DF11D929FF00D839F31
:10E6A000F00D749FF00D659FF00D9927729FB00DCE
:10E6B000E11DF91F639FB00DE11DF91FBD01CF01E1
:10E6C0001124089597FB092E05260ED057FD04D07E
:10E6D00020DF0AD0001C38F45095409530952195E4
:10E6E0003F4F4F4F5F4F0895F6F790958095709587
:0EE6F00061957F4F8F4F9F4F0895F894FFCF95
:10E6FE00680168010000F401000001000200010041
:02E70E00000009
:00000001FF
